:100000000C9440050C945B050C945B050C945B050B
:100010000C945B050C945B050C945B050C945B05E0
:100020000C945B050C9477180C945B050C945B05A1
:100030000C946D2C0C945B050C945B050C945B0587
:100040000C945B050C945B050C940B170C945B05EE
:100050000C940F0C0C945B050C94D60B0C945B0564
:100060000C949D1D0C945B050C94282B0C945B0543
:100070000C9479670C945B050C945B054B1E3E1E3B
:10008000321E181EFE1DDA1DEC1D4F21832080201C
:10009000DA1D6D20532033201320C11F6F1F571E00
:1000A0009D2B902BDD2BC12BB52B4E2B5F2B5F2B6C
:1000B000662B822B7D2B622B6A2B662B792B862B52
:1000C000622B6A2B662B752B8B2B622BEF2B0A0D69
:1000D000426174743A0020332043656C6C732020B5
:1000E0000020342043656C6C73202000204C6F7717
:1000F000207761726E696E67206C6576656C3A2058
:1001000025642E2564000A0D3D3D3D3D3D3D3D3DB0
:100110003D3D3D3D3D3D3D3D3D3D3D3D3D3D3D3D0F
:100120003D3D3D3D3D3D3D3D3D3D3D000A0D466C67
:1001300069676874436F6E74726F6C0A0D48617200
:1001400064776172653A25642E25640A0D536F66E3
:1001500074776172653A5625642E25642563200004
:100160000A0D74686520757365206F662074686970
:100170007320736F667477617265206973206F6E88
:100180006C79207065726D6974746564200A0D6FF6
:100190006E206F726967696E616C204D696B726F5A
:1001A0004B6F707465722D4861726477617265007F
:1001B0000A0D7777772E4D696B726F4B6F70746590
:1001C000722E646520286329204869537973746509
:1001D0006D7320476D6248000A0D3D3D3D3D3D3D3C
:1001E0003D3D3D3D3D3D3D3D3D3D3D3D3D3D3D3D3F
:1001F0003D3D3D3D3D3D3D3D3D3D3D3D3D000A0DCF
:1002000047656E65726174696E67206465666175C5
:100210006C74204D69786572205461626C65000AC7
:100220000D4D697865722D436F6E6669673A2027B8
:1002300025732720282575204D6F746F7273290050
:100240000A0D466F756E6420424C2D4374726C3AF1
:100250002000256420000A0D0A0D2121204D49535C
:1002600053494E4720424C2D4354524C3A2025646A
:10027000202121000A0D3D3D3D3D3D3D3D3D3D3DA3
:100280003D3D3D3D3D3D3D3D3D3D3D3D3D3D3D3D9E
:100290003D3D3D3D3D3D3D3D3D000A0D496E69748E
:1002A0002E20454550524F4D003A2047656E6572ED
:1002B0006174696E672044656661756C742D506168
:1002C00072616D65746572207573696E67206F6CFD
:1002D0006420537469636B2053657474696E67732B
:1002E000000A0D466C696768742D74696D65202578
:1002F00075206D696E2020546F74616C3A257520ED
:100300006D696E000A0D414343206E6F7420636176
:100310006C696272617465642021000A0D5573690D
:100320006E6720706172616D6574657273657420AB
:100330002564000A0D43616C6962726174696E67BD
:100340002070726573737572652073656E736F725A
:100350002E2E004F4B0A0D000A0D436F6E74726F04
:100360006C3A200048656164696E67486F6C640090
:100370004E6F726D616C20284143432D4D6F646553
:1003800029000A0D3D3D3D3D3D3D3D3D3D3D3D3D51
:100390003D3D3D3D3D3D3D3D3D3D3D3D3D3D3D3D8D
:1003A0003D3D3D3D3D3D3D0A0D002E000A0D2044E2
:1003B0004143206F7220493243204552524F52210F
:1003C00020436865636B204932432C2033567265A5
:1003D000662C2044414320616E6420424C2D4374BE
:1003E000726C005B25695D005B25695D002B204D0B
:1003F000696B726F4B6F70746572202B0048573AAF
:100400005625642E25642053573A25642E256425ED
:10041000632D41727468757220500053657474695D
:100420006E673A25642025730049324320455252B5
:100430004F52212121004D697373696E6720424C30
:100440002D4374726C3A25642121002863292048C9
:100450006F6C676572204275737300486F656865DD
:100460003A202020202025356900536F6C6C486F9E
:100470006568653A20253569004C75667464727547
:10048000636B3A20253569004F66662020202020C6
:10049000203A20253569004B65696E65200048F6D5
:1004A00068656E726567656C756E6700616B742E4A
:1004B000204C616765004E69636B3A202020202044
:1004C0002025356900526F6C6C3A202020202020B6
:1004D000253569004B6F6D706173733A20202025BC
:1004E0003569004B313A25346920204B323A2534A6
:1004F0006920004B333A25346920204B343A2534A7
:100500006920004B353A25346920204B363A253492
:100510006920004B373A25346920204B383A25347E
:100520006920004E693A2534692020526F3A2534FB
:1005300069200047733A253469202047693A2534F9
:1005400069200050313A253469202050323A253450
:1005500069200050333A253469202050343A25343C
:100560006920004779726F202D2053656E736F727A
:10057000004E69636B2025346920282533692E25B8
:10058000692900526F6C6C20253469202825336955
:100590002E256929004769657220253469202825A0
:1005A000336929004E69636B20253469202825337F
:1005B000692E25782900526F6C6C2025346920281B
:1005C0002533692E2578290047696572202534690D
:1005D000202825336929004E69636B202534692062
:1005E0002825336929282533692900526F6C6C202E
:1005F00025346920282533692928253369290047AE
:100600006965722025346920282533692928253316
:10061000692900414343202D2053656E736F72009A
:100620004E69636B202534692028253369290052DF
:100630006F6C6C2025346920282533692900486FA8
:1006400063682025346920282533692900566F6C9A
:10065000746167653A2020202535690052432D4C8E
:100660006576656C3A20202535690052432D436834
:10067000616E6E656C733A253469004B6F6D706105
:100680007373202020202020200052696368747535
:100690006E673A2020253569004D65737377657262
:1006A000743A20202535690053746172743A202011
:1006B00020202025356900506F7469313A202025AB
:1006C000336900506F7469323A2020253369005035
:1006D0006F7469333A202025336900506F74693490
:1006E0003A202025336900536572766F202000532D
:1006F0006574706F696E74202025336900537465CA
:100700006C6C756E673A202533690052616E6765BF
:100710003A2533692D2533690045787465726E4337
:100720006F6E74726F6C2020004E693A2534692018
:1007300020526F3A253469200047733A25346920E6
:100740002047693A253469200048693A25346920F0
:100750002043663A2534692000424C2D4374726C64
:10076000204572726F72732000202533642020258B
:100770003364202025336420202533642000202585
:100780003364202025336420202533642020253342
:100790006420002025336420202533642020253365
:1007A0006420202533642000424C2D4374726C2059
:1007B000666F756E6420002025632020202563204D
:1007C0002020256320202025632000202563202071
:1007D0002025632020202563202020256320002061
:1007E00025632020202D2020202D2020202D0031A9
:1007F0003000313100313200466C696768742D5425
:10080000696D652020002020202020202535756D71
:10081000696E00546F74616C3A2535756D696E00B0
:1008200028726573657429000A0D506C65617365E3
:1008300020636F6E6E656374205370656B747275A0
:100840006D20726563656976657220666F722062DD
:10085000696E64696E67204E4F572E2E2E006F6BA7
:100860002E0A0D0054696D656F75742E0A0D000017
:10087000010203040405060708090A0B0B0C0D0E00
:100880000F101111121314151516171818191A1B19
:100890001B1C1D1D1E1F1F20212122232324242554
:1008A00025262727282829292A2A2B2B2C2C2D2DB1
:1008B0002D2E2E2F2F303030313132323233333330
:1008C00034343435353536363637373737383838C7
:1008D000393939393A3A3A3A3B3B3B3B3C3C3C3C70
:1008E0003C3D3D3D3D3E3E3E3E3E3F3F3F3F3F3F28
:1008F00040404040404041414141414142424242EA
:1009000042424243434343434343444444444444B4
:100910004444454545454545454545464646464684
:10092000464646464747474747474747474747485A
:100930004848484848484848484849494949494931
:1009400049494949494949494A4A4A4A4A4A4A4A0F
:100950004A4A4A4A4A4A4B4B4B4B4B4B4B4B4B4BED
:100960004B4B4B4B4B4B4B4C4C4C4C4C4C4C4C4CCE
:100970004C4C4C4C4C4C4C4C4C4C4D4D4D4D4D4DB1
:100980004D4D4D4D4D4D4D4D4D4D4D4D4D4D4D4D97
:100990004E4E4E4E4E4E4E4E4E4E4E4E4E4E4E4E77
:1009A0004E4E4E4E4E4E4E4E4E4E4F4F4F4F4F4F61
:1009B0004F4F4F4F4F4F4F4F4F4F4F4F4F4F4F4F47
:1009C0004F4F4F4F4F4F4F4F4F00008F001E01AD05
:1009D000013B02CA025803E603740402058F051B9B
:1009E00006A7063307BE074808D2085B09E3096B70
:1009F0000AF20A780BFD0B810C040D860D070E8799
:100A00000E060F840F00107B10F5106E11E5115BC0
:100A100012CF124213B31323149214FE146A15D387
:100A2000153B16A11605176717C81727188318DE78
:100A30001837198E19E319361A871AD61A231B6E1E
:100A40001BB61BFD1B411C831CC31C001D3C1D75DC
:100A50001DAB1DE01D121E421E6F1E9A1EC31EE915
:100A60001E0D1F2E1F4D1F691F841F9B1FB01FC30C
:100A70001FD31FE11FEC1FF51FFB1FFF1F002000EE
:100A800011241FBECFEFD0E1DEBFCDBF13E0A0E049
:100A9000B1E0E8E6F8ED02C005900D92A63DB10781
:100AA000D9F71AE0A6EDB3E001C01D92A931B10754
:100AB000E1F70C948C060C940000282FFB01815068
:100AC000853008F023E0842F9927332721503040C8
:100AD000829FD001839FB00D929FB00D1124AC591D
:100AE000BF4F019724F00E94166C0192FACF0E942A
:100AF000D1650895863038F085E0A2E0B0E0082E98
:100B00000E94236C08958823C1F70895582F8630DA
:100B100048F155E0842F9927252F33272150304065
:100B2000829FD001839FB00D929FB00D1124AC59CC
:100B3000BF4FFB01019724F001900E94236CFACF74
:100B4000A2E6B0E0042E0E94236CA0E5B0E088E0AD
:100B5000FB01182E0E942F6C852F0E947A050E949F
:100B6000D16508958823B1F60895CF93A2E0B0E04F
:100B70000E94166C802DC82F8150853020F0C3E074
:100B80008C2F0E947A058C2F9927CF910895809100
:100B9000E108E82FFF27EE0FFF1FE155F74F808197
:100BA00091818D5E9F4F14F010920301808191819D
:100BB0008A5B9F4F24F480910301882319F02091D0
:100BC0007E0717C081E08093030120917E07280FE4
:100BD00020937E07253038F088EE93E09093FC0355
:100BE0008093FB0306C066E970E0822F0E948E317D
:100BF000E6CF822F992790934C0880934B08089555
:100C00001F93CF93DF93182F882351F48091FF080F
:100C10008233A0F080930001112309F479C038C019
:100C20008EEC90E09F938F931F920E9476140F900A
:100C30000F900F908091FF08823360F784EF91E06E
:100C40000E94F517EC01112309F042C0809127039F
:100C500090912803823891050CF046C08091FF08DE
:100C600023E0829FC0011124809300011123A1F28F
:100C700068EC70E0822F0E948E3186ED90E09F93A9
:100C80008F931F920E9476140F900F900F90C4CFF5
:100C9000809100016AE00E94A66B892F99279F939B
:100CA0008F93809100010E94A66B99279F938F9349
:100CB0008CEE90E09F938F931F920E9476148DB7D5
:100CC0009EB707960FB6F8949EBF0FBE8DBF20C08B
:100CD000CE010E94FE17882309F0B8CFCE010E94F2
:100CE000FE178823A9F3B2CF8091FF089927880FB8
:100CF000991F880F991F80930001112309F48CCF4D
:100D000068EC70E084E00E948E3181EE90E0B7CF15
:100D1000DF91CF911F910895CFEFD0E1DEBFCDBF1E
:100D2000EE24FF2414B815B8C7EED3E0E297D7FF3E
:100D3000FDCF189B6FC1199B78C12DE02093020154
:100D400081E887B93E9A8FEF88B98BE184B981E059
:100D500085B98EE38AB987E48BB9469A84B7877FD1
:100D600084BF809160008861809360001092600071
:100D700080ED97E09093FC038093FB031092D804DE
:100D80001092D7041092B4081092B3081092DA04AB
:100D90001092D9041092DC041092DB04243108F480
:100DA0003FC188E894E0A0E0B0E080938603909390
:100DB0008703A0938803B09389032A3009F465C19F
:100DC000243109F462C1289A0E9460180E943118E7
:100DD0000E944B110E94582C0E946B1C0E94E72A13
:100DE0000E940662789486E091E09F938F931F9211
:100DF0000E9476140F900F900F9087E690E09F93DB
:100E00008F938CE490E09F938F931F921F92809119
:100E100002016AE00E94A66B892F99279F938F9306
:100E2000809102010E94A66B99279F938F938CE279
:100E300091E09F938F931F920E9476148DB79EB777
:100E40000D960FB6F8949EBF0FBE8DBF80E691E061
:100E50009F938F931F920E9476140F900F900F9084
:100E600080EB91E09F938F931F920E9476140F90D6
:100E70000F900F9088ED91E09F938F931F920E94A7
:100E800076148091C8000F900F900F90803209F473
:100E9000F4C0809102018C3008F0C0C0299A49E06A
:100EA00061EE78E083E00E945D05C8EED3E0DE01EC
:100EB0000E94166C802D813009F4B9C08EEF91E04C
:100EC0009F938F931F920E9476140F900F900F9014
:100ED00023ED35E0F9018FE0158616861786108A16
:100EE0008150349687FFF8CF80E48093E0058093AB
:100EF000E1051092E2058093E3058093E40590EC10
:100F00009093E5051092E6058093E7058093E80548
:100F10001092E9059093EA059093EB058093EC0518
:100F20001092ED058093EE059093EF0581E080939C
:100F3000D30544ED55E08BE0E4E0F1E0DA01019007
:100F40000D928A95E1F78DE4DE01F901182E0E94D9
:100F50002F6C8091850399279F938F935F934F9375
:100F60008FE192E09F938F931F920E9476148DB72A
:100F70009EB707960FB6F8949EBF0FBE8DBF80E454
:100F800092E09F938F931F920E94761410924704D1
:100F90001092FF030E947B3F0F900F900F90809163
:100FA000FF038823E1F31092470480ED97E00E944D
:100FB000F517EC01CC24DD2472E5A72E72E0B72EE4
:100FC0001092FF030E947B3F8091FF038823E1F38F
:100FD000F601EE0FFF1FEE0FFF1FED52FA4F858552
:100FE00018160CF054C086010E55174FCE010E9402
:100FF000FE17882309F04EC0D8018C91882309F090
:1010000049C08093FF030E947B3F8091FF038823A8
:10101000E1F3ECCF199B2FC024E190CE29983FCF6C
:101020008BE095E0A0E0B0E0C0CE2BE087CEA1E061
:10103000B0E00E94166C802D8F3F09F43FCF1092D4
:10104000850323ED35E08DE4DE01F901182E0E94C1
:101050001E6C90918503F9013D962FE080813496B6
:1010600018160CF49F5F215027FFF8CF909385034B
:1010700044ED55E06ECF2AE061CE8091CA00863003
:1010800009F007CF0E94806604CF28989DCE860184
:101090000E55174FF8018081882309F03FC0860163
:1010A0000F5F1F4F68010C30110508F489CFCC2465
:1010B000DD2456E5A52E52E0B52EC1E025C0F6018F
:1010C000EE0FFF1FEE0FFF1FED52FA4F858518162A
:1010D0000CF586010F5F1F4F1F930F93BF92AF92C6
:1010E0009F930E947614C093F9030F900F900F9076
:1010F0000F900F9086E898E0C80ED91ED6011C927A
:1011000068010C301105D0F4F601EE55F74F9081CF
:101110009923A9F286010F5F1F4FECCF86010F5F65
:101120001F4F1F930F93BF92AF921F920E9476148E
:101130000F900F900F900F900F90B4CF84E792E034
:101140009F938F931F920E9476140E947B3F0F9073
:101150000F900F90A1E0B0E00E94166C802D8035BA
:1011600009F029C20EE010E0D8010E94166C802D13
:101170009927582F442748010894811C911CD401B9
:101180000E94166C802D480F511DECEFAE2EEFEF34
:10119000BE2EA00EB11ED5010E94166C802D99277F
:1011A000382F22276DEFC62E6FEFD62EC00ED11E20
:1011B000D6010E94166C802D280F311DEFEF2F3FB6
:1011C0003E0709F4B9C2FFEF4F3F5F0709F4B4C20D
:1011D0003093D7032093D6035093D9034093D80379
:1011E0008091D6039091D7039F938F938091D803DA
:1011F0009091D9039F938F9381EE92E09F938F9369
:101200001F920E9476148DB79EB707960FB6F8947A
:101210009EBF0FBE8DBFA4E0B0E00E94166C802D73
:10122000853008F0B8C20E94B50545E661EE78E069
:101230000E945D050E94B50599279F938F938BE1CE
:1012400093E09F938F931F920E9476148091E908F8
:101250000F900F900F900F900F9080FD7BC20E9417
:10126000D53C809102018A3009F472C2843109F4BC
:101270006FC2289A80ED97E09093FC038093FB0364
:1012800085E58093800788E593E09F938F931F9275
:101290000E9476148091E9080F900F900F9082FFC2
:1012A00054C284E693E09F938F931F920E9476141A
:1012B0000F900F900F900E94322288E893E1909354
:1012C000AD038093AC0381E080937F070E9400060A
:1012D00082E893E09F938F931F920E94761480ED93
:1012E00097E00E94F517EC010F900F900F908091FE
:1012F000FF03882309F4A1C080911903882309F40E
:101300009CC01092FF0380917E07882309F4D0C00F
:101310000E94C7050E947B3F209102012A3009F4F8
:10132000D0C0243109F4CDC0289A8091DE048823EE
:1013300009F4CDC08091DE0481508093DE04809159
:10134000C205882369F081508093C205882341F447
:101350001092C0051092BF051092BE051092BD05F7
:101360008091AC039091AD0301979093AD0380936E
:10137000AC038091AC039091AD03892B29F080914F
:101380004604882309F4D7C08091AC039091AD0343
:10139000892B09F4D6C080911203909113038F5FBB
:1013A0009F4F09F4E7C08091FF03882321F08091CB
:1013B000D404882311F40E9487110E94700ECE017C
:1013C0000E94FE178823B9F1649680910F03882349
:1013D00009F489C0815080930F0380910001282F68
:1013E00033278091270390912803821793070CF0ED
:1013F00074C08091AD0480628093AD04809112032B
:10140000909113038F5F9F4F09F4C8C00E94F86446
:1014100084E08093FA038091D404882321F45AEA6B
:10142000E52E55E0F52E0894E11CF11CF2E7EF16CD
:10143000FBE0FF0651F00E94E0658091FA038823EB
:1014400009F055CF0E943C6552CFEE24FF24209135
:10145000D8033091D9032F5F3F4F3093D9032093A6
:10146000D8038091D6039091D70301969093D70328
:101470008093D603832F9927D801082E0E94236CCE
:101480008091D803D401082E0E94236C8091D70349
:10149000D501082E0E94236C8091D603D601082E18
:1014A0000E94236C84E190E00E94F517EC01C3CF09
:1014B0000E9494430E947B3F209102012A3009F050
:1014C00030CF28988091DE04882309F033CF8091B3
:1014D0006F00806280936F0032CF8091AD048F7D6A
:1014E0008093AD0493CF80938A071092B904109231
:1014F000B8041092B7041092B6041092B50410927A
:10150000B40480911203909113038F5F9F4F09F0F1
:1015100064CF8091DE04882309F05FCF88E99AE3E5
:101520009093FC038093FB0380E09CE09093130373
:101530008093120352CF2A3079F1243169F1289A2D
:1015400032CF0E94FD2A85E090E09093AD03809316
:10155000AC0380915D0890915E08019690935E08BF
:1015600080935D0880911203909113038F5F9F4FCA
:1015700009F019CF8091D404882309F414CF80E1B5
:1015800097E29093FC038093FB0380E890E09093B4
:1015900013038093120307CF289805CF80E797E1C4
:1015A0009093FC038093FB0380E093E090931303FC
:1015B000809312032BCF0E94F92E8AE992E09F9329
:1015C0008F931F920E94761431E0932E0F900F900C
:1015D0000F90C0E5D0E08E010F5F1F4F22E0C22EBA
:1015E000D12CCC0EDD1E93E0A92EB12CAC0EBD1E6D
:1015F00084E0682E712C6C0E7D1EB5E04B2E512CB4
:101600004C0E5D1EA6E02A2E312C2C0E3D1EE2E073
:101610009E1609F48BC0F3E09F1609F48AC023E0FC
:10162000291508F483C080910201843168F085E0B7
:101630008093FC0810921A098BE18093F8088EE4DD
:101640008093170980931809DE010E94166C802D83
:101650008C3008F068C0D8010E94166C802D8C3048
:1016600008F061C0D6010E94166C802D8C3008F005
:101670005AC0D5010E94166C802D8C3008F053C0E2
:10168000DE010E94166C802D8093E108D8010E9433
:10169000166C802D8093E208D6010E94166C802D76
:1016A0008093E308D5010E94166C802D8093E40896
:1016B000D3010E94166C802D8093E508D2010E9410
:1016C000166C802D8093E608D1010E94166C802D47
:1016D0008093E708A7E5B0E00E94166C802D809308
:1016E000E80881E0981651F4A9EAB2E0BF93AF93FD
:1016F0001F920E9476140F900F900F9045E661EEB6
:1017000078E0892D0E9486059394B5E0B91508F01C
:101710007ECF83E00E947A0580E5A1E0B0E0082E4C
:101720000E94236C1FCD0E94E02EE8CF0E94C62F9E
:101730007ACF0E94913077CF1092D9031092D803BC
:101740001092D7031092D6034BCD80E793E0ABCD38
:10175000289890CD83E393E09F938F931F920E94EC
:10176000761488EE93E00E94F517EC010E94711C3C
:101770000F900F900F90CE010E94FE178823D9F38F
:1017800083E593E09F938F931F920E9476140F90AE
:101790000F900F9064CD84E093E09F938F931F92FE
:1017A0000E9476140F900F900F903DCD1F920F92D4
:1017B0000FB60F9211248F939F93EF93FF93809115
:1017C00011038823A9F48091ED039091EE03019613
:1017D000FC01E05DF94FE081ED3079F0863991054B
:1017E00061F09093EE038093ED03E093C6000EC08A
:1017F0001092EE031092ED0309C01092EE031092C6
:10180000ED0381E080931103E093C600FF91EF9117
:101810009F918F910F900FBE0F901F9018951F9260
:101820000F920FB60F9211242F933F934F935F9314
:101830008F939F93AF93BF93EF93FF9390E080912B
:10184000C6008093E5035091F303563910F090934E
:10185000F4038091E5038D3091F02091F403822F01
:1018600099278130910509F46CC0823091050CF400
:101870008EC0029709F47FC01092F403A8C0209193
:10188000F403223061F79093F403852F992783574F
:10189000984FFC01329740812091EF033091F00383
:1018A000241B3109DC0111978C91281B3109C901D6
:1018B0009F709093F0038093EF030024880F991F8B
:1018C000001C880F991F001C892F902D982F935C66
:1018D0009093F1032F733070235C2093F203808187
:1018E000891709F46EC090E08091E2038F5F8093C6
:1018F000E2033091E403332309F069C0992309F42A
:1019000066C081E08093E403580F5093E103515087
:10191000E52FFF27E357F84F8DE0808380918F07F5
:10192000823509F054C088E190E02CE00FB6F894BD
:10193000A895809360000FBE209360003093F90358
:1019400046C02F5F2093F403E52FFF27E357F84F9E
:101950008091E50380835F5F5093F3032091E5035B
:101960008091EF039091F003820F911D9093F0030B
:101970008093EF032CC0E52FFF27E357F84F8091AA
:10198000E5038083563938F31092F403E7CF892BAF
:1019900009F072CF8091E503833259F08091E5031D
:1019A00080938D0781E08093F3038091E50399276D
:1019B000DDCF8091E403882389F781E08093F403ED
:1019C000EDCF8C91821709F08ECF91E092CFFF91ED
:1019D000EF91BF91AF919F918F915F914F913F9107
:1019E0002F910F900FBE0F901F901895AC01A0E0A3
:1019F000B0E09D01A817B90748F4E0E3F6E0819153
:101A0000280F311D1196A417B507C8F33F70FD01CB
:101A1000E05DF94FC9010024880F991F001C880F51
:101A2000991F001C892F902D835C80831196FD01E6
:101A3000E05DF94F2F733070822F835C8083AF5C41
:101A4000B94F8DE08C9310921103809130068093F2
:101A5000C6000895BF92CF92DF92EF92FF920F934C
:101A60001F93CF93DF93CDB7DEB72C859D857E8501
:101A7000BB2483E2809330069F59909331062093D4
:101A8000320603E010E0772309F4ADC0CF84D88894
:101A900043E1E42EF12CEC0EFD1EA989BA897150A8
:101AA000109709F4A0C0109709F43CC0F601EB0DA3
:101AB000F11DB3949081119789F47723A1F1F70177
:101AC00022E030E0E20EF31ED701C080D180E20EAA
:101AD000F31E0D90BC91A02DBB247150109719F1ED
:101AE000F601EB0DF11DB3944081119709F466C026
:101AF0001097D1F0F601EB0DF11DB39460811197B1
:101B0000A1F4772391F0F7013296D701CD90DC90C4
:101B100032E0E32EF12CEE0EFF1EA081B181BB243A
:101B2000715003C090E040E060E0F801E05DF94FE3
:101B3000892F86958695835C80830F5F1F4FF80100
:101B4000E05DF94F892F9927837090708295929567
:101B5000907F9827807F982755279A013295229564
:101B60002F7023273F702327822B835C80830F5F96
:101B70001F4FF801E05DF94F4F705070440F551F33
:101B8000440F551F862F99270024880F991F001C8A
:101B9000880F991F001C892F902D842B835C8083D4
:101BA0000F5F1F4FF801E05DF94F6F73635C608357
:101BB0000F5F1F4F109709F076CF15C0772309F4F8
:101BC000B3CFF701A2E0B0E0EA0EFB1ED701C08060
:101BD000D18022E030E0E20EF31E0D90BC91A02DEA
:101BE000BB24715085CFC8010E94F60CDF91CF91C4
:101BF0001F910F91FF90EF90DF90CF90BF900895CD
:101C0000A3E07A2F4091E103465009F45FC0E72F2B
:101C1000FF27E357F84F80818D537F5FE72FFF2722
:101C2000E357F84F20812D537F5FE72FFF27E357BE
:101C3000F84F30813D537F5FE72FFF27E357F84F81
:101C400060816D537F5F9927880F991F880F991FB7
:101C5000522F52955F70582B822F99278F7090705A
:101C600082959295907F9827807F9827232F26959D
:101C70002695282B832F99278370907000249695A2
:101C800087950794969587950794982F802D682BB4
:101C900041504F3FD9F0EA2FFF27E357F84F5083C9
:101CA000AF5F41504F3F91F0EA2FFF27E357F84FC6
:101CB0002083AF5F41504F3F49F0EA2FFF27E357A2
:101CC000F84F6083AF5F442309F0A1CF80E997E02C
:101CD0009093E0038093DF03A350A093DE03089565
:101CE000CF93DF93CDB7DEB722970FB6F894DEBF60
:101CF0000FBECDBF8091E403882309F4AFC20E94D8
:101D0000000E80918E07823609F471C080918F0792
:101D100099278436910509F457C08536910584F5D5
:101D20008136910509F44EC1823691050CF4C2C08A
:101D30008236910509F49AC183369105C1F48091E8
:101D4000DA039091DB03892B09F04FC2A091DF03E6
:101D5000B091E0039C91992309F03DC29C918AE0E7
:101D6000989FC00111249093DB038093DA031092B3
:101D7000E4031092E0031092DF031092DE036EC2C0
:101D80008C36910509F410C18D3691050CF0B3C065
:101D90008736910509F42BC18836910541F78FEFFD
:101DA00080930F03E091DF03F091E0038081909135
:101DB0003F04892B80933F04882311F01092E6039F
:101DC00081E08093EA03D3CFE091DF03F091E00359
:101DD00090818AE0989FC001112490930D03809315
:101DE0000C03892B21F281E08093E903C0CF80911D
:101DF0008F0799278037910509F4F2C08137910543
:101E00000CF485C08337910509F45BC184379105D3
:101E10000CF03CC18137910509F078CFA091DF0328
:101E2000B091E0038C918F3F09F40CC28C91882310
:101E300009F003C281E08C93A091DF03B091E0032D
:101E400045E661EE78E08C910E945D05809111037A
:101E50008823E1F3E091DF03F091E003808189833F
:101E600080E58A8385E690E09F938F9381EE98E0EA
:101E70009F938F9321E030E03F932F93CE01029602
:101E80009F938F933F932F93CE01820F931F9F9326
:101E90008F9383E08F9381E08F9381E58F930E94EE
:101EA0002A0DADB7BEB71F960FB6F894BEBF0FBED2
:101EB000ADBF2CCF8B34910509F059CFE091DF03F2
:101EC000F091E003808191819093F0048093EF047E
:101ED0002091ED043091EE04821B930B845E9D4FA4
:101EE00068E671E00E94C66B845B90409093EC04BE
:101EF0008093EB043CCF8437910509F47CC086378E
:101F0000910509F034CF81E08093E80330CF8D361E
:101F1000910529F18E3691050CF093C08B34910513
:101F200009F0F4CEA091DF03B091E0038D919C9174
:101F30009093F0048093EF042091ED043091EE042F
:101F4000821B930B845E9D4F68E671E00E94C66B16
:101F5000845B90409093EC048093EB04D7CE809107
:101F600011038823E1F3A091DF03B091E0039C917A
:101F7000913009F43FC1198281E090E09F938F93E3
:101F8000CE0101969F938F9381E08F938F938DE481
:101F90008F930E942A0D8DB79EB707960FB6F894BF
:101FA0009EBF0FBE8DBFB2CE8FEF80930F03E09127
:101FB000DF03F091E00380818093400481E080930F
:101FC000EB03D5CEE091DF03F091E003E081E03256
:101FD00058F08FE1809310038FEF80930F03C7CEEB
:101FE00081E08093E70392CEE0931003F5CF81E088
:101FF0008093EC03BCCE8091E103853108F4DAC014
:10200000E091DF03F091E00380E1A8E6B7E0019002
:102010000D928A95E1F7809111038823E1F31F92D5
:1020200080910E038F9384E58F930E942A0D8AEF8F
:102030008093DC038FEF80930F030F900F900F902E
:1020400096CE8E36910509F061CE809111038823DA
:10205000E1F38DE490E09F938F9383ED95E09F9360
:102060008F9381E08F938F938EE492CFA091DF03C3
:10207000B091E0038BE0E0E8F7E00D9001928A95E3
:10208000E1F78091890780936508A6CF8437910591
:1020900009F03CCE8091E103853108F4BCC0A091E9
:1020A000DF03B091E00380E1E8E6F7E00D900192F4
:1020B0008A95E1F780EF8093DC038FEF80930F0325
:1020C00025CE2091DF033091E003F901808181501A
:1020D000853018F481818035E9F0198280911103EF
:1020E0008823E1F381E090E09F938F93CE010196E6
:1020F0009F938F9381E08F938F9383E58F930E94BB
:102100002A0DEDB7FEB737960FB6F894FEBF0FBE97
:10211000EDBFFCCD61EE78E085E62E5F3F4FDB0141
:10212000F901982F01900D929A95E1F722503040D5
:10213000482FD9018C910E94860580911709992713
:10214000AA27BB27BC01CD0124EC39E040E050E0D8
:102150000E94876BDC01CB018093A6039093A703B9
:10216000A093A803B093A903809118099927AA27DF
:10217000BB27BC01CD010E94876BDC01CB018093A2
:10218000A2039093A303A093A403B093A503E091AB
:10219000DF03F091E00380810E947A050E94B5057B
:1021A000898380E00E9400066EE670E089810E94CB
:1021B0008E3194CFE091DF03F091E0038081918133
:1021C000A281B3818093680790936907A0936A07FF
:1021D000B0936B0720CF8AE0989FC00111240E9422
:1021E000F51790932F0680932E06A091DF03B091F0
:1021F000E003B4CD43ED55E08DE4FA01282F0D90B6
:1022000001922A95E1F7A8EEB3E0FA01182E0E9498
:102210002F6C9983B1CEA091DF03B091E0038D9133
:102220009D910D90BC91A02D8093680790936907B4
:10223000A0936A07B0936B073DCF863008F400CEB9
:1022400085E0F9CD0E94B505E091DF03F091E00350
:102250008083A091DF03B091E003E8CD22960FB612
:10226000F894DEBF0FBECDBFDF91CF910895CF931D
:10227000C82F8A3029F08091C00085FFFCCF04C0B0
:102280008DE00E943711F7CFC093C60080E090E048
:10229000CF910895089588E18093C1008091C00096
:1022A00082608093C0008091C10080688093C100EB
:1022B0008091C10080648093C1008AE28093C40051
:1022C00080910C0390910D030E94F51790935D0788
:1022D00080935C078CED90E00E94F51790938C073B
:1022E00080938B0710925E078CE480935F0786E0F3
:1022F000809362078AE08093600781E080936107A2
:102300001092E0031092DF031092DE030895EF9223
:10231000FF920F931F9380911103882309F478C2D1
:102320008091EA03882309F082C08091EB0388231F
:1023300029F080911103882309F07FC18091E8037F
:10234000882329F080911103882309F05BC18091D3
:10235000EC03882329F080911103882309F036C10A
:1023600080918B0790918C070E94FE17882329F09B
:1023700080911103882309F0C8C080910C039091CB
:102380000D03892B09F084C18091E903882329F08A
:1023900080911103882309F00FC28091DA03909194
:1023A000DB03892B09F07EC1209110032F3F59F1E7
:1023B00080E190E09F938F93822F99278295929549
:1023C000907F9827807F9827845F9E4F9F938F935D
:1023D00081E090E09F938F9380E193E09F938F93B0
:1023E00082E08F9381E08F9381E48F930E942A0D86
:1023F0008FEF809310038DB79EB70B960FB6F894AE
:102400009EBF0FBE8DBF80916508882329F0809103
:102410001103882309F05EC08091E703882309F443
:10242000F7C180911103882309F4F2C139C080916A
:102430001103882309F479CF0E943B2284E190E0C4
:102440009F938F939091E60384E1989FC00111249C
:10245000865D9C4F9F938F9381E090E09F938F9335
:1024600086EE93E09F938F9382E08F9381E08F932A
:1024700088E48F930E942A0D8091E6038F5F2DB729
:102480003EB7255F3F4F0FB6F8943EBF0FBE2DBF3E
:10249000843008F4B8C11092E6031092EA0345CFE5
:1024A00086E190E09F938F938FEA98E09F938F93BC
:1024B00081E08F938F9380E58F930E942A0D109275
:1024C000E7038DB79EB707960FB6F8949EBF0FBE71
:1024D0008DBF9EC181E090E09F938F9385E698E049
:1024E0009F938F9381E08F938F9382E48F930E94C9
:1024F0002A0D109265082DB73EB7295F3F4F0FB6E2
:10250000F8943EBF0FBE2DBF87CF8091F808992762
:10251000880F991F880F991F7C010027F7FC0095F1
:10252000102F8091290590912A05A0912B05B0913B
:102530002C05BC01CD01A80197010E94FB6B3093D3
:102540007907209378078091210590912205A09129
:102550002305B0912405BC01CD01A80197010E947B
:10256000FB6B30937B0720937A078091C1048093A3
:102570007C078091C00480937D0788E090E09F9362
:102580008F9388E797E09F938F9381E08F9383E009
:102590008F9387E78F930E942A0D80917E072DB736
:1025A0003EB7295F3F4F0FB6F8943EBF0FBE2DBF19
:1025B000853018F086E080937E0783E690E00E94E5
:1025C000F51790938C0780938B07D7CE8BE090E024
:1025D0009F938F9380E897E09F938F9381E08F93F1
:1025E00080910E038F9387E48F930E942A0D10929F
:1025F000EC038DB79EB707960FB6F8949EBF0FBE3B
:102600008DBFAECE8AE090E09F938F938EE597E0EA
:102610009F938F9381E08F938F9386E58F930E9492
:102620002A0D1092E8032DB73EB7295F3F4F0FB632
:10263000F8943EBF0FBE2DBF8ACE0E943B2280E59C
:1026400090E09F938F938AE293E09F938F9321E092
:1026500030E03F932F9389E293E09F938F933F93D2
:102660002F9380E494E09F938F9383E08F9381E096
:102670008F938CE48F930E942A0D1092EB038DB7F9
:102680009EB70F960FB6F8949EBF0FBE8DBF56CE65
:1026900080915C0790915D070E94FE17882309F0E6
:1026A00077CE72CE80912E0690912F060E94FE1753
:1026B000882309F479CE80911103882309F474CE1C
:1026C0008091F8089927880F991F880F991F7C011E
:1026D0000027F7FC0095102F8091290590912A057D
:1026E000A0912B05B0912C05BC01CD01A80197014B
:1026F0000E94FB6B309321062093200680912105D8
:1027000090912205A0912305B0912405BC01CD0133
:10271000A80197010E94FB6B3093230620932206A9
:102720002091AB093091AC094091AD095091AE09AF
:10273000DA01C90103E0880F991FAA1FBB1F0A9580
:10274000D1F7820F931FA41FB51F820F931FA41FE1
:10275000B51F2091860330918703409188035091E3
:102760008903BC01CD010E94FB6B309325062093A9
:1027700024068EE090E09F938F9380E296E09F93F3
:102780008F9381E08F938F9383E48F930E942A0D20
:102790008091DA039091DB030E94F51790932F0646
:1027A00080932E062DB73EB7295F3F4F0FB6F894A2
:1027B0003EBF0FBE2DBFF8CD82E490E09F938F9374
:1027C00083E298E09F938F9381E08F938F9384E4CB
:1027D0008F930E942A0D1092E9038DB79EB707963A
:1027E0000FB6F8949EBF0FBE8DBF80910C039091E1
:1027F0000D03009709F4D1CD0E94F51790935D0762
:1028000080935C07CACD8093E6031092EA038DCDD6
:102810001F910F91FF90EF900895982F8091660877
:10282000813031F0892F0E943711282F33270CC0B7
:1028300080914104E82FFF27E65DFC4F90838F5F76
:102840008093410421E030E0C90108950F931F9364
:10285000CF93DF938C01EB01672B71F0F80181912D
:102860008F010E940D14219739F0F80181918F0199
:102870000E940D14219791F7DF91CF911F910F9135
:1028800008950F931F93CF93DF938C01EB01672B78
:1028900081F0F8010F5F1F4F84910E940D14219762
:1028A00041F0F8010F5F1F4F84910E940D14219792
:1028B00081F7DF91CF911F910F910895CF93C82F8A
:1028C000181634F480E20E940D14C1501C16D4F383
:1028D000CF910895CF93C82F181634F480E30E9447
:1028E0000D14C1501C16D4F3CF9108952F923F922E
:1028F0004F925F926F927F928F929F92AF92BF9210
:10290000CF92DF92EF92FF920F931F93CF93DF93BB
:10291000CDB7DEB7E0970FB6F894DEBF0FBECDBFE0
:1029200026968FAD26972896EEADFFAD2897882482
:10293000992454018093660848E4C42ED12CCC0E0F
:10294000DD1E7F01C701F7011491112331F015320B
:1029500021F00894E11CF11CF6CFB701681B790B3C
:1029600009F095C0112309F43DC20894E11CF11C43
:102970001FA63FA4232C0FEF39A6F7010894E11CF2
:10298000F11C14911537C9F1812F80628837A9F1A4
:10299000103209F440C0133209F48DC01A3209F420
:1029A00079C01D3209F476C01B32C9F11E32C9F15B
:1029B000103309F48AC0812F8153893008F07EC01A
:1029C00060E070E0CB01880F991F880F991F880F76
:1029D000991F860F971F680F791F610F711D605334
:1029E0007040F7010894E11CF11C1491812F805371
:1029F0008A3040F3262E153739F630FE3DC0F601F9
:102A000084E090E0C80ED91E80809180A280B380BF
:102A1000103209F0C0CF89A5882309F0AECF19A7DD
:102A2000ACCFF7010894E11CF11C14911A3209F49F
:102A300051C060E070E014C0CB01880F991F880F6F
:102A4000991F880F991F860F971F680F791F610FB5
:102A5000711D60537040F7010894E11CF11C149142
:102A6000812F80538A3040F3EFEF6F3F7E0714F4DD
:102A70006FEF7FEF062F86CFF60182E090E0C80E61
:102A8000D91E808191814C01AA24BB2481CF0E9450
:102A9000411468CF1A3251F4F60182E090E0C80E7A
:102AA000D91E208022200CF068CF219490E1392A91
:102AB000EFED3E2262CF98E0392A5FCF1836C9F099
:102AC0001C36D1F481E0382A58CF34FC56CFF0E2DE
:102AD0003F2A53CFF60182E090E0C80ED91E6081F4
:102AE00071819FEF6F3F790714F46FEF7FEF062F2F
:102AF00044CF24E0322A41CF133609F44DC11434B7
:102B000009F41FC1143609F41CC1193609F419C19E
:102B10001F3409F40FC11F3609F40CC1103709F432
:102B2000F9C0133709F4B2C0153509F4ECC01537F4
:102B300009F4E9C0183509F444C0183709F441C054
:102B4000112309F44FC1CE0101969DA78CA71983CB
:102B500081E0482E19A6632C7724042D5FA4541815
:102B600057FC2DC029A5222331F10F5F050DC301AC
:102B700080739070892B09F42FC1222309F027C19B
:102B800066FC1BC1C30180739070809709F410C16B
:102B9000852D0E946A14842D992787FD9095BC018C
:102BA0008CA59DA50E94261464FECCCE822D801B90
:102BB0000E945E14C7CE66FED9CF0E5FD7CF5524D4
:102BC000D1CFE0E1EEA733FE07C081149104A10448
:102BD000B10411F0F0E43F2A19A60FA707FD02C0C7
:102BE0002FED3222CE0189969DA78CA781149104E6
:102BF000A104B10419F49FA5992361F1EEA54E2E0D
:102C000055246624772418AA84149504A604B704CE
:102C100010F0F1E0F8ABC501B401A30192010E94EC
:102C2000D96BDC01CB01082F8A30F0F4005DECA5F4
:102C3000FDA50293FDA7ECA7C501B401A301920174
:102C40000E94D96B49015A01F8A9FF23E1F62EA58C
:102C5000283079F0632C7724CE010196482EFCA50C
:102C60004F1A28E2420E79CF095A183501F70F7D25
:102C7000DECF632C772463FEEFCF003369F380E36C
:102C8000ECA5FDA58293FDA7ECA7E6CFF60182E0B7
:102C900090E0C80ED91E0190F081E02DFDA7ECA7B1
:102CA000EF2B81F4FE013196FDA7ECA788E2898322
:102CB0008EE6818385E78B838CE68C838D8389E226
:102CC0008E831F8207FD15C0802F992787FD909561
:102CD000AC0160E070E08CA59DA50E94A06A009701
:102CE00031F0482EFCA54F1A04150CF033CF402EBE
:102CF00031CFECA5FDA501900020E9F731974E2ECC
:102D00002CA5421A27CF153511F481E0382A9AE014
:102D10009EA762CFF60182E090E0C80ED91E8081A6
:102D200091814C01AA24BB2490E19EA7E0E43E2AB5
:102D300018E752CF1F3411F4E1E03E2AF8E0FEA775
:102D40004BCF143411F491E0392A30FE18C0F6014B
:102D500084E090E0C80ED91E80809180A280B3806C
:102D6000B7FE0AC0B094A09490948094811C911CEA
:102D7000A11CB11C8DE289A79AE09EA72ECFF60177
:102D800082E090E0C80ED91E808191814C01AA2476
:102D900097FCA094BA2CE4CFFE013196FDA7ECA7D6
:102DA000F60182E090E0C80ED91E80818983D0CEE2
:102DB000822D801B0E946A14EBCE80E38AA71BA79A
:102DC00062E070E0CE018A960E942614DBCE61E0BC
:102DD00070E0CE018996F8CF822D801B0E945E1490
:102DE00029A5CBCEE0960FB6F894DEBF0FBECDBFBF
:102DF000DF91CF911F910F91FF90EF90DF90CF90D7
:102E0000BF90AF909F908F907F906F905F904F900A
:102E10003F902F9008951F920F920FB60F9211249A
:102E20002F933F935F936F937F938F939F93AF9372
:102E3000BF93EF93FF938091FA03882329F0809149
:102E4000FA0381508093FA038091CE05882319F00C
:102E500081508093CE058091020481508F3F09F408
:102E600093C0809302048091FB039091FC03892B13
:102E700001F18091FB039091FC0301979093FC0377
:102E80008093FB038091FB039091FC03209112033C
:102E90003091130382239323892B89F080910201BF
:102EA0008A3009F48BC0479A8091E90883FF8DC06E
:102EB00010C08FEF9FEF90931303809312038091C4
:102EC00002018A3009F478C047988091E90883FFAD
:102ED0007CC086B19927FC01E071F07084FF0AC0C4
:102EE0008091FD039091FE0301969093FE038093E1
:102EF000FD036BC08091FD039091FE03892B49F186
:102F00008091FD039091FE038A56914010F58091C7
:102F1000FD039091FE0369E270E00E94B26B809124
:102F2000FD039091FE03860F971F9093FE038093FD
:102F3000FD038091FD039091FE030B9708F440C0C0
:102F40008091FD039091FE030A979093F004809383
:102F5000EF048091EF049091F0042091ED04309102
:102F6000EE04821B930B845E9D4F68E671E00E9425
:102F7000C66B845B90409093EC048093EB041092BA
:102F8000FE031092FD0321C089E08093020480912A
:102F900014038F5F817080931403882319F481E0F8
:102FA0008093FF0380910004909101040196909317
:102FB00001048093000457CF5A9887CF5A9A85CF3F
:102FC000F093F004E093EF04C4CFFF91EF91BF9131
:102FD000AF919F918F917F916F915F913F912F91D1
:102FE0000F900FBE0F901F90189520910004309104
:102FF0000104280F391FC90101960895209100048A
:1030000030910104821B930B892F99278695807438
:1030100090700895CF93DF930E94F517EC01CE01D5
:103020000E94FE178823D9F3DF91CF9108951F9353
:10303000CF93DF930E94F517EC011FEC08C080913D
:103040001903882321F09093190310937A00CE017D
:103050000E94FE17982F882391F3DF91CF911F9143
:1030600008959FB7F8945F983E9A469A8091B00071
:103070008F708093B0008091B00083608093B00027
:103080008091B1008B738093B1008091B1008B600F
:103090008093B1001092B2008FEF8093B3008091C3
:1030A000B00080688093B000809170008A7F809328
:1030B0007000809170008260809370009FBF0895BF
:1030C0008AE090E00E94F51790930A048093090427
:1030D00082E085BD83EA84BD17BC88E788BD86E0B1
:1030E00086BD80916E00816080936E0008951F926E
:1030F0000F920FB60F9211242F933F934F935F932C
:103100006F937F938F939F93AF93BF93EF93FF93AF
:10311000809102018431D8F48091BA0487FD17C0F0
:1031200080910304882309F461C020910404309144
:10313000050451E02F373507E8F18FEF8093B30096
:103140002F5F30403093050420930404B3C3809173
:103150000304882351F78091B00086FFF9C0809165
:10316000B0008F7B8093B00080910804882309F021
:1031700043C180911009282F33278DED96E0289FB9
:10318000A001299F500D389F500D1124CA01209194
:10319000060430910704821B930B909305048093DF
:1031A00004041092070410920604469A81E080936A
:1031B0000304BBCF2F3F310571F068F0A9014F5FC9
:1031C00050404F37510508F0EDC080E88093B300C0
:1031D00020583040B7CF809104048093B300109200
:1031E0000504109204041092030464C38091B0009B
:1031F00086FFE0C08091B0008F7B8093B00089EAA9
:1032000093E09093050480930404809115039091BA
:1032100016039C01220F331F280F391F8091920340
:103220009927880F991F880F991F280F391F37FD7D
:103230008BC2C901959587959595879590931603AF
:10324000809315039093F8038093F70380913809D6
:1032500080FD7BC180910909682F772788279927EE
:103260002091290530912A0540912B0550912C057C
:1032700057FD9FC2E7E05595479537952795EA9505
:10328000D1F70E94876B9B01AC0197FD8DC276E060
:1032900055954795379527957A95D1F78091F703FE
:1032A0009091F803821B930B9093F8038093F7039C
:1032B00080910A09282F3327220F331F220F331F33
:1032C0008091F7039091F803821793077CF0809127
:1032D0000B09282F3327220F331F220F331F809112
:1032E000F7039091F8032817390724F43093F80373
:1032F0002093F7032091F7033091F80380910404A1
:1033000090910504280F391F205032408091F70317
:103310009091F80397FD1BC2959587959595879594
:103320009093F8038093F70345E02D3D340708F4AC
:1033300060C18CED95E09093050480930404209186
:10334000040430910504309307042093060450C010
:103350008091B00080648093B0008CEB90E09093FB
:10336000050480930404809106049091070484541A
:103370009F4F90930704809306048091F90388235C
:1033800029F08091DE04853B08F00AC1469A9091AD
:1033900008049F5F80911009891708F0D3C010922C
:1033A000080404CF8FEF8093B3005093050440933B
:1033B000040480C28091B00080648093B00080914A
:1033C0001009282F33278DED96E0289FA001299F13
:1033D000500D389F500D1124CA01209106043091E0
:1033E0000704821B930B90930504809304049C01B3
:1033F00081E0809303049DCE29EA33E0992782304F
:10340000910509F409C1833091050CF0CBC03093CC
:10341000050420930404019709F0CBC080911503A3
:10342000909116039C01220F331F280F391F8091A2
:1034300092039927880F991F880F991F280F391F0A
:1034400037FD21C2C90195958795959587959093EC
:103450001603809315039093F8038093F7038091EC
:10346000380980FFCFC180910909682F7727882705
:1034700099272091290530912A0540912B055091DB
:103480002C0557FD03C2E7E05595479537952795DD
:10349000EA95D1F70E94876B9B01AC0197FDFBC1B8
:1034A000B6E05595479537952795BA95D1F7809110
:1034B000F7039091F803820F931F9093F803809382
:1034C000F70380910A09282F3327220F331F220F79
:1034D000331F8091F7039091F803821793077CF0D4
:1034E00080910B09282F3327220F331F220F331F00
:1034F0008091F7039091F8032817390724F430934B
:10350000F8032093F7038091F7039091F80320913B
:10351000040430910504820F931F805092409093D1
:103520000504809304048091F7039091F80397FDBC
:10353000A8C195958795959587959093F803809365
:10354000F70337C09093080431CE80910909682FA2
:103550007727882799272091290530912A054091BE
:103560002B0550912C0557FD2EC1A7E05595479589
:1035700037952795AA95D1F70E94876B9B01AC01DF
:1035800097FD1CC1F6E05595479537952795FA9517
:10359000D1F78091F7039091F803820F931F84CEA7
:1035A0004698F5CE039709F413C130930504209390
:1035B0000404209104043091050485E02D3D380772
:1035C000F8F08CED95E090930504809304049C0141
:1035D0002C5B304030930504209304048091060452
:1035E00090910704820F931F909307048093060421
:1035F000DDCD51E02737350750F487E791E09BCECA
:1036000041E02737340720F787E791E0DCCF30939C
:1036100005042093040493CE3093050420930404FE
:1036200080911703909118039C01220F331F280FDC
:10363000391F809191039927880F991F880F991F2F
:10364000280F391F37FDDBC0C901959587959595E2
:10365000879590931803809317039093F6038093B4
:10366000F5038091380981FF74C080910D09682F9E
:1036700077278827992720912105309122054091AD
:1036800023055091240557FDF7C0A7E055954795B0
:1036900037952795AA95D1F70E94876B9B01AC01BE
:1036A00097FDDBC0F6E05595479537952795FA9538
:1036B000D1F78091F5039091F603820F931F9093B9
:1036C000F6038093F50380910E09282F3327220FEC
:1036D000331F220F331F8091F5039091F603821759
:1036E00093077CF080910F09282F3327220F331F77
:1036F000220F331F8091F5039091F60328173907A5
:1037000024F43093F6032093F5038091F503909110
:10371000F6032091040430910504820F931F80501A
:10372000924090930504809304048091F503909156
:10373000F60397FD62C0959587959595879590932B
:10374000F6038093F50335CF2D5F3F4F72CD03967F
:10375000E3CD80910D09682F77278827992720913D
:10376000210530912205409123055091240557FDF4
:103770007EC0E7E05595479537952795EA95D1F7AF
:103780000E94876B9B01AC0197FD6CC066E055956C
:103790004795379527956A95D1F78091F5039091D4
:1037A000F603821B930B8BCF215C3F4F4F4F5F4F34
:1037B0006ECD21583F4F4F4F5F4F5CCD215C3F4F47
:1037C0004F4F5F4FDFCE21583F4F4F4F5F4FCDCE12
:1037D0008091E708E82FFF27EE0FFF1FE155F74F15
:1037E00080819181805E9F4F0CF0DFCE87E791E072
:1037F0009093050480930404DCCE03969CCF2D5F48
:103800003F4F22CF80910909682F77278827992772
:103810002091290530912A0540912B0550912C05C6
:1038200057FD43C0A7E05595479537952795AA952D
:10383000D1F70E94876B9B01AC0197FD31C0F6E088
:103840005595479537952795FA95D1F78091F703C8
:103850009091F803821B930B30CE215C3F4F4F4F6A
:103860005F4F20CF215C3F4F4F4F5F4F8FCF21588D
:103870003F4F4F4F5F4F7DCF21583F4F4F4F5F4FCF
:1038800004CF039656CE2D5F3F4FDCCD21583F4FDE
:103890004F4F5F4FF8CD215C3F4F4F4F5F4F00CEF2
:1038A000215C3F4F4F4F5F4FCACF21583F4F4F4F83
:1038B0005F4FB8CFFF91EF91BF91AF919F918F91E3
:1038C0007F916F915F914F913F912F910F900FBE1C
:1038D0000F901F90189510927C008FEC80937A00C7
:1038E0000895EF92FF920F931F93CF93DF9303E01E
:1038F00010E0D8010E94166C802DC82FDD27C5313D
:10390000D10508F02A97C7BD1092120484E690E012
:103910000E94171880911D0390911E0380529340BE
:1039200010F4C0E0D0E0CA3FD105E0F48AEAE82E06
:1039300083E0F82EC7BD82E390E00E941718FF9243
:10394000EF921F920E94761480911D0390911E03A6
:103950000F900F900F908052934020F02196CA3F15
:10396000D10540F3D8010C2E0E94236CC09373083C
:103970008CE291E00E941718DF91CF911F910F9177
:10398000FF90EF900895EF92FF920F931F93CF93C4
:10399000DF9300E000930D0400930C0400930B04EC
:1039A00080ED97E00E94F517EC011CE821E0F22E73
:1039B00095EFE92E033009F4ABC000E080912204BA
:1039C000909123048C5F93400CF091C080911C0374
:1039D000815080931C0380912004909121048C5F7E
:1039E00093400CF079C080911B03815080931B039E
:1039F00080911E0490911F048C5F93400CF04AC08C
:103A000080911A03815080931A0388E080934904BF
:103A10000E94ED2A80911C038A3008F055C0F09274
:103A20000D048AE080931C0380911B038A3008F008
:103A300043C0F0920C048AE080931B0380911A0328
:103A40008A3098F5F0920B048AE080931A038091F3
:103A50004904882379F0CE010E94FE178823B9F328
:103A60008CEA93E09F938F931F920E9476140F909D
:103A70000F900F90109219038FEC80937A00809131
:103A800019038823E1F31A3008F447C0115009F0F4
:103A900091CF48C080911E0490911F04875094409C
:103AA0008CF180911A038F5FAECF863F80F2F09247
:103AB0000B04E0921A03CBCF863F08F4BFCFF092FD
:103AC0000C04E0921B03BACF863F08F4ADCFF0920E
:103AD0000D04E0921C03A8CF809120049091210452
:103AE000875094408CF080911B038F5F7FCF809133
:103AF0002204909123048750944044F080911C0349
:103B00008F5F67CF0F5F81CF0F5F72CF01E063CF11
:103B10001B3008F452CF19E050CF8AE090E00E94A9
:103B20001718B4CF86E490E00E941718DF91CF9168
:103B30001F910F91FF90EF9008951F920F920FB673
:103B40000F921124AF92BF92CF92DF92EF92FF9229
:103B50000F931F932F933F934F935F936F937F9395
:103B60008F939F93AF93BF93EF93FF9320912B0479
:103B7000822F9927AA27BB272F5FFC01429740F489
:103B8000E25CFF4FEE0FFF1F0590F491E02D0994CA
:103B900010922B0482E080932A0480912A0480935F
:103BA0007C0080912B04882309F443C48FEC80931C
:103BB0007A003FC420932B04809178009091790083
:103BC0002091300430913104820F931F909331047F
:103BD0008093300481E0DFCF20932B048091780024
:103BE0009091790020912E0430912F04820F931F21
:103BF00090932F0480932E0484E0CDCF20932B0448
:103C000080917800909179002091370530913805A6
:103C1000821B930B909372088093710880917108B6
:103C200090917208909339048093380482E0B3CF66
:103C300020932B04809135059091360520917800D2
:103C400030917900821B930B9093680880936708EA
:103C500080916708909168089093370480933604A8
:103C600087E099CF20932B04809178009091790080
:103C700090932D0480932C0486E08DCF20932B0409
:103C8000209178003091790030932F0420932E04F6
:103C900010922A0482CF20932B0420917800309137
:103CA0007900309331042093300481E074CF109276
:103CB0002B0481E08093190380910E0490910F04EE
:103CC000019690930F0480930E0480917800909158
:103CD000790090931E0380931D0380911D039091A2
:103CE0001E035C01CC24DD2480913A0490913B04B6
:103CF000A0913C04B0913D04A80EB91ECA1EDB1E63
:103D000080913E048F5F823108F4E8C280911F03E6
:103D100090912003A0912103B09122037C018D0199
:103D200023E0EE0CFF1C001F111F2A95D1F7E81AA3
:103D3000F90A0A0B1B0BEA0CFB1C0C1D1D1D8091C4
:103D40001204992787FD9095A92FB92FBC01CD01A9
:103D500026EC34E240E050E00E94876BDC01CB01AE
:103D6000E81AF90A0A0B1B0BD801C7010496A11D1A
:103D7000B11DB7FD23C313E0B595A795979587951A
:103D80001A95D1F780931F0390932003A0932103EA
:103D9000B093220380916B0890916C087C010027FE
:103DA000F7FC0095102F80911F0390912003A091A4
:103DB0002103B0912203E81AF90A0A0B1B0BE092C7
:103DC000D004F092D1040093D2041093D304209134
:103DD000130430911404409115045091160457FDBA
:103DE000FDC2A4E05595479537952795AA95D1F73B
:103DF0008091130490911404A0911504B0911604BD
:103E0000821B930BA40BB50B8093130490931404A3
:103E1000A0931504B0931604809113049091140498
:103E2000A0911504B09116048E0D9F1DA01FB11F07
:103E30008093130490931404A0931504B093160474
:103E40008091100490911104BC0162957295707F6D
:103E50007627607F7627681B790B209113043091B9
:103E60001404409115045091160457FDB2C2E4E0C9
:103E70005595479537952795EA95D1F78091D004C8
:103E80009091D104821B930B880F991F880F991F63
:103E9000880F991F860F971F97FDA9C29595879543
:103EA0009595879595958795959587959093110408
:103EB00080931004D601C501D7FC95C2B595A7958E
:103EC0009795879580933A0490933B04A0933C0484
:103ED000B0933D0489E080933E0482E05CCE209361
:103EE0002B04209178003091790080912E049091DC
:103EF0002F04280F391F809102018A3009F448C22B
:103F0000220F331F220F331F30932F0420932E04D0
:103F1000C90137FD73C295958795959587959595B8
:103F2000879590932104809320048091340490918C
:103F30003504820F931F97FD66C2959587959093E0
:103F400035048093340420913F0530914005821B55
:103F5000930B9093240380932303209126043091A4
:103F600027048091230390912403280F391F37FDE4
:103F700047C235952795309327042093260483E084
:103F80000ACE20932B042091780030917900809103
:103F9000300490913104280F391F809102018A303A
:103FA00009F407C2220F331F220F331F309331044D
:103FB00020933004C90137FDFFC1959587959595EC
:103FC00087959595879590932304809322048091FB
:103FD000320490913304820F931F97FD0DC2959583
:103FE000879590933304809332042091410530915A
:103FF0004205821B930B9093260380932503209107
:104000002804309129048091250390912603280FDC
:10401000391F37FDEEC1359527953093290420933C
:10402000280481E0B8CD20932B04809178009091F2
:1040300079002091370530913805821B930B9093BE
:104040007208809371088091710890917208209194
:10405000380430913904820F931F90931B0480938E
:104060001A0482E098CD20932B048091350590911D
:1040700036052091780030917900821B930B909344
:10408000680880936708809167089091680820917C
:10409000360430913704820F931F90931D04809350
:1040A0001C0487E078CD20932B04809102018A3094
:1040B00009F471C1843109F4A8C18091780090910C
:1040C000790020912C0430912D04820F931F90933E
:1040D0001F0480931E0486E05ECD20932B04809104
:1040E00078009091790020912E0430912F04820F56
:1040F000931F90932F0480932E0410922A044DCD89
:1041000020932B04E2CD20932B0480917800909192
:104110007900AA2797FDA095BA2FBC01CD010E9476
:104120000D6B7B018C0180912F0590913005A09142
:104130003105B09132059C01AD01C801B7010E9463
:10414000AD6ADC01CB01BC01CD010E94F06ADC014B
:10415000CB019093190480931804809118049091D6
:10416000190402970CF4C6C080912F059091300578
:10417000A0913105B091320520E030E84BE354E4E2
:10418000BC01CD010E94176B8823DCF580912F05BF
:1041900090913005A0913105B09132052AE037EDBC
:1041A00043EA5CE3BC01CD010E94AE6ADC01CB01B5
:1041B00080932F0590933005A0933105B09332057D
:1041C0008091AE049091AF04845F9140D0F48091CF
:1041D0002F0590913005A0913105B09132052DEC5D
:1041E0003CEC4CEC5DE3BC01CD010E94AE6ADC010D
:1041F000CB0180932F0590933005A0933105B093A8
:10420000320581E0809317048091780090917900C5
:1042100090936A088093690880911804909119041A
:10422000AA2797FDA095BA2F2091F1043091F204AE
:104230004091F3045091F404820F931FA41FB51F03
:104240008093F1049093F204A093F304B093F404E8
:104250002091F1043091F2044091F3045091F40460
:1042600057FDB2C00AE055954795379527950A95B1
:10427000D1F78091F1049091F204A091F304B091F0
:10428000F404821B930BA40BB50B8093F104909361
:10429000F204A093F304B093F40483E07CCC209365
:1042A0002B0480912703909128039C01220F331F38
:1042B000280F391F809178009091790063E070E0B9
:1042C0000E94B26B260F371F369527953695279596
:1042D000309328032093270385E05DCC80933E0430
:1042E000A0923A04B0923B04C0923C04D0923D04A8
:1042F00082E051CC80911804909119048F5F9F4FF8
:104300000CF07FCF80912F0590913005A091310561
:10431000B091320520E030E849E054E4BC01CD0121
:104320000E941A6B18160CF06CCF80912F0590919B
:104330003005A0913105B09132052AE037ED43EA0E
:104340005CE3BC01CD010E94AD6ADC01CB0180932E
:104350002F0590933005A0933105B09332058091DD
:10436000AE049091AF04845F914008F04ACF8091F1
:104370002F0590913005A0913105B09132052DECBB
:104380003CEC4CEC5DE3BC01CD010E94AD6A2FCF4B
:10439000220F331FB9CD8091780090917900209140
:1043A0002C0430912D04820F931F019696958795CA
:1043B0008ECE220F331FFACD0796FFCDD801C7014D
:1043C0000B96A11DB11DD7CC21503C4F4F4F5F4FD5
:1043D00049CF215F3F4F4F4F5F4F49CD215F3F4F47
:1043E0004F4F5F4FFECC0196A11DB11D67CD0F96BB
:1043F00055CD2F5F3F4F0FCE0196F1CD07968BCD58
:104400002F5F3F4FB6CD019698CD80917800909167
:10441000790020912C0430912D04820F931F2FEFEF
:1044200037E0281B390B30931F0420931E0486E0CD
:10443000B2CBFF91EF91BF91AF919F918F917F91FF
:104440006F915F914F913F912F911F910F91FF902D
:10445000EF90DF90CF90BF90AF900F900FBE0F9076
:104460001F90189590E2EAE2F3E08FE49193815077
:1044700087FFFCCF08951F93CF93DF938091400473
:1044800020912903281710F42093400490913F04B1
:1044900090FF08C080914004882309F41EC1815018
:1044A0008093400491FF08C080914004821709F472
:1044B000E4C18F5F80934004892F992780FF02C059
:1044C00081FD08C10E943222909140049A3008F088
:1044D000A2C081E180934104892F99279F938F93F4
:1044E00083EE93E09F938F9381E08F930E947614E5
:1044F0000F900F900F900F900F9080914004C82F55
:10450000DD27C730D10509F4BBC1C830D1050CF097
:104510008CC0C330D10509F455C2C430D1050CF0AC
:10452000DFC0C130D10509F4BBC2C230D1050CF4E3
:1045300038C3109241048CEA94E09F938F93C1E0BA
:10454000CF930E94761484E1809341040F900F90E2
:104550000F908091290590912A05A0912B05B0918B
:104560002C05B7FD58C63AE0B595A7959795879560
:104570003A95D1F7BF93AF939F938F9386EB94E0D7
:104580009F938F93CF930E94761488E28093410487
:104590008DB79EB707960FB6F8949EBF0FBE8DBF1E
:1045A0008091210590912205A0912305B0912405C9
:1045B000B7FD2CC62AE0B595A795979587952A95BE
:1045C000D1F7BF93AF939F938F9385EC94E09F9324
:1045D0008F93CF930E9476148CE3809341042DB780
:1045E0003EB7295F3F4F0FB6F8943EBF0FBE2DBFB9
:1045F0008091EF049091F0049F938F9384ED94E069
:104600009F938F93CF930E9476140F900F900F90EB
:104610000F900F90D6C780E180934104892F99278E
:104620009F938F9388EE93E05DCFCB30D10509F453
:104630005DC1CC30D1050CF00FC1C930D10509F4F2
:104640000BC52A970CF01CC3109241048BE796E02F
:104650009F938F9311E01F930E94761484E18093BF
:1046600041040F900F900F908091EB049091EC0417
:104670009F938F938AE896E09F938F931F930E9456
:10468000761488E2809341040F900F900F900F9062
:104690000F908091EF049091F0049F938F9389E99C
:1046A00096E09F938F931F930E9476148CE38093E0
:1046B00041040F900F900F900F900F908091ED0498
:1046C0009091EE049F938F9388EA96E09F938F9347
:1046D0001F9399CF10924004F5CE20934004E2CE70
:1046E000C530D10509F403C426970CF08CC3109291
:1046F00041048091E208E82FFF27EE0FFF1FE155EC
:10470000F74F808191819F938F938091E108E82FEB
:10471000FF27EE0FFF1FE155F74F808191819F9397
:104720008F9383E295E09F938F9311E01F930E94F4
:10473000761484E1809341048DB79EB707960FB637
:10474000F8949EBF0FBE8DBF8091E408E82FFF272D
:10475000EE0FFF1FE155F74F808191819F938F935B
:104760008091E308E82FFF27EE0FFF1FE155F74F79
:104770008081918188589F4F9F938F9383E395E029
:104780009F938F931F930E94761488E28093410435
:104790002DB73EB7295F3F4F0FB6F8943EBF0FBE0F
:1047A0002DBF8091E608E82FFF27EE0FFF1FE15590
:1047B000F74F8081918182599F4F9F938F93809172
:1047C000E508E82FFF27EE0FFF1FE155F74F808127
:1047D000918182599F4F9F938F9383E495E09F939C
:1047E0008F931F930E9476148CE3809341046DB7DE
:1047F0007EB7695F7F4F0FB6F8947EBF0FBE6DBF67
:104800008091E808E82FFF27EE0FFF1FE155F74FD3
:104810008081918182599F4F9F938F938091E70868
:10482000E82FFF27EE0FFF1FE155F74F80819181A1
:1048300082599F4F9F938F9383E595E09F938F932A
:104840001F930E9476148DB79EB707960FB6F89403
:104850009EBF0FBE8DBFB5C6CD30D10509F447C48C
:10486000CD30D1050CF452C22E9709F4D9C4815031
:104870008093290310924004A4C6109240041CCED9
:1048800084E18093410480912703909128039F93B2
:104890008F938DE496E09F938F9311E01F930E9476
:1048A000761488E2809341040F900F900F900F9040
:1048B0000F908091DE0499279F938F938CE596E06B
:1048C0009F938F931F930E9476148CE380934104EF
:1048D0000F900F900F900F900F908091AE08992736
:1048E00001979F938F938BE696E0F0CE1092410450
:1048F00089E197E09F938F9311E01F930E947614B4
:1049000084E1809341040F900F900F908091840771
:10491000992787FD90959F938F938091830799277F
:1049200087FD90959F938F9389E297E09F938F9354
:104930001F930E94761488E2809341048DB79EB73E
:1049400007960FB6F8949EBF0FBE8DBF8091850766
:10495000992787FD90959F938F938091860799273C
:104960009F938F9389E397E09F938F931F930E9468
:1049700076148CE3809341042DB73EB7295F3F4FF7
:104980000FB6F8943EBF0FBE2DBF80918A079927BE
:104990009F938F9380918707992787FD90959F9389
:1049A0008F9389E497E09F938F931F930E947614CF
:1049B0006DB77EB7695F7F4F0FB6F8947EBF0FBEAD
:1049C0006DBFFFC5109241048091B3089091B40867
:1049D0009F938F938091B1089091B2089F938F938A
:1049E00083EE94E09F938F9311E01F930E947614BF
:1049F00084E1809341046DB77EB7695F7F4F0FB646
:104A0000F8947EBF0FBE6DBF8091B7089091B80833
:104A10009F938F938091B5089091B6089F938F9341
:104A200083EF94E09F938F931F930E94761488E204
:104A3000809341048DB79EB707960FB6F8949EBF3A
:104A40000FBE8DBF8091BB089091BC089F938F9340
:104A50008091B9089091BA089F938F9383E095E075
:104A60009F938F931F930E9476148CE3809341044D
:104A70002DB73EB7295F3F4F0FB6F8943EBF0FBE2C
:104A80002DBF8091BF089091C0089F938F93809114
:104A9000BD089091BE089F938F9383E195E083CFEB
:104AA0008091E90880FD1CC084E18093410487E97E
:104AB00094E09F938F9311E01F930E94761488E2F5
:104AC000809341040F900F900F908EE994E09F9394
:104AD0008F931F930E9476140F900F900F9071C5C3
:104AE000109241048091D0049091D104A091D204FD
:104AF000B091D304BC01CD0125E030E040E050E0AE
:104B00000E94FB6B3F932F938BE594E09F938F93D1
:104B100011E01F930E94761484E1809341040F906A
:104B20000F900F900F900F908091CC049091CD0436
:104B3000A091CE04B091CF04BC01CD0125E030E0BE
:104B400040E050E00E94FB6B3F932F938AE694E095
:104B50009F938F931F930E94761488E28093410461
:104B60000F900F900F900F900F9080911D039091D8
:104B70001E039F938F9389E794E09F938F931F93D6
:104B80000E9476148CE3809341040F900F900F9055
:104B90000F900F9087B599279F938F9388E894E0A3
:104BA00095CD209709F063CE109241048DEE93E0ED
:104BB0009F938F9311E01F930E94761484E180935A
:104BC00041040F900F900F9087E690E09F938F9392
:104BD0008CE490E09F938F93DF93CF9380910201B9
:104BE0006AE00E94A66B892F99279F938F938091EB
:104BF00002010E94A66B99279F938F938DEF93E0FC
:104C00009F938F931F930E94761488E280934104B0
:104C10002DB73EB7235F3F4F0FB6F8943EBF0FBE90
:104C20002DBF84ED95E09F938F930E94B505992742
:104C30009F938F938BE194E09F938F931F930E9498
:104C400076148091AC039091AD036DB77EB7695F28
:104C50007F4F0FB6F8947EBF0FBE6DBF069708F466
:104C600088C490914604992309F47DC48CE3809311
:104C70004104892F99279F938F9386E394E026CD53
:104C80001092410487EE96E09F938F9311E01F935B
:104C90000E94761484E1809341040F900F900F904E
:104CA0008091920399279F938F938FEE96E09F9325
:104CB0008F931F930E94761488E2809341040F9093
:104CC0000F900F900F900F908091F7039091F80341
:104CD0009F938F938DEF96E09F938F931F930E94E6
:104CE00076148CE3809341040F900F900F900F90F7
:104CF0000F9080910B0999279F938F9380910A09B8
:104D000099279F938F938BE097E04DCE10924104AB
:104D100089E597E09F938F9311E01F930E9476148B
:104D200084E1809341040F900F900F908091890847
:104D300099279F938F938091880899279F938F93AA
:104D40008091870899279F938F9380918608992750
:104D50009F938F9389E697E09F938F931F930E9471
:104D6000761488E2809341048DB79EB70B960FB6F8
:104D7000F8949EBF0FBE8DBF80918D0899279F9399
:104D80008F9380918C0899279F938F9380918B08A4
:104D900099279F938F9380918A0899279F938F9348
:104DA0008EE797E09F938F931F930E9476148CE376
:104DB000809341042DB73EB7255F3F4F0FB6F8945F
:104DC0003EBF0FBE2DBF8091910899279F938F936F
:104DD0008091900899279F938F9380918F089927AE
:104DE0009F938F9380918E0899279F938F9383E948
:104DF00097E09F938F931F930E9476146DB77EB7B1
:104E0000655F7F4FD9CD1092410483E196E09F9377
:104E10008F9311E01F930E94761484E180934104E4
:104E20000F900F900F9080913705909138059F93C8
:104E30008F9380911A0490911B049F938F9380E22B
:104E400096E09F938F931F930E94761488E280933D
:104E500041046DB77EB7695F7F4F0FB6F8947EBF90
:104E60000FBE6DBF80913505909136059F938F934E
:104E700080911C0490911D049F938F938FE296E084
:104E80009F938F931F930E9476148CE38093410429
:104E90008DB79EB707960FB6F8949EBF0FBE8DBF15
:104EA00080912F0590913005A0913105B091320588
:104EB000BC01CD010E94F06ADC01CB019F938F936E
:104EC00080916209909163099F938F938EE396E09E
:104ED0009F938F931F930E9476142DB73EB7295F3F
:104EE0003F4F0FB6F8943EBF0FBE2DBF6AC310925E
:104EF000410483E695E09F938F93C1E0CF930E9496
:104F00007614809102010F900F900F908A3009F46F
:104F1000A5C28B3009F4DEC1843109F4DBC18D30C8
:104F200009F04FC384E18093410480911C039927C9
:104F30009F938F934091410550914205CA0157FDBF
:104F400039C3959587959595879595958795959569
:104F500087959F938F939A0157FD29C33595279580
:104F600035952795359527958091220490912304B6
:104F7000821B930B9F938F9387ED95E09F938F9365
:104F8000CF930E94761488E2809341046DB77EB778
:104F9000675F7F4F0FB6F8947EBF0FBE6DBF8091E5
:104FA0001B0399279F938F9340913F055091400594
:104FB000CA0157FD04C39595879595958795959555
:104FC0008795959587959F938F939A0157FDF4C286
:104FD000359527953595279535952795809120040A
:104FE00090912104821B930B9F938F938BEE95E0FE
:104FF0009F938F93CF930E9476148CE38093410408
:105000008DB79EB709960FB6F8949EBF0FBE8DBFA1
:1050100080911A0399279F938F9320913D0530919A
:105020003E05C90137FDC1C2959587959F938F9322
:1050300080911E0490911F04281B390B3F932F93DE
:105040008FEF95E09F938F93CF930E9476142DB7A7
:105050003EB7275F3F4F45CF109241048091E50452
:105060009091E6049F938F9387EB96E09F938F93A5
:1050700011E01F930E94761484E1809341040F9005
:105080000F900F900F900F908091E3049091E404A3
:105090009F938F9383EC96E09F938F931F930E942F
:1050A000761488E2809341040F900F900F900F9038
:1050B0000F908091E1049091E2049F938F938FEC85
:1050C00096E09F938F931F930E9476148CE38093B6
:1050D00041040F900F900F900F900F908091DF047C
:1050E0009091E0049F938F938BED96E0EFCA10921E
:1050F000410488EA97E09F938F93C1E0CF930E9489
:10510000761484E1809341040F900F900F9080916A
:10511000A50899278D969F938F938091A40899272E
:105120008D969F938F938091A30899278D969F9337
:105130008F938091A20899278D969F938F9387EBE9
:1051400097E09F938F93CF930E94761488E2809389
:1051500041048DB79EB70B960FB6F8949EBF0FBE55
:105160008DBF8091A90899278D969F938F938091E9
:10517000A80899278D969F938F938091A7089927C8
:105180008D969F938F938091A60899278D969F93D4
:105190008F938BEC97E09F938F93CF930E9476141D
:1051A0008CE3809341042DB73EB7255F3F4F0FB688
:1051B000F8943EBF0FBE2DBF8091AA0899278D9607
:1051C0009F938F938FED97E09F938F93CF930E9440
:1051D00076140F900F900F900F900F908091AB0866
:1051E000882309F02DC18091AC08882309F01AC1E9
:1051F0008091AD08882309F4E4C188E480934104D8
:1052000085EF97E09F938F93CF9364CC81509C4F11
:10521000AF4FBF4FCFC981509C4FAF4FBF4FA3C9B6
:105220001092410488EF97E09F938F9311E01F93B2
:105230000E94761484E1809341040F900F900F90A8
:105240008091D8039091D9039F938F9386E098E043
:105250009F938F931F930E94761488E2809341045A
:105260000F900F900F900F900F908091D603909118
:10527000D7039F938F9383E198E09F938F931F931E
:105280000E94761489E4809341040F900F900F9050
:105290000F900F9080E298E09F938F931F930E944E
:1052A000761480913F040F900F900F9083FF89C177
:1052B0001092D9031092D803AEE0B0E080E0082E3F
:1052C0000E94236CAFE0B0E08091D803082E0E94CA
:1052D000236C77C184E18093410440914105509152
:1052E0004205CA0157FD57C19C0135952795359553
:1052F00027953595279535952795C90182959295DE
:10530000907F9827807F9827BA01681B790BCB0183
:1053100077FD3FC1959587959F938F933F932F93EB
:105320009A0157FD33C135952795359527953595C4
:1053300027958091220490912304821B930B9F93C5
:105340008F9384EA95E09F938F93CF930E94761476
:1053500088E2809341048DB79EB709960FB6F89402
:105360009EBF0FBE8DBF40913F0550914005CA01C1
:1053700057FD0AC19C01359527953595279535959B
:10538000279535952795C90182959295907F982705
:10539000807F9827BA01681B790BCB0177FDF2C09B
:1053A000959587959F938F933F932F939A0157FDE0
:1053B000E6C03595279535952795359527958091A4
:1053C000200490912104821B930B9F938F9386EB73
:1053D00095E09F938F93CF930E9476148CE38093F4
:1053E00041048DB79EB709960FB6F8949EBF0FBEC5
:1053F0008DBF20913D0530913E05C90137FDCDC0DF
:10540000959587959F938F9380911E0490911F048B
:10541000281B390B3F932F9388EC95E09F938F9334
:10542000CF9359CD84E48093410482EF97E09F931A
:105430008F93CF930E9476140F900F900F90D8CE39
:1054400080E4809341048FEE97E09F938F93CF93F6
:105450000E9476140F900F900F90C5CE84E1809338
:10546000410440914105509142059A0157FD9AC06F
:10547000359527953595279535952795C901880F39
:10548000991F880F991F880F991F481B590B5F930D
:105490004F933F932F938091220490912304821B7A
:1054A000930B9F938F9381E795E09F938F93CF9377
:1054B0000E94761488E2809341042DB73EB7275F9F
:1054C0003F4F0FB6F8943EBF0FBE2DBF40913F0532
:1054D000509140059A0157FD62C035952795359545
:1054E000279535952795C901880F991F880F991F12
:1054F000880F991F481B590B5F934F933F932F932E
:105500008091200490912104821B930B9F938F9391
:1055100083E895E09F938F93CF930E9476148CE35A
:10552000809341046DB77EB7675F7F4F0FB6F894E5
:105530007EBF0FBE6DBF80913D0590913E059F934C
:105540008F9380913D0590913E0520911E043091EE
:105550001F04821B930B9F938F9385E995E09F9384
:105560008F93CF936EC98CE3809341048BE494E0D6
:10557000AECA8CE38093410489E294E0A8CA295F13
:105580003F4F17CF01960CCF0F96F4CE295F3F4FB8
:10559000CACE0196BFCE0F96A7CE019631CF295F16
:1055A0003F4F9BCF295F3F4F63CF01963DCD295F92
:1055B0003F4FD4CC0F96C5CC295F3F4F09CD0F96F6
:1055C000FACC10923F04DF91CF911F910895109271
:1055D000B9008AE28093B800089585EA8093BC0000
:1055E000089584E98093BC0008951092B9008093D7
:1055F000BB0085E88093BC0008950E94F12A1092B8
:1056000049048091BB001092480480E88093BC005C
:105610001092BD001092BA001092BB001092B90017
:105620001092B8000E94E72A0E94ED2A80E00E94B2
:10563000F52A08958093BB0085E88093BC00089507
:1056400085EC8093BC00089585E88093BC000895A4
:105650001F920F920FB60F9211242F933F934F93E7
:105660005F936F937F938F939F93AF93BF93EF93CA
:10567000FF9380914904282F3327442755278F5FB4
:1056800080934904F90127313105C8F4E05BFF4FED
:10569000EE0FFF1F0590F491E02D099480914704CF
:1056A000E82FFF27EA58F74F9091BB0090838F5F58
:1056B0008C3008F49DC0109247040E94F12A109289
:1056C0004904E0C080E80E94F52ADCC088E90E9415
:1056D000F52AD8C00E94F12A8AE090E09093AD03A9
:1056E0008093AC030E94ED2ACDC084E10E94F52A8C
:1056F000C9C082E10E94F52AC5C080911C030E94A6
:10570000F52AC0C080E10E94F52ABCC080911B032D
:105710000E94F52AB7C080911A030E94F52AB2C0F0
:1057200080914804E82FFF27EA56F64F8F5F809359
:10573000480480810E94F52AA5C090914804292F31
:10574000E92FFF27EE0FFF1FEE0FFF1FED52FA4F5D
:10575000858518160CF054C09C3009F467C0990F69
:10576000892F8E5A0E94F52A8DC080914704E82F18
:10577000FF27EE56F74F8091BB0080830E94242BB9
:1057800081C08091B900803409F46EC080914704D3
:10579000E82FFF27EE55F74F10828F5F8C3068F1AE
:1057A000109247040E94F12A1092490480914A0401
:1057B0008093460410924A0465C08091B9008033FA
:1057C00009F440C00E94F12A8AE090E09093AD0372
:1057D0008093AC03109249040E94ED2A53C00E94AA
:1057E000F12A8AE090E09093AD038093AC0367CFF9
:1057F000809347040E94F12A62CF80934704D2CF5E
:105800009C3008F0A9CF922F9F5FE92FFF27EE0F62
:10581000FF1FEE0FFF1FED52FA4F858518161CF083
:10582000292F9C3080F39093480496CF109248041F
:1058300083E08093490480914704880F8D5A0E9429
:10584000F52A20C080914A048823C9F49091480425
:1058500090934A04E92FFF27EB57F74F80818F5F22
:1058600009F48FEF8083AECF80914704E82FFF27A4
:10587000EE55F74F8C5F80830E94202B97CF90913D
:105880004804E8CF8091BC0080688093BC00FF9101
:10589000EF91BF91AF919F918F917F916F915F91A8
:1058A0004F913F912F910F900FBE0F901F90189521
:1058B00083EC8093810080916F00806280936F0001
:1058C00010923E0510923D051092400510923F0542
:1058D000109242051092410508951F920F920FB643
:1058E0000F921124EF92FF920F931F932F933F93E8
:1058F0004F935F936F937F938F939F93AF93BF93D8
:10590000CF93DF93EF93FF938091390982FD2CC0F1
:10591000209186003091870080914C0490914D0435
:10592000281B390B809186009091870090934D043D
:1059300080934C04C9018D549440835F9A4108F0D0
:10594000B5C080914E048093AE0880914E04909132
:105950004F04049714F010928403C1E0D0E0D09378
:105960004F04C0934E0415C24091860050918700A9
:105970008091500490915104481B590B80918600EE
:10598000909187009093510480935004CA018D54E4
:105990009440835F9A4138F58091AA0480934B0428
:1059A00080914B04843008F00EC18091AB048536A1
:1059B00008F47BC18AE08093AB04809102018A30B5
:1059C00009F476C1843109F473C1289881E0809389
:1059D000AA048091D404882309F0DBC180914B0490
:1059E0008093AE08D6C10091AA040A3008F0E4C042
:1059F000CA018B5F9040845B914008F05BC1425DBF
:105A00005140E02FFF27EE0FFF1FEE5AFB4F808122
:105A10009181FA01E81BF90BCF0105960B9708F469
:105A20005CC1E02FFF27EE0FFF1FEE5AFB4F808176
:105A300091819C01220F331F280F391F240F351F1E
:105A400037FDA4C1E901D595C795D595C795CA017C
:105A500001968C179D070CF071C121978091DE048F
:105A60008E3B08F462C1E02FFF27EE0FFF1FDF011E
:105A7000AE5ABB4F8D919C919E01281B390BC901D9
:105A800063E070E00E94C66BCB01880F991F860F00
:105A9000971FE859FB4F91838083E02FFF27EE0F7C
:105AA000FF1FEE5AFB4FD183C0830BC1C0914E0440
:105AB000D0914F04CA30D1050CF06BC1C9018B5F86
:105AC0009040845B914008F060C0225D3140FE014F
:105AD000EC0FFD1FE155F74F80819181D901A81B83
:105AE000B90BCD01B7FD0EC1069754F48091DE04C9
:105AF000883C08F046C18091DE04865F8093DE0416
:105B0000FE01EC0FFD1FE155F74F80819181AC0143
:105B1000440F551F480F591F420F531F57FD33C1E4
:105B20007A01F594E794F594E794C90101968E15EE
:105B30009F050CF013C10894E108F1088091DE0480
:105B4000833C08F403C18E010C0F1D1FF801E155C1
:105B5000F74F80819181F701E81BF90BCF0163E0DA
:105B600070E00E94C66BCB01880F991F860F971FAC
:105B70000B53174FD80111969C938E93FE01EC0F97
:105B8000FD1FE155F74FF182E082FE013196F0935F
:105B90004F04E0934E04E530F10509F4B9C05D9877
:105BA000E630F10509F4BFC05C98379709F4B9C035
:105BB0005B98EFC05C9A5B98043108F054C00F5FAB
:105BC0000093AA04E6C09091AE0880914B04981708
:105BD00009F0EBCE4091AB044B3008F49BC010921F
:105BE00084031092AA043AC00091AA04E02FFF2770
:105BF000EE0FFF1F9F0122583B4FDF01A155B74F0A
:105C00008D919C91D9018D939C93DF01AB53B74F3C
:105C10008D919C91EC56FB4F91838083E02FFF2761
:105C2000EE0FFF1F9F012155374FDF01AE5ABB4FCB
:105C30008D919C91D90111969C938E93DF01A85967
:105C4000BB4F8D919C91EB53F74F91838083E02F55
:105C5000EF5FEB3008F05EC0E093AA044F3120F60E
:105C60000091AA04DBCF043109F093C080910201B6
:105C70008A3009F47DC0843109F47AC028988EE115
:105C80008093AA042AE0C5ECD8E0AEE7B4E0EFEADE
:105C9000F8E08D919D9191838083329619821882CC
:105CA0002296215027FFF5CF74C01092AB0485CE09
:105CB000289A8CCE809102018A3011F1843101F151
:105CC0002898053019F15D98063009F473CF5C9877
:105CD000073009F070CF5B9A72CF8091AB048A31A4
:105CE00008F448C08091DE04865F8093DE048091D2
:105CF000DE04893C08F495CE88EC8093DE0491CED6
:105D0000289ADFCF909581959F4FEECE5D9ADFCF99
:105D10005D9A46CF4F3F09F459CE4F5F4093AB0495
:105D200055CE5B9A36C05C9A40CFE02FFF27EE0F2E
:105D3000FF1FE859FB4F11821082AFCE41505040F7
:105D4000C417D5070CF08ACE219688CEFE01EC0F41
:105D5000FD1FEB53F74F1182108210CF21503040BE
:105D6000E216F3060CF0EACE0894E11CF11CE6CE34
:105D7000289A85CF8B3008F4BACF8091DE048E5FED
:105D8000B4CF88ECBBCE4D5F5F4FCACE2D5F3F4F87
:105D900059CEFF91EF91DF91CF91BF91AF919F913C
:105DA0008F917F916F915F914F913F912F911F91B3
:105DB0000F91FF90EF900F900FBE0F901F901895CE
:105DC00081E08093E30882E08093E20883E080939F
:105DD000E10884E08093E40885E08093E50886E0AC
:105DE0008093E60887E08093E70888E08093E808DE
:105DF00008951F938AE68093E90851E0509339098A
:105E00004EE14093EA088BEF8093EC088AE08093A0
:105E1000ED084093EB084093EF0885E08093F0088D
:105E200080E48093F1081092F20884E18093EE08F8
:105E30008EE08093F308E0E1E093F4081CE0109317
:105E4000F508F8E0F093F60886EE8093F7084093A3
:105E5000F80880E88093F90830E53093FA0896E96D
:105E60009093FB0883E08093FC083093FD089093A7
:105E7000FE0881E28093FF0883E28093000940934B
:105E800001091092020960E260930309109204096B
:105E900010920509109206091092070910921C0928
:105EA00010921D0910921E0910921F0924E62093DA
:105EB000080998E2909309095093380910920A0949
:105EC0008AEF80930B0976E07093100920930C09F8
:105ED00090930D0910920E0980930F0982E380932D
:105EE00011099AE5909312098093130910923709CA
:105EF00090931409309315095093160985E5809302
:105F0000170980931809E093190960931A092093DF
:105F10001B098FE58093200983EF809322098AEA89
:105F200080932409809325098FE080932109809331
:105F300023098CEF80932609209327099093280941
:105F40009093290990932A098BE480932B098093DD
:105F50002C0980932D0910922E0970932F09F0932C
:105F600030099093310940933209209333092093EB
:105F7000340984E080933509AEEAB3E0EAE3F9E05E
:105F80000D9001921A95E1F71F9108958AE680938A
:105F9000E90871E0709339095EE15093EA088BEFEC
:105FA0008093EC089AE09093ED085093EB0850939F
:105FB000EF0885E08093F00880E48093F108109268
:105FC000F2088FE08093EE089093F30880E18093CD
:105FD000F40866E06093F508E8E0E093F60886EEE2
:105FE0008093F7085093F80880E88093F9082AE531
:105FF0002093FA0898E79093FB0883E08093FC08CD
:106000002093FD089093FE0881E28093FF0883E2CD
:1060100080930009509301091092020940E24093D5
:1060200003091092040910920509109206091092B2
:10603000070910921C0910921D0910921E09109256
:106040001F0934E63093080998E290930909709388
:10605000380910920A098AEF80930B09609310099E
:1060600030930C0990930D0910920E0980930F093B
:1060700082E38093110920931209809313091092EF
:1060800037092093140980E5809315098CE38093E8
:10609000160985E58093170980931809409319091B
:1060A00040931A099BE490931B098FE58093200984
:1060B00083EF809322098AEA80932409809325093B
:1060C00084E180932109809323098CEF8093260932
:1060D00030932709209328092093290920932A091E
:1060E00090932B0990932C0990932D0910922E09CF
:1060F00060932F09E09330092093310950933209BE
:10610000309333093093340984E0809335098CE06F
:10611000A5EBB3E0EAE3F9E00D9001928A95E1F78F
:1061200008958AE68093E90871E0709339094EE199
:106130004093EA088BEF8093EC088AE08093ED08A7
:106140004093EB084093EF0885E08093F00880E4EB
:106150008093F1081092F2088FE08093EE0868E0D7
:106160006093F30820E12093F40856E05093F5087B
:106170006093F60886EE8093F7084093F80880E86D
:106180008093F90834E63093FA0898E79093FB0877
:1061900083E08093FC083093FD089093FE0881E231
:1061A0008093FF0883E28093000984E180930109D2
:1061B0001092020920930309109204091092050914
:1061C000109206091092070910921C0910921D09DD
:1061D00010921E0910921F093093080998E29093BB
:1061E00009097093380910920A098AEF80930B0904
:1061F0005093100930930C0990930D0910920E09D9
:1062000080930F0992E3909311092AE520931209D4
:1062100090931309109237092093140980E5809315
:10622000150986E48093160985E580931709809304
:10623000180980E28093190980931A0990931B0929
:106240008FE58093200983EF809322098AEA809367
:1062500024098093250940932109409323098CEF59
:106260008093260930932709209328092093290930
:1062700020932A098BE480932B0980932C09809327
:106280002D0910922E0950932F0960933009209305
:10629000310940933209309333093093340984E053
:1062A000809335098CE0ADEBB3E0EAE3F9E00D90C3
:1062B00001928A95E1F70895FC01681779073CF48B
:1062C000680F791F77FD19C07595679525C02091D6
:1062D000BC04222331F4681B790BE61BF70BBF01CA
:1062E0001BC0213069F03327CB018E1B9F0BB901F6
:1062F0000E94C66B6E0F7F1F0FC06F5F7F4FE4CF92
:10630000681B790B77FD03C075956795E6CF6F5FC6
:106310007F4F75956795E1CFCB010895EF92FF927E
:106320000F931F93CF93C82F8B018091D4048823A0
:10633000A9F4C150CF3F91F07B01E60EF71E1093F8
:10634000FC030093FB038091FB039091FC03892BDA
:10635000D1F7C7010E940A18C15088F7CF911F9149
:106360000F91FF90EF9008952F923F924F925F927E
:106370006F927F928F929F92AF92BF92CF92DF9255
:10638000EF92FF920F931F93CF93DF93CDB7DEB7BA
:10639000ED970FB6F894DEBF0FBECDBF20913D053F
:1063A00030913E0580911E0490911F04281B390BEB
:1063B0003A8729873093A5092093A40920912804BE
:1063C0003091290437FDD4C7359527953595279504
:1063D000359527953AA729A73C872B8779012091E6
:1063E00026043091270437FDC0C73595279535958C
:1063F0002795359527953CA72BA73E872D87F092AB
:106400006509E092640930935B0920935A098091F1
:10641000930990919409AA2797FDA095BA2F7C0122
:106420008D01EE0CFF1C001F111FE80EF91E0A1F44
:106430001B1F80911A0490911B049C01442737FD77
:106440004095542FDA01C901880F991FAA1FBB1F5D
:10645000880F991FAA1FBB1F820F931FA41FB51F70
:10646000820F931FA41FB51FE80EF91E0A1F1B1FE2
:1064700017FD9CC715950795F794E7941595079513
:10648000F794E794F0929409E09293098091AF0910
:106490009091B009AA2797FDA095BA2F7C018D0194
:1064A000EE0CFF1C001F111FE80EF91E0A1F1B1F18
:1064B00080911C0490911D049C01442737FD409558
:1064C000542FDA01C901880F991FAA1FBB1F880F1B
:1064D000991FAA1FBB1F820F931FA41FB51F820FF6
:1064E000931FA41FB51FE80EF91E0A1F1B1F17FDDF
:1064F00054C715950795F794E79415950795F79464
:10650000E794F092B009E092AF098091620990910E
:106510006309AA2797FDA095BA2F9C01AD01220F10
:10652000331F441F551F280F391F4A1F5B1F8091BF
:10653000180490911904AA2797FDA095BA2F280F47
:10654000391F4A1F5B1F57FD16C75595479537954D
:10655000279555954795379527953093630920934F
:10656000620920911A0430911B04C901880F991FF8
:10657000880F991F820F931F820F931FAA2797FDE1
:10658000A095BA2F2091190530911A0540911B054D
:1065900050911C05820F931FA41FB51F80931905EE
:1065A00090931A05A0931B05B0931C0520911C0421
:1065B00030911D04C901880F991F880F991F820F00
:1065C000931F820F931FAA2797FDA095BA2F2091A2
:1065D0001505309116054091170550911805820F49
:1065E000931FA41FB51F8093150590931605A093C4
:1065F0001705B093180580916D0990916E0920914F
:106600001A0430911B04820F931F90936E0980939C
:106610006D098091A7099091A80920911C043091DF
:106620001D04820F931F9093A8098093A70980915E
:10663000330590913405019690933405809333058A
:106640008091110590911205A0911305B091140548
:10665000BC01CD010E940D6B5B016C01809169084A
:1066600090916A08AA2797FDA095BA2FBC01CD0189
:106670000E940D6B7B018C0180912F05909130055C
:10668000A0913105B09132059C01AD01C801B7015F
:106690000E94AD6ADC01CB019C01AD01C601B501D0
:1066A0000E94AE6ADC01CB01BC01CD010E94F06A00
:1066B000DC01CB018093110590931205A093130583
:1066C000B09314058FEC80937A00109219032090F8
:1066D000010530900205409003055090040539E40F
:1066E00023163BE6330631E0430630E053060CF454
:1066F00014C188E49BE6A1E0B0E08D839E83AF8364
:10670000B8876090090570900A0580900B059090FD
:106710000C0539E463163BE6730631E0830630E08E
:1067200093060CF4DCC488E49BE6A1E0B0E0898326
:106730009A83AB83BC8349855A85CA01AA2797FDF2
:10674000A095BA2F2091F9043091FA044091FB04EE
:106750005091FC04280F391F4A1F5B1F2DA33EA335
:106760004FA358A7A090AB09B090AC09C090AD0959
:10677000D090AE09A80EB91ECA1EDB1E8601750197
:106780003091C7043BA3332309F0DAC08091C604DB
:10679000882309F0C2C44091E9084CA346FF13C600
:1067A000EBA5FCA5CF01AA2797FDA095BA2FBC01A8
:1067B000CD0129813A814B815C810E94876B9B01CD
:1067C000AC0197FD2CC7BBE05595479537952795AC
:1067D000BA95D1F780918E03E82EFF240027112768
:1067E000C801B7010E94876B97FD14C7ACE095956F
:1067F000879577956795AA95D1F76F87788B898B61
:106800009A8B60934D0570934E0580934F0590933E
:10681000500529A53AA5C901AA2797FDA095BA2F29
:10682000BC01CD012D813E814F8158850E94876B2F
:106830009B01AC0197FD01C7FBE055954795379546
:106840002795FA95D1F7C801B7010E94876B97FD8C
:10685000EFC6DC01CB01ECE0B595A7959795879540
:10686000EA95D1F78093510590935205A093530573
:10687000B093540520914D0530914E053093DC08BE
:106880002093DB0820915105309152053093E008A8
:106890002093DF082F85388949895A89821B930BF9
:1068A000A40BB50B8AAF9BAFACAFBDAF80935105C6
:1068B00090935205A0935305B0935405A80EB91EAA
:1068C000CA1EDB1E8601750130918D033DA733235F
:1068D00009F0A3C58EA79FA7A8ABB9ABB7FD61C64A
:1068E0002EA53FA548A959A95595479537952795B0
:1068F0008DA19EA1AFA1B8A5821B930BA40BB50BD4
:106900008DA39EA3AFA3B8A78093F9049093FA0434
:10691000A093FB04B093FC048CC598EB291694E972
:1069200039069EEF49069FEF59060CF0F1C328EB9C
:1069300034E94EEF5FEF2D833E834F835887E1CEDE
:106940002DA13EA14FA158A52093F9043093FA043C
:106950004093FB045093FC043091E9083CA310924F
:10696000E0081092DF081092DC081092DB08109209
:10697000490510924A0510924B0510924C05109251
:106980004505109246051092470510924805309132
:106990008D033DA78091490590914A05A0914B0533
:1069A000B0914C05BC01CD0124E630E040E050E060
:1069B0000E94FB6BDA01C9014091450550914605E3
:1069C000481B590B58A34F8F809145059091460560
:1069D000A0914705B0914805BC01CD0124E630E007
:1069E00040E050E00E94FB6BDA01C90120914905AB
:1069F00030914A05821B930B9AA389A38091860349
:106A000090918703A0918803B0918903BC01CD01C7
:106A100028E631E040E050E00E94876BE616F7067A
:106A20000807190744F057016801A61AB70AC80AEF
:106A3000D90A8601750117FDA3C4A092AB09B092D3
:106A4000AC09C092AD09D092AE092BA53CA58F8DA3
:106A500098A1280F391F79010027F7FC0095102F06
:106A60008091FD049091FE04A091FF04B091000577
:106A7000E80EF91E0A1F1B1F570168018091CA0406
:106A80009091CB04281B390BC901AA2797FDA0952B
:106A9000BA2F280E391E4A1E5B1E2091A203309188
:106AA000A3034091A4035091A50322153305440587
:106AB000550574F4A8EAEA2EA1E6FA2E012D112D4F
:106AC000E21AF30A040B150B17012801570168019C
:106AD00088279927DC01821B930BA40BB50B281682
:106AE00039064A065B060CF0E9C2F8E52F2EFEE9EE
:106AF0003F2EFFEF4F2EFFEF5F2E220E331E441E60
:106B0000551E2092010530920205409203055092D5
:106B10000405820171012092FD043092FE0440922E
:106B2000FF045092000529A53AA5A9A1BAA12A0FF0
:106B30003B1FA901662757FD6095762F80910505BB
:106B400090910605A0910705B0910805480F591FBF
:106B50006A1F7B1F5A016B018091C8049091C90480
:106B6000281B390BC901AA2797FDA095BA2F680EDB
:106B7000791E8A1E9B1E8091A6039091A703A09167
:106B8000A803B091A9038EAB9FABA8AFB9AF861590
:106B90009705A805B90564F448EA51E660E070E09D
:106BA000481B590B6A0B7B0B3A014B015A016B01D5
:106BB0008EA99FA9A8ADB9ADB095A09590958195E6
:106BC0009F4FAF4FBF4F681679068A069B060CF0A1
:106BD00064C2E8E56E2EEEE97E2EEFEF8E2EEFEF2B
:106BE0009E2E2EA93FA948AD59AD620E731E841E7C
:106BF000951E6092090570920A0580920B0590928D
:106C00000C05B401A30160920505709206058092FF
:106C10000705909208058DA19EA1AFA1B8A580930C
:106C20000D0590930E05A0930F05B093100560928B
:106C3000290570922A0580922B0590922C052092AE
:106C4000210530922205409223055092240540935D
:106C50002505509326056093270570932805E0923B
:106C60001D05F0921E0500931F05109320058091CD
:106C700025039091260397FDA4C37C01F594E79426
:106C8000F594E794F594E794FAA6E9A68091230396
:106C90009091240397FD93C38C0115950795159545
:106CA0000795159507951CA70BA780912204909135
:106CB00023040F9734F458E1E52E5CEFF52EFAA685
:106CC000E9A68091220490912304079734F440E3CD
:106CD000E42E48EFF42EFAA6E9A6209102012A300C
:106CE00009F46BC28091220490912304815D974046
:106CF0000CF007C28091220490912304805E97409B
:106D000034F080EDE82E87E0F82EFAA6E9A680910F
:106D10002004909121040F9724F408E11CEF1CA794
:106D20000BA78091200490912104079724F400E39D
:106D300018EF1CA70BA72A3009F455C28091200434
:106D400090912104815D974024F008EE13E01CA788
:106D50000BA78091200490912104805E974024F03D
:106D600000ED17E01CA70BA7A0919903AA2309F433
:106D700097C06091250370912603809155059091ED
:106D80005605681B790B2091250330912603280FA7
:106D9000391F37FD3FC3359527953093560520930E
:106DA0005505613871050CF43AC260E870E07093E3
:106DB0005C0560935B058A2F9927869FF001879F6A
:106DC000F00D969FF00D1124CF01F7FD21C37C013A
:106DD000F594E794F594E794F594E794F594E794A3
:106DE00029A53AA5E20EF31EFAA6E9A640912303CF
:106DF000509124038091570590915805481B590BD9
:106E00002091230330912403280F391F37FDFDC241
:106E100035952795309358052093570541385105EE
:106E20000CF4F5C140E850E050935A0540935905E1
:106E30008A2F9927849FD001859FB00D949FB00D14
:106E40001124AD019D01B7FDDDC28901159507959E
:106E5000159507951595079515950795EBA5FCA52F
:106E60000E0F1F1F1CA70BA7869F9001879F300D39
:106E7000969F300D1124C9012091250330912603DE
:106E8000820F931F90932603809325038091230301
:106E900090912403480F591F5093240340932303D8
:106EA0004D855E85141615060CF0C1C18091DB0876
:106EB0009091DC0897FDA2C2AA2797FDA095BA2F52
:106EC0006DA5262F332744275527BC01CD010E94ED
:106ED000876B97FD8EC256E0959587957795679558
:106EE0005A95D1F7AF8DB8A1A60FB71FB093560929
:106EF000A09355094B855C85141615060CF0C1C18D
:106F00008091DF089091E00897FD6FC2AA2797FD56
:106F1000A095BA2F6DA5262F332744275527BC01EE
:106F2000CD010E94876B97FD5BC236E095958795F2
:106F3000779567953A95D1F7A9A1BAA1A60FB71F82
:106F4000B0934B09A0934A093CA137FDC1C11093EE
:106F5000490900934809F0925809E0925709809135
:106F6000E508E82FFF27EE0FFF1FE155F74F80815F
:106F7000918182599F4FA091E504B091E604A81732
:106F8000B9070CF0EEC0CD0101969093E604809312
:106F9000E504DC018091E608E82FFF27EE0FFF1FD4
:106FA000E155F74F8081918182599F4F6091E304B1
:106FB0007091E404681779070CF0C4C0CB01019606
:106FC0009093E4048093E304BC018091E708E82FE8
:106FD000FF27EE0FFF1FE155F74F80819181825906
:106FE0009F4F4091E1045091E204481759070CF07B
:106FF000D5C0CA0101969093E2048093E104AC01EC
:107000008091E808E82FFF27EE0FFF1FE155F74FAB
:107010008081918182599F4F2091DF043091E0045B
:10702000281739070CF0ABC0C90101969093E00412
:107030008093DF049C01B7FD93C1AF3FB10539F0E8
:1070400034F08FEF90E09093E6048093E50477FDB1
:1070500076C16F3F710539F034F08FEF90E0909377
:10706000E4048093E30457FD70C14F3F510539F0AC
:1070700034F08FEF90E09093E2048093E10437FDC9
:107080006AC12F3F310509F00CF4EEC28FEF90E09A
:107090009093E0048093DF04E7C260920905709248
:1070A0000A0580920B0590920C05A0920505B092FE
:1070B0000605C0920705D0920805ADCD20920105C6
:1070C000309202054092030550920405A092FD04FF
:1070D000B092FE04C092FF04D092000524CD98EB3C
:1070E000691694E979069EEF89069FEF99062CF5BB
:1070F00028EB34E94EEF5FEF29833A834B835C83BF
:107100001ACB98EEE92E93E0F92EFAA6E9A6F2CD75
:107110002D823E824F825886F4CA8DA19EA1AFA1D6
:10712000B8A58093F9049093FA04A093FB04B0935C
:10713000FC049091E9089CA312CC69827A828B822C
:107140009C82F9CA8081918182599F4F8617970747
:107150000CF03BCF6115710509F437CFCB010197D6
:107160002FCF8081918182599F4F8A179B070CF006
:1071700011CF109709F40ECFCD01019706CF808172
:10718000918182599F4F821793070CF054CF21159C
:10719000310509F450CFC901019748CF8081918111
:1071A00082599F4F841795070CF02ACF411551053E
:1071B00009F426CFCA0101971ECF80912204909135
:1071C0002304835F934034F038EEE32E33E0F32E54
:1071D000FAA6E9A680912204909123048A5F934045
:1071E0000CF495CD8ECD8091200490912104835F85
:1071F000934024F008EE13E01CA70BA78091200415
:10720000909121048A5F93400CF4AECDA9CD3FEF5D
:10721000403853070CF008CE40E85FEF05CE8FEF03
:10722000603878070CF0C3CD60E87FEFC0CD809167
:10723000DB089091DC0897FD9BC1AA2797FDA095DC
:10724000BA2FEDA52E2F332744275527BC01CD019A
:107250000E94876B97FDADC146E095958795779520
:1072600067954A95D1F72F8D38A1261B370B3093A0
:107270005609209355094B855C85141615060CF4A8
:107280003FCE8091DF089091E00897FD6DC1AA275D
:1072900097FDA095BA2FEDA52E2F3327442755270C
:1072A000BC01CD010E94876B97FD88C126E09595B2
:1072B0008795779567952A95D1F729A13AA1261B3D
:1072C000370B30934B0920934A093CA137FF3FCE3F
:1072D0004BA1442309F03BCE8091C604882309F0DA
:1072E00036CE8B859C85A1E081309A070CF044C195
:1072F0002B853C854FEF203034070CF0A3C189A5C6
:107300009AA5280F391F3C872B8720503F4F309379
:10731000580920935709AD85BE85E1E0A130BE072D
:107320000CF465C12BA53CA5A20FB31FBE87AD878A
:10733000A050B140B0934909A093480910CE1092D3
:10734000E4041092E30457FF90CE1092E2041092EE
:10735000E10437FF96CE1092E0041092DF0484C15E
:107360001092E6041092E50472CE295F3F4F3DC8AB
:10737000295F3F4F29C82D5F3F4F4F4F5F4FE5C8F3
:10738000E60EF71E081F191FE092AB09F092AC0938
:107390000093AD091093AE0958CB23E030E040E0F4
:1073A00050E0E20EF31E041F151FA3C883E090E017
:1073B000A0E0B0E0E80EF91E0A1F1B1F5BC807968D
:1073C0006BCC07965ACC2DA13EA14FA158A5209376
:1073D000F9043093FA044093FB045093FC04BFCAB1
:1073E000615C7F4F8F4F9F4FA0CD909581959F4FB0
:1073F0008DCD615C7F4F8F4F9F4F6DCD9095819567
:107400009F4F5ACD215F3F4F20CD2F5F3F4F00CD83
:107410000F96DDCC2F5F3F4FBECC2DA13EA14FA1DB
:1074200058A52093F9043093FA044093FB04509339
:10743000FC0489859A85AA2797FDA095BA2F2AADC5
:107440003BAD4CAD5DAD820F931FA41FB51F8B8B61
:107450009C8BAD8BBE8BBC01CD0129813A814B81C8
:107460005C810E94876B9B01AC0197FDBBC06BE008
:1074700055954795379527956A95D1F760918F0374
:10748000862F9927AA27BB278F8B988FA98FBA8F12
:10749000BC01CD010E94876B97FD9FC02CE09595A4
:1074A0008795779567952A95D1F76B8F7C8F8D8F10
:1074B0009E8F609345057093460580934705909392
:1074C00048056B897C898D899E892D813E814F81FC
:1074D00058850E94876B9B01AC0197FD79C08BE0BA
:1074E00055954795379527958A95D1F76F89788D6A
:1074F000898D9A8D0E94876B97FD65C0BCE095953C
:10750000879577956795BA95D1F76AAB7BAB8CABCE
:107510009DAB6093490570934A0580934B0590930A
:107520004C0529853A8537FD7FC0213431050CF49F
:1075300031CA6B8D7C8D8D8D9E8D97FD2AC06138F3
:1075400071058105910564F46AA97BA98CA99DA99F
:1075500097FD82C061387105810591050CF41ACA46
:1075600081E08093E90416CA909581959F4F8FCE54
:10757000909581959F4F61CEE9A5FAA58E0F9F1F2B
:107580009C878B878050914090935809809357092E
:10759000C2CE90958095709561957F4F8F4F9F4F8C
:1075A000CECF0196A11DB11D8EA79FA7A8ABB9ABE9
:1075B00097C9615C7F4F8F4F9F4F4ECE615C7F4F6D
:1075C0008F4F9F4F73CE6150704F8F4F9F4F96CF0D
:1075D0002150384F4F4F5F4F82CF6150704F8F4FC8
:1075E0009F4F5CCF2150384F4F4F5F4F40CF4D855D
:1075F0005E856FEF4030560754F58BA59CA5480F6C
:10760000591F5E874D8740505F4F50934909409303
:107610004809A5CC6150704F8F4F9F4FE7C821504C
:10762000384F4F4F5F4FCFC8309521953F4F7DCF9B
:107630006150704F8F4F9F4F0CC92150384F4F4FA3
:107640005F4FFAC8F0925809E092570964CE109340
:1076500049090093480983CC909580957095619570
:107660007F4F8F4F9F4F76CFED960FB6F894DEBFCA
:107670000FBECDBFDF91CF911F910F91FF90EF9083
:10768000DF90CF90BF90AF909F908F907F906F9042
:107690005F904F903F902F900895809102018D3020
:1076A00009F455C110927A0080912204909123042C
:1076B0009093580980935709809120049091210458
:1076C000909349098093480980911E0490911F046A
:1076D0009093A5098093A40980911A0490911B04AA
:1076E0009C01442737FD4095542FDA01C901880FCA
:1076F000991FAA1FBB1F880F991FAA1FBB1F820FAC
:10770000931FA41FB51F820F931FA41FB51F909333
:1077100094098093930980911C0490911D049C010D
:10772000442737FD4095542FDA01C901880F991F6E
:10773000AA1FBB1F880F991FAA1FBB1F820F931F71
:10774000A41FB51F820F931FA41FB51F9093B009EC
:107750008093AF0980911804909119049093630964
:10776000809362098FEC80937A008091E508E82F7E
:10777000FF27EE0FFF1FE155F74F8081918182595E
:107780009F4FA091E504B091E604A817B9070CF04B
:1077900085C0CD0101969093E6048093E504DC0159
:1077A0008091E608E82FFF27EE0FFF1FE155F74F06
:1077B0008081918182599F4F6091E3047091E4042C
:1077C000681779070CF096C0CB0101969093E404FA
:1077D0008093E304BC018091E708E82FFF27EE0FB8
:1077E000FF1FE155F74F8081918182599F4F409152
:1077F000E1045091E204481759070CF06CC0CA012B
:1078000001969093E2048093E104AC018091E80832
:10781000E82FFF27EE0FFF1FE155F74F8081918181
:1078200082599F4F2091DF043091E00428173907D7
:107830000CF042C0C90101969093E0048093DF04EC
:107840009C01B7FD7FC0AF3FB10511F00CF061C0E6
:1078500077FD67C06F3F710539F034F08FEF90E02E
:107860009093E4048093E30457FD61C04F3F5105BA
:1078700039F034F08FEF90E09093E2048093E104CC
:1078800037FD5BC02F3F310509F00CF463C08FEF6B
:1078900090E09093E0048093DF045CC0808191814C
:1078A00082599F4F8A179B070CF07ACF109709F4E3
:1078B00077CFCD0101976FCF8081918182599F4F02
:1078C000821793070CF0BDCF2115310509F4B9CF0C
:1078D000C9010197B1CF8081918182599F4F84174F
:1078E00095070CF093CF4115510509F48FCFCA01CC
:1078F000019787CF8081918182599F4F8617970783
:107900000CF069CF6115710509F465CFCB010197C2
:107910005DCF8FEF90E09093E6048093E50477FFCE
:1079200099CF1092E4041092E30457FF9FCF109276
:10793000E2041092E10437FFA5CF1092E004109208
:10794000DF0408C01092E6041092E50481CF0E9483
:10795000C31CA8CE809117099927AA27BB27BC0171
:10796000CD0124EC39E040E050E00E94876BDC015F
:10797000CB018093A6039093A703A093A803B09391
:10798000A903809118099927AA27BB27BC01CD011B
:107990000E94876BDC01CB018093A2039093A30329
:1079A000A093A403B093A50308956F927F928F9242
:1079B0009F92AF92BF92CF92DF92EF92FF920F937E
:1079C0001F93CF9300E010E078016801469A10936E
:1079D000380500933705109336050093350580E090
:1079E00090E0A0E0B0E080932F0590933005A09345
:1079F0003105B09332051093420500934105109371
:107A0000400500933F0510933E0500933D051093FC
:107A100075090093740910928F0310928E031092CF
:107A200012040E944D3B84E690E00E9417180E94C9
:107A30004D3B8091E90880FF10C080911D0390911B
:107A40001E03875B934008F0FBC180911D0390915A
:107A50001E038E5E924008F4F3C1CFE18AE090E00D
:107A60000E94171880911E0490911F04080F191F7F
:107A70008091220490912304E80EF91E8091200445
:107A800090912104C80ED91EC150C7FFE7CFA701AE
:107A9000405F5F4F569547955695479550934205E1
:107AA000409341059601205F3F4F369527953695C7
:107AB00027953093400520933F05C8014096969541
:107AC0008795929582958F7089279F7089279093CB
:107AD0003E0580933D05909375098093740930931A
:107AE0003C0520933B0550933A054093390544E00B
:107AF00050E0DA010E94166C802D853008F4A3C195
:107B00008091AF099091B00997FDD2C16CE070E00F
:107B10000E94C66B7093360560933505809193097A
:107B20009091940997FDD5C16CE070E00E94C66BFE
:107B300070933805609337058091690890916A08C1
:107B4000AA2797FDA095BA2FBC01CD010E940D6B0D
:107B5000DC01CB0180932F0590933005A093310574
:107B6000B0933205109258091092570910924909A2
:107B7000109248091092A5091092A40984E690E099
:107B80000E94171880911A0490911B04AA2797FD50
:107B9000A095BA2F9C01AD01220F331F441F551F22
:107BA000220F331F441F551F280F391F4A1F5B1F09
:107BB000280F391F4A1F5B1F3093940920939309A4
:107BC00080911C0490911D04AA2797FDA095BA2FBF
:107BD0007C018D01EE0CFF1C001F111FEE0CFF1C21
:107BE000001F111FE80EF91E0A1F1B1FE80EF91EC9
:107BF0000A1F1B1FF092B009E092AF098091F808AC
:107C0000682E772488249924C9019C01442737FDD4
:107C10004095542FC401B3010E94876B5B016C0136
:107C20006093290570932A0580932B0590932C056A
:107C30009701442737FD4095542FC401B3010E949A
:107C4000876BDC01CB018093210590932205A093E3
:107C50002305B0932405A0920505B0920605C092B5
:107C60000705D09208058093FD049093FE04A0932D
:107C7000FF04B09300051092F9041092FA041092D8
:107C8000FB041092FC0480911F0390912003A091AB
:107C90002103B091220390936C0880936B0810929B
:107CA0001104109210041092F1041092F204109238
:107CB000F3041092F4048091EF049091F0049093F7
:107CC000EE048093ED040E94DC6182E390E09093E7
:107CD000FC038093FB03809117099927AA27BB27F0
:107CE000BC01CD0124EC39E040E050E00E94876BFC
:107CF000DC01CB018856954CAF4FBF4F8093A60354
:107D00009093A703A093A803B093A90380911809A7
:107D10009927AA27BB27BC01CD010E94876BDC01F4
:107D2000CB018856954CAF4FBF4F8093A2039093E1
:107D3000A303A093A403B093A50310928B03109206
:107D40008A038091EF049091F004AA2797FDA095F3
:107D5000BA2F209186033091870340918803509178
:107D60008903BC01CD010E94876BDC01CB018093AC
:107D7000AB099093AC09A093AD09B093AE091092F2
:107D8000E8041092E70481E0809301010E94D1652C
:107D90008091AD0484608093AD048FEF8093140ACA
:107DA0001092150A80E28093160A8091E508E82F68
:107DB000FF27EE0FFF1FE155F74F80819181825918
:107DC0009F4F9093E6048093E5048091E608E82FA6
:107DD000FF27EE0FFF1FE155F74F808191818259F8
:107DE0009F4F9093E4048093E3048091E708E82F89
:107DF000FF27EE0FFF1FE155F74F808191818259D8
:107E00009F4F9093E2048093E1048091E808E82F6B
:107E1000FF27EE0FFF1FE155F74F808191818259B7
:107E20009F4F9093E0048093DF0484E68093DE0408
:107E30008091F903882309F450C0469A579A4DC09F
:107E40000E94711C0ACEDA010E94166C802D9927BF
:107E5000982F8827DA0111960E94166C202D820F28
:107E6000911D9093380580933705DA0112960E9490
:107E7000166C802D9927982F8827DA0113960E9477
:107E8000166C202D820F911D909336058093350539
:107E9000DA0114960E94166C802D9927982F882756
:107EA000DA0115960E94166C202D820F911D48CE86
:107EB000909581959F4F6CE070E00E94C66B709327
:107EC000360560933505809193099091940997FF49
:107ED0002BCE909581959F4F27CECF911F910F91DB
:107EE000FF90EF90DF90CF90BF90AF909F908F90DA
:107EF0007F906F9008959091D404992381F580919B
:107F0000AD048C7F8093AD0410C0A92FBB27FD0169
:107F1000E859F84F8083FD01E859F84F8081AA564F
:107F2000B64F8C939F5F9C3080F48091DC03882354
:107F300061F3A92FBB27FD01E859F84F8081AA56AC
:107F4000B64F8C939F5F9C3080F38091DC03882335
:107F500059F08091DC0381508093DC0305C080914F
:107F6000AD0481608093AD04809196099927909328
:107F70003E0880933D088091970999279093400887
:107F800080933F08809199099927909342088093A4
:107F90004108809198099927909344088093430859
:107FA00010924904109248040E94ED2A089580918D
:107FB000EC088B3F68F08B3F09F4D5C28C3F09F485
:107FC00074C38D3F09F4F6C28E3F21F48091DF0423
:107FD00080939E038091EB088B3F08F439C28B3F5E
:107FE00009F434C28C3F09F448C38D3F09F4D9C267
:107FF0008E3F09F478C380919F03882309F02DC236
:1080000080939F038091ED088B3F08F42DC28B3F36
:1080100009F428C28C3F09F442C38D3F09F4C4C25D
:108020008E3F09F45AC380919D03882309F021C231
:1080300080939D038091EF088B3F68F08B3F09F49C
:1080400095C28C3F09F42EC38D3F09F4B0C28E3F18
:1080500021F48091DF0480939C038091F1088B3F91
:1080600068F08B3F09F479C28C3F09F4E2C28D3F7E
:1080700009F4BEC28E3F21F48091DF0480939A03FD
:108080008091F9088B3F68F08B3F09F469C28C3FFF
:1080900009F4FCC28D3F09F490C28E3F21F4809117
:1080A000DF0480939B038091FA088B3F08F4E8C1BA
:1080B0008B3F09F4E3C18C3F09F4EEC28D3F09F414
:1080C00094C28E3F09F412C3809198038B3008F458
:1080D000DCC18F3F11F4809398038091FB088B3FA4
:1080E00068F08B3F09F427C28C3F09F4D2C28D3F60
:1080F00009F466C28E3F21F48091DF0480939703D8
:108100008091FC088B3F68F08B3F09F417C28C3FCD
:1081100009F489C28D3F09F46EC28E3F21F480912B
:10812000DF04809399038091FD088B3F68F08B3FBB
:1081300009F407C28C3F09F479C28D3F09F452C299
:108140008E3F21F48091DF04809396038091FE0896
:108150008B3F68F08B3F09F4F7C18C3F09F4ABC249
:108160008D3F09F43CC28E3F21F48091DF0480935F
:108170009503209103092B3F08F48BC12B3F09F491
:1081800086C12C3F09F47CC22D3F09F404C22E3F66
:1081900009F4A6C220919303809104098B3F08F053
:1081A0007FC18093C104809105098B3F68F08B3FAC
:1081B00009F4D0C18C3F09F466C28D3F09F4EEC1C9
:1081C0008E3F21F48091DF048093C00480910609E2
:1081D0008B3F68F08B3F09F484C18C3F09F471C276
:1081E0008D3F09F4D2C18E3F21F48091DF0480934A
:1081F000BF04809107098B3F68F08B3F09F474C17D
:108200008C3F09F461C28D3F09F4C2C18E3F21F455
:108210008091DF048093BE0480911C098B3F68F03D
:108220008B3F09F464C18C3F09F454C28D3F09F4BB
:10823000A3C18E3F21F48091DF048093BD0480911F
:108240001D098B3F68F08B3F09F454C18C3F09F442
:108250002FC28D3F09F493C18E3F21F48091DF043A
:108260008093BC0480911E098B3F68F08B3F09F41A
:1082700044C18C3F09F4ECC18D3F09F4C5C18E3F68
:1082800021F48091DF048093BB0480911F098B3F10
:1082900068F08B3F09F434C18C3F09F4DCC18D3F99
:1082A00009F4B5C18E3F21F48091DF048093BA04B4
:1082B000809108098B3F68F08B3F09F424C18C3F03
:1082C00009F4CFC18D3F09F484C18E3F21F4809120
:1082D000DF048093920380910C098B3F68F08B3F01
:1082E00009F414C18C3F09F4BFC18D3F09F474C176
:1082F0008E3F21F48091DF048093910380911109D6
:108300008B3F68F08B3F09F404C18C3F09F4AFC187
:108310008D3F09F458C18E3F21F48091DF04809392
:108320009003809114098B3F68F08B3F09F4F4C0EF
:108330008C3F09F49FC18D3F09F448C18E3F21F461
:108340008091DF0480938F03809115098B3F68F043
:108350008B3F09F4E4C08C3F09F46EC18D3F09F4F2
:108360004DC18E3F21F48091DF0480938E03809174
:1083700016098B3F68F08B3F09F4D4C08C3F09F499
:1083800064C18D3F09F43DC18E3F21F48091DF042B
:1083900080938D0380911B098B3F68F08B3F09F41C
:1083A000C4C08C3F09F45AC18D3F09F433C18E3FDC
:1083B00021F48091DF0480938C03809121098B3F0D
:1083C00008F47FC08B3F09F47AC08C3F09F437C1B1
:1083D0008D3F09F422C18E3F09F48BC180916F0952
:1083E000823008F473C08F3F11F480936F0980913D
:1083F00023098B3F08F46EC08B3F09F469C08C3FA2
:1084000009F420C18D3F09F40BC18E3F09F474C1FA
:108410008091A209823008F462C08F3F11F48093EA
:10842000A209809136098B3F70F08B3F09F480C020
:108430008C3F09F44CC18D3F09F49BC08E3F09F07D
:108440005EC18091DF048093B20959C18091E50437
:1084500080939F03882309F4D3CD843608F4D2CDCA
:1084600084E6CECD8091E50480939D03882309F4B2
:10847000DFCD843608F4DECD84E6DACD8091E504E4
:10848000809398038B3008F024CE8AE024CE20918C
:10849000E50420939303809104098B3F08F481CE77
:1084A0008B3F09F454C08C3F09F408C18D3F09F497
:1084B00069C08E3F09F077CE8091DF0472CE809143
:1084C000E50480936F09823008F08DCF81E08DCF75
:1084D0008091E5048093A209823008F09ECF81E06C
:1084E0009ECF8091E50483CE8091E50493CE809168
:1084F000E504A3CE8091E504B3CE8091E504C3CE1C
:108500008091E504D3CE8091E504E3CE8091E5042B
:10851000F3CE8091E50403CF8091E50413CF8091E1
:10852000E50423CF8091E50433CF8091E50443CF68
:108530008091E50488CF8091E504E0CD8091E50449
:10854000F0CD8091E50400CE8091E50410CE8091BD
:10855000E50427CE8091E50437CE8091E5048ECDE9
:108560008091E5049ECD8091E50432CD8091E504B3
:1085700072CD8091E10467CF8091E1045ECE80915D
:10858000E1046ECE8091E1040CCE8091E1042FCE07
:108590008091E1043FCE2091E1047BCF8091E10402
:1085A00013CE8091E10454CF8091E1045DCF80919E
:1085B000E10451CD8091E1040BCD8091E10471CDB6
:1085C0008091E1049BCD8091E104A9CE8091E104EA
:1085D000B9CE8091E1047DCE8091E1048DCE809171
:1085E000E104C5CD8091E104AFCD8091E10448CF95
:1085F0008091E10443CD8091E10493CD8091E10429
:10860000B4CE8091E104C4CE8091E1043CCE80914F
:10861000E1044CCE8091E104CECE8091E10451CFB3
:108620008091E10457CF8091E3047BCD8091E304F6
:108630008BCD8091E30422CD8091E30496CE80918E
:10864000E3043FCF8091E30445CF8091E304A0CEC3
:108650008091E30418CE8091E30428CE8091E30456
:10866000AACE8091E30435CE8091E30445CE80917B
:10867000E30455CE8091E30465CE8091E304E8CE17
:108680002091E30406CF8091E3049ECD8091E30422
:1086900008CD8091E30432CD8091E304F1CE809146
:1086A000E304E2CE8091E304D6CC8091E30490CC45
:1086B0008091E304D5CD8091E30459CD8091E3040A
:1086C00070CD8091E30493CD8091E304A3CD80919C
:1086D000E304B9CE8091E304B0CD8091DF04C4CE31
:1086E0002091DF04D6CE8091DF04B2CE8091DF04EA
:1086F000C7CE8091DF04E5CE8091DF04EBCE332737
:108700002F5F3F4F8CE398E2B9010E94C66B7093D4
:10871000A1036093A0038091F7088093A30980913F
:10872000F60880935C0908952F923F924F925F92D2
:108730006F927F928F929F92AF92BF92CF92DF9271
:10874000EF92FF920F931F93CF93DF93CDB7DEB7D6
:10875000ED970FB6F894DEBF0FBECDBF8091AC048D
:10876000815009F485E08093AC040E94B4312091DB
:1087700002012C3008F0BAC2299AA090D504B0901A
:10878000D604BA82A98280915C0999270A96A81614
:10879000B90614F49A8389838091DE04843608F044
:1087A000A7C28091790590917A05009709F081C45C
:1087B0001092D4048091AD048F7E8093AD042A3052
:1087C00009F47FC4243109F47CC428988091AE0454
:1087D0009091AF04895E934008F47CC480910009B5
:1087E000282F33273A8329838091AD0480618093B9
:1087F000AD048091E108A82FBB27AA0FBB1FFD0184
:10880000EB53F74F118210828091E208282F332713
:10881000220F331FC9018B53974FFC011182108225
:10882000A155B74F11961C921E922155374FD90171
:1088300011961C921E928091E408E82FFF27EE0FFC
:10884000FF1FE155F74F1182108280918403815000
:1088500080938403809184038F3F21F08091AD0445
:1088600084FF3BC40E94D73F809188059091890581
:10887000AC01440F551F480F591F0091E108A02F6C
:10888000BB27AA0FBB1FFD01E155F74FE090F3088E
:10889000CE2CDD24808191818C9D50018D9DB00C6A
:1088A0009C9DB00C11244A0D5B1D57FF02C00C9417
:1088B0008B585595479555954795AB53B74F809134
:1088C000F408682F77278D919C91869F9001879F50
:1088D000300D969F300D1124240F351F30938905DC
:1088E000209388058091BF059091C0054091BB05FC
:1088F0005091BC05840F951F281B390B3093DC0465
:108900002093DB0480918A0590918B05AC01440F84
:10891000551F480F591F1091E208A12FBB27AA0F1E
:10892000BB1FFD01E155F74F808191818C9D900126
:108930008D9D300D9C9D300D1124420F531F57FF0C
:1089400002C00C9487585595479555954795AB535C
:10895000B74F8D919C91869F9001879F300D969F78
:10896000300D1124240F351F30938B0520938A0579
:108970008091BD059091BE054091B9055091BA0511
:10898000840F951F281B390B3093DA042093D904E8
:108990008091E408E82FFF27EE0FFF1FE155F74F06
:1089A00080819181909581959F4F8330910514F43A
:1089B0000C94594F02979093D8048093D7048091D8
:1089C000E308E82FFF27EE0FFF1FE155F74FC080A8
:1089D000D18048E750E0C40ED51E809198039927B6
:1089E000AA2797FDA095BA2FBC01CD010E940D6B5F
:1089F000DC01CB0120E030E040E251E4BC01CD01DC
:108A00000E94AE6ADC01CB01BC01CD010E94F06A7C
:108A1000DC01CB018093A909F09097038091960324
:108A20009927AA2797FDA095BA2FBC01CD010E94D6
:108A30000D6BDC01CB0120E030E040E251E4BC01F1
:108A4000CD010E94AE6ADC01CB01BC01CD010E94C8
:108A5000F06ADC01CB0180934F095091950350934C
:108A6000660980918A0780FF06C08091B20981382B
:108A700010F00C94BC4FD092D604C092D5048091D3
:108A8000D5049091D60497FF02C00C948158F091C0
:108A9000E908FAA3F2FD02C00C94A34F10927609E4
:108AA0004091DB045091DC04CA0157FF02C00C94D2
:108AB000AE4F959587959595879597FF02C00C9435
:108AC000B74F2091B2043091B3042817390714F03E
:108AD0000C94614FCA0157FF02C00C944C5C97FF85
:108AE00002C00C94515CBC017595679575956795AE
:108AF0006536710514F40C94644F64E670E040919F
:108B0000D9045091DA04CA0157FD02C00C946D4F8C
:108B10000396959587959595879597FD02C00C943A
:108B2000754F909581959F4F2091B0043091B1047D
:108B30002817390714F40C947E4F2150304080914F
:108B4000AD0484FD02C00C94994F1092B3041092AE
:108B5000B2041092B1041092B004E12FFF27EE0F7F
:108B6000FF1FE155F74F40911209242F33278081D1
:108B700091812817390734F48091370982FF02C0A8
:108B80000C943050E12FFF27EE0FFF1FE155F74FF8
:108B9000842F992720911309821B9109208131810B
:108BA0002817390714F41092C504E12FFF27EE0FA0
:108BB000FF1FE155F74F842F992722273327281BC2
:108BC000390B808191818217930734F480913709A2
:108BD00083FF02C00C942B508091C404882391F031
:108BE000E12FFF27EE0FFF1FE155F74F809113098B
:108BF0009927841B9109208131818217930714F4EE
:108C00000C945C50E02FFF27EE0FFF1FE155F74F4C
:108C1000242F3327808191812817390734F48091DC
:108C2000370980FF02C00C9425505091C20455238F
:108C300099F0E02FFF27EE0FFF1FE155F74F842F2C
:108C4000992720911309821B9109208131812817CE
:108C5000390714F40C945750E02FFF27EE0FFF1F35
:108C6000E155F74F842F992722273327281B390BEB
:108C7000808191818217930734F48091370981FFB5
:108C800002C00C9420508091C304882391F0E02FFF
:108C9000FF27EE0FFF1FE155F74F8091130999272A
:108CA000841B9109208131818217930714F40C945D
:108CB00060508091C504882331F48091C4048823D6
:108CC00011F40C941D5091E0552331F48091C304AC
:108CD000882311F40C943B5081E08093C7041092D8
:108CE000C6041092C5041092C404FAC1299845CD57
:108CF0008091DE048D3808F4A8CD8091AD048F7E7C
:108D00008093AD049091010982E3989FC0011124E2
:108D100090937A0580937905E981FA81B99714F0E7
:108D20000C9440508091AE049091AF048F3F910518
:108D300019F010F00C947A5810925D0510925E05AF
:108D400010925F0510926005109261051092620505
:108D500010926305109264058A3F910511F40C94FA
:108D6000A05D3091E308E32FFF27EE0FFF1FE155D1
:108D7000F74F80819181813591050CF4E9C04091D4
:108D8000D404442309F0E4C08091E408E82FFF27CD
:108D9000EE0FFF1FE155F74F808191818C349105D3
:108DA00014F40C94E75C80917B058F5F893C10F490
:108DB0000C94D15D2C3010F00C94A75F2998109280
:108DC000D40410927B051092AF041092AE0400916F
:108DD000E108E02FFF27EE0FFF1FE155F74F8081DD
:108DE00091818734910514F00C94615F1091E20831
:108DF000E12FFF27EE0FFF1FE155F74F8081918193
:108E00000190F081E02DF7FF02C00C944B61E73434
:108E1000F1050CF470C021E0A12FBB27AA0FBB1FE6
:108E2000A155B74F8D919C9111978734910544F0CE
:108E3000E02FFF27EE0FFF1FE155F74F8081918153
:108E40008D919C918734910564F0E02FFF27EE0F00
:108E5000FF1FE155F74F80819181873491050CF018
:108E600022E0E12FFF27EE0FFF1FE155F74F808132
:108E700091818634910564F4E02FFF27EE0FFF1FE8
:108E8000E155F74F80819181873491050CF023E003
:108E9000E12FFF27EE0FFF1FE155F74F80819181F2
:108EA0008A5B9F4F64F4E02FFF27EE0FFF1FE15511
:108EB000F74F80819181873491050CF024E0E12FF8
:108EC000FF27EE0FFF1FE155F74F808191818A5BED
:108ED0009F4F64F4E02FFF27EE0FFF1FE155F74F80
:108EE00080819181863491050CF425E0822F0E94C7
:108EF0007A051091E208E12FFF27EE0FFF1FE155E1
:108F0000F74F808191810190F081E02DF7FF02C041
:108F10000C9472607E9714F00C944D5E8091E10881
:108F2000E82FFF27EE0FFF1FE155F74F808191815A
:108F30008A5B9F4F14F00C944D5E81E080937E0716
:108F400088EE93E09093FC038093FB033091E30859
:108F5000E32FFF27EE0FFF1FE155F74F808191812F
:108F60008B5A9F4F0CF071CCD090E408ED2DFF2769
:108F7000EE0FFF1FE155F74F80819181855B9F4F79
:108F800014F00C949D5980917C058F5F893C10F4FE
:108F90000C94DB5C88EC80937C0581E090E09093FE
:108FA000AF048093AE0481E08093D40410926505F1
:108FB0001092660510926705109268051092F904E8
:108FC0001092FA041092FB041092FC041092F50423
:108FD0001092F6041092F7041092F8048091F808A9
:108FE000E82EFF240027112780919309909194097E
:108FF0009C01442737FD4095542FC801B7010E94BA
:10900000876BDC01CB018093090590930A05A0933F
:109010000B05B0930C058091AF099091B0099C01AC
:10902000442737FD4095542FC801B7010E94876B34
:10903000DC01CB018093010590930205A093030509
:10904000B09304058091290590912A05A0912B05E4
:10905000B0912C058093050590930605A093070514
:10906000B09308058091210590912205A0912305D8
:10907000B09124058093FD049093FE04A093FF0417
:10908000B093000510925D0510925E0510925F0589
:1090900010926005109261051092620510926305AE
:1090A000109264058091AD0488608093AD040C94A7
:1090B0009F59019790937A05809379052A3009F09A
:1090C00081CB289A8091AE049091AF04895E934041
:1090D00008F084CB1092D404B8CBA090E908AAA2DF
:1090E0000091C6040E8B002321F48091C7048823CD
:1090F00069F080911109992729813A818217930794
:1091000014F49A83898381E08093E9048091AD040B
:1091100084FFCBC61092D8041092D7041092DC04BE
:109120001092DB041092DA041092D9049AE590931D
:10913000A90988E78093760990934F0989A38093C2
:1091400066091092C6041092C7041E8A209169090C
:1091500030916A0940916B0950916C096091290521
:1091600070912A0580912B0590912C05698B7A8B43
:109170008B8B9C8B260F371F481F591F80917009BE
:1091800090917109A0917209B0917309A090210585
:10919000B0902205C0902305D0902405AFA2B8A6B8
:1091A000C9A6DAA68A0D9B1DAC1DBD1DC0905E0927
:1091B000D0905F09E0906009F0906109C8AAD9AA2F
:1091C000EAAAFBAAE0902505F09026050091270564
:1091D00010912805E88EF98E0A8F1B8FA8A8B9A8D0
:1091E000CAA8DBA8AE0CBF1CC01ED11EA8AAB9AA73
:1091F000CAAADBAAC0905009D0905109E090520948
:10920000F0905309CCA6DDA6EEA6FFA6E0901D05C2
:10921000F0901E0500911F0510912005EBA2FCA205
:109220000DA31EA3ACA4BDA4CEA4DFA4AE0CBF1C92
:10923000C01ED11EACA6BDA6CEA6DFA6B090C704A8
:10924000BF8ABB2009F0D0C50E89002309F0CCC528
:109250008093700990937109A0937209B093730978
:109260002093690930936A0940936B0950936C0904
:109270008091690890916A08815092400CF07EC4F8
:109280008091D404882309F079C480910E049091D0
:109290000F048F3F910509F008F47FC5BF89BB23F8
:1092A00009F017C7EE89EE2309F013C7F091E9041E
:1092B000FD8BFF2309F00DC7A0901A09ABA6AA20C9
:1092C00009F407C7C8A8D9A8EAA8FBA8C0925E09F4
:1092D000D0925F09E0926009F0926109ECA4FDA4CC
:1092E0000EA51FA5E0925009F09251090093520972
:1092F000109353098091690990916A09A0916B09B3
:10930000B0916C09B7FF02C00C94E55F292E3A2E8C
:109310004B2E552447FC5A942092690930926A09D1
:1093200040926B0950926C0980917009909171097B
:10933000A0917209B0917309B7FF02C00C94DF5F6E
:10934000892F9A2FAB2FBB27A7FDBA958D839E83BC
:10935000AF83B8878093700990937109A0937209C5
:10936000B09373098091F808E82EFF240027112795
:109370002091190530911A0540911B0550911C054B
:10938000C801B7010E94876B97FF02C00C94FD5F74
:10939000672E782E892E992487FC9A9420911505A2
:1093A000309116054091170550911805C801B70175
:1093B0000E94876B97FF02C00C94F75FA72EB82E10
:1093C000C92EDD24C7FCDA94D201C10186199709A0
:1093D000A809B90920911909E22EFF2400271127B5
:1093E000BC01CD01A80197010E94FB6B39014A0124
:1093F00019012A018D819E81AF81B8858A199B0947
:10940000AC09BD09BC01CD01A80197010E94FB6B0D
:10941000D401C30197FE02C00C94F15F892F9A2FEB
:10942000AB2FBB27A7FDBA95BC01DA01C90157FFD5
:1094300002C00C94EB5F892F9A2FAB2FBB27A7FD9F
:10944000BA956C018091B2049091B3048134910576
:10945000D4F48091B0049091B104813491059CF4CE
:109460008091E408E82FFF27EE0FFF1FE155F74F2B
:10947000808191810190F081E02DF7FF02C00C9472
:109480005C617A9734F08091140A8F3F11F40C9448
:10949000915F088D198D2A8D3B8D89899A89AB89B9
:1094A000BC89081B190B2A0B3B0B0AAF1BAF2CAF57
:1094B0003DAF0093690510936A0520936B053093C7
:1094C0006C05EBA0FCA00DA11EA12FA138A549A5FC
:1094D0005AA5E21AF30A040B150BE986FA860B87E4
:1094E0001C87E0926D05F0926E0500936F05109356
:1094F00070058AAD9BADACADBDAD80937105909309
:109500007205A0937305B0937405E0927505F0920F
:109510007605009377051093780580910505909165
:109520000605A0910705B0910805EAACFBAC0CADAF
:109530001DAD8E199F09A00BB10B8093050590936B
:109540000605A0930705B09308058091FD0490914E
:10955000FE04A091FF04B091000509851A852B85B2
:109560003C85801B910BA20BB30B8093FD04909361
:10957000FE04A093FF04B09300051BA5112371F115
:109580002091E7043091E8042138310594F080916E
:109590003D0590913E05019690933E0580933D05D3
:1095A0008091740990917509019690937509809343
:1095B000740920583F4F94F480913D0590913E05E9
:1095C000019790933E0580933D0580917409909199
:1095D0007509019790937509809374091092E804B6
:1095E0001092E70401E0A02EB12C8AAD9BADACAD8A
:1095F000BDADB7FF02C00C94B35F81509240A04054
:10960000B0401CF014E0A12EB12C809192059091F5
:109610009305A0919405B0919505E0906909F090AB
:109620006A0900916B0910916C098E199F09A00BB2
:10963000B10B815E914BAF4FBF4F8F539C49A04000
:10964000B04010F40C94E35DF091150AFC8FF931F1
:1096500014F40C947B5FB0928D05A0928C058AADBA
:109660009BADACADBDAD81509041A040B04014F475
:109670000C94EC5D80918E05882311F40C940360AA
:109680007093C9046093C8048AAD9BADACADBDAD09
:10969000B7FF02C00C9442619C01AD01B7FF02C04C
:1096A0000C943C61B9E05595479537952795BA9547
:1096B000D1F780918C0590918D05820F931F909327
:1096C0008D0580938C052AAD3BAD4CAD5DAD57FF4C
:1096D00002C00C94366139014A01A3E09594879445
:1096E00077946794AA95D1F713012401F9E86F16CE
:1096F000F3E17F06F0E08F06F0E09F0644F0F8E823
:109700006F2EF3E17F2E812C912C13012401D401C3
:10971000C30197FE02C00C947061892F9A2FAB2F62
:10972000BB27A7FDBA95680F791F2AAD3BAD4CAD9D
:109730005DAD203080EF38078FEF48078FEF580777
:1097400014F00C94FC5D80918F05882311F40C9427
:10975000D25F7093C9046093C804DA01C90157FF4E
:1097600002C00C942D619C01AD01B7FF02C00C94A6
:10977000856169E055954795379527956A95D1F7A5
:1097800080918C0590918D05820F931F90938D058C
:1097900080938C052AAD3BAD4CAD5DAD57FF02C04B
:1097A0000C947F6139014A0143E095948794779442
:1097B00067944A95D1F798E769169CEE79069FEF72
:1097C00089069FEF990644F438E7632E3CEE732E2A
:1097D0003FEF832E3FEF932E6092800570928105BC
:1097E0008092820590928305D401C30197FE02C046
:1097F0000C942761892F9A2FAB2FBB27A7FDBA9511
:109800006091C8047091C904680F791FABA52A2F15
:10981000332780918C0590918D052817390724F402
:1098200030938D0520938C05BC8DBB2379F02B2FB5
:10983000332727FD309580918C0590918D05281751
:10984000390724F430938D0520938C052AAD3BAD68
:109850004CAD5DAD213831054105510574F0809165
:1098600041059091420520918C0530918D05820F24
:10987000931F90934205809341058AAD9BADACAD9B
:10988000BDAD80589F4FAF4FBF4F74F480914105DD
:109890009091420520918C0530918D05821B930B90
:1098A0009093420580934105B1E0AB2EB12C8985A0
:1098B0009A85AB85BC85B7FF02C00C94C95F815007
:1098C0009240A040B0401CF0A4E0AA2EB12C20E0B1
:1098D00030E040E050E08091960590919705A0918E
:1098E0009805B09199056090700970907109809009
:1098F00072099090730986199709A809B909815EC0
:10990000914BAF4FBF4F8F539C49A040B04028F0C0
:10991000FC8DF93114F40C94655FB0928D05A09222
:109920008C0589859A85AB85BC8581509041A04086
:10993000B04014F40C94F05D80919005882311F4EC
:109940000C94BC5FD092CB04C092CA0489859A85DE
:10995000AB85BC85B7FF02C00C947661B7FF02C02F
:109960000C942161F9E0B595A79597958795FA959F
:10997000D1F7A80EB91EB0928D05A0928C0529854D
:109980003A854B855C8557FF02C00C941B61E3E070
:109990005595479537952795EA95D1F72938F3E1FD
:1099A0003F07F0E04F07F0E05F0714F40C94B1605C
:1099B00088E893E1A0E0B0E080938405909385056A
:1099C000A0938605B09387058091840590918505C5
:1099D000A0918605B0918705B7FF02C00C94FF6087
:1099E000892F9A2FAB2FBB27A7FDBA95C090CA0429
:1099F000D090CB04C80ED91E29853A854B855C854D
:109A0000203080EF38078FEF48078FEF580714F0AA
:109A10000C94085E80919105882311F40C94AA5F40
:109A2000D092CB04C092CA04DA01C90157FF02C028
:109A30000C9467619C01AD01B7FF02C00C94616199
:109A4000B9E05595479537952795BA95D1F7809107
:109A50008C0590918D05820F931F90938D058093B7
:109A60008C0529853A854B855C8557FF02C00C948F
:109A70000961A3E05595479537952795AA95D1F7A4
:109A800028379CEE39079FEF49079FEF590714F0DD
:109A90000C94BB6088E79CEEAFEFBFEF809384052A
:109AA00090938505A0938605B093870580918405E2
:109AB00090918505A0918605B0918705B7FF02C0FA
:109AC0000C945661892F9A2FAB2FBB27A7FDBA950F
:109AD000C090CA04D090CB04C80ED91EABA52A2FC3
:109AE000332780918C0590918D052817390724F430
:109AF00030938D0520938C05BC8DBB2379F02B2FE3
:109B0000332727FD309580918C0590918D0528177E
:109B1000390724F430938D0520938C0529853A85E7
:109B20004B855C85213831054105510574F08091E4
:109B30003F059091400520918C0530918D05820F55
:109B4000931F9093400580933F0589859A85AB8547
:109B5000BC8580589F4FAF4FBF4F0CF0D0C2809153
:109B60003F059091400520918C0530918D05821B19
:109B7000930B9093400580933F05C1C29090140AC7
:109B80006FEF961611F40C9491588091F808A82E56
:109B9000BB24CC24DD2469897A898B899C89A60120
:109BA00095010E94FB6B79018A0180919309909144
:109BB0009409AA2797FDA095BA2FE81AF90A0A0B6B
:109BC0001B0B6FA178A589A59AA5A60195010E94F6
:109BD000FB6B59016A018091AF099091B009AA27E6
:109BE00097FDA095BA2FA81AB90ACA0ADB0A292C30
:109BF000332427FC3094432C532CC201B101A8011B
:109C000097010E94876B97FD5FC23B014C01F9E011
:109C10009594879477946794FA95D1F7C201B1012E
:109C2000A60195010E94876B97FF02C00C94A45C6B
:109C30005B016C01E9E0D594C794B794A794EA95C9
:109C4000D1F78091B2049091B304813491053CF432
:109C50008091B0049091B10481349105C4F0D40195
:109C6000C30197FE02C00C949B5D3C014D0195948D
:109C7000879477946794D601C501D7FE02C00C94EF
:109C8000965D5C016D01D594C794B794A7948091BB
:109C9000E408E82FFF27EE0FFF1FE155F74F808103
:109CA00091810190F081E02DF7FF02C00C949F5C40
:109CB0007A97A4F0C401B30123E030E040E050E023
:109CC0000E94FB6B39014A01C601B50123E030E077
:109CD00040E050E00E94FB6B59016A018091160A36
:109CE000282F332727FD3095432F532F261537056F
:109CF0004805590514F439014A01992787FD9095C3
:109D0000909581959F4FAA2797FDA095BA2F681629
:109D100079068A069B0614F43C014D012A153B0581
:109D20004C055D0514F459016A01A816B906CA0666
:109D3000DB0614F45C016D018091090590910A0520
:109D4000A0910B05B0910C0586199709A809B909CE
:109D50008093090590930A05A0930B05B0930C0519
:109D60008091010590910205A0910305B091040531
:109D70008A199B09AC09BD098093010590930205DE
:109D8000A0930305B093040580910E0490910F04F5
:109D90008F3F910511F008F081CAA8A8B9A8CAA8F8
:109DA000DBA8A0925E09B0925F09C0926009D092D0
:109DB0006109CCA4DDA4EEA4FFA4C0925009D09206
:109DC0005109E0925209F09253090091E9040D8B78
:109DD000A090D704B090D804C501B7FEF0C1882781
:109DE00099278A199B09EBC11092190510921A053F
:109DF00010921B0510921C05109215051092160565
:109E000010921705109218051092690910926A09AC
:109E100010926B0910926C091092700910927109DE
:109E200010927209109273091CA61DA61EA61FA6E9
:109E300020E030E040E050E028AB39AB4AAB5BAB10
:109E40008091090590910A05A0910B05B0910C0530
:109E50008093050590930605A0930705B093080528
:109E60008091010590910205A0910305B091040530
:109E70008093FD049093FE04A093FF04B09300052B
:109E800010920F0410920E041092C9041092C8048C
:109E90001092CB041092CA043F89332309F0F5C90C
:109EA0004E89442309F0F1C9E3C93091660939A309
:109EB0004DC93FEF8E3F93070CF0D7C002960C942C
:109EC000DB44B901615070404091D9045091DA04EB
:109ED000CA0157FF02C00C948845959587959595C2
:109EE000879597FF02C00C9491452091B004309162
:109EF000B1042817390714F00C949D45CA0157FF87
:109F000002C00C94575C97FF02C00C94545C9C01F7
:109F100035952795359527952536310514F40C94FC
:109F20009F4524E630E08091AD0484FF02C00C948C
:109F3000A5453093B1042093B0047093B3046093AB
:109F4000B2040C94AD45F09276094091DB04509137
:109F5000DC04CA0157FD02C00C945945039695953F
:109F600087959595879597FD02C00C9461459095CE
:109F700081959F4F0C94614580918307992787FDB8
:109F800090954E2D5527849FB001859F700D949F0D
:109F9000700D1124CB012091DB043091DC04820F81
:109FA000931F9093DC048093DB04809184079927AE
:109FB00087FD9095849FD001859FB00D949FB00D33
:109FC0001124CD012091D9043091DA04820F931F1E
:109FD0009093DA048093D90480918507992787FDAF
:109FE00090952091D7043091D804820F931F9093BD
:109FF000D8048093D70480918707282F332727FD23
:10A0000030958091EE089927289FF001299FF00D47
:10A01000389FF00D1124F0938B03E0938A03809115
:10A02000860799278C159D0514F00C943B45909359
:10A03000D6048093D5040C943F45982F0C94644625
:10A0400081E08093C3040C94594681E08093C2045C
:10A05000582F0C942C4681E08093C4040C94024643
:10A0600081E08093C5040C94D5451092D8041092D9
:10A07000D7040C94DF449093C6048093C70430C87F
:10A080008091D404882311F40C9492468091AE04FC
:10A090009091AF04FFEF8F3F9F0711F40C94964609
:10A0A00001969093AF048093AE040C949646109260
:10A0B000C20450E00C942C461092C4040C94024646
:10A0C0001092C3040C94594661507E4F8F4F9F4F9E
:10A0D0009CCD60E070E06B011092E9041D8AE09075
:10A0E0006909F0906A0900916B0910916C09609000
:10A0F0007009709071098090720990907309809135
:10A100007609882309F0B6C71092CB041092CA04CE
:10A110001092C9041092C804E0929205F09293053F
:10A12000009394051093950560929605709297059B
:10A1300080929805909299051092190510921A052F
:10A1400010921B0510921C05109215051092160511
:10A150001092170510921805109211051092120511
:10A1600010921305109214051092690910926A0951
:10A1700010926B0910926C0910927009109271097B
:10A18000109272091092730910925E0910925F0981
:10A1900010926009109261091092500910925109B1
:10A1A000109252091092530910920F0410920E044B
:10A1B000A090D704B090D804C501B7FC10CE40974A
:10A1C00074F068EE262E63E0362E3092AB032092B8
:10A1D000AA031AA114FD03C081E080937F05D090EB
:10A1E000F508ED2CFF2400271127B501882777FDFE
:10A1F0008095982F9501B7FC78C7442737FD409587
:10A20000542F0E94876B9B01AC01C801B7010E94CB
:10A21000876B97FD65C759E0959587957795679505
:10A220005A95D1F79B018D2D99278A9DA0018B9D71
:10A23000500D9A9D500D1124CA0157FD43C79595A5
:10A24000879595958795280F391FC901AA2797FDEE
:10A25000A095BA2F8093650590936605A093670536
:10A26000B0936805E090F904F090FA040091FB04C3
:10A270001091FC04E81AF90A0A0B1B0B51E5E516CC
:10A2800053ECF50650E0050750E015070CF4E9C65D
:10A2900080E593ECA0E0B0E08093F9049093FA0499
:10A2A000A093FB04B093FC048091F9049091FA040C
:10A2B000A091FB04B091FC04805B9C43AF4FBF4F67
:10A2C00064F480EB9CE3AFEFBFEF8093F9049093CD
:10A2D000FA04A093FB04B093FC04C090EF04D09068
:10A2E000F004C114D10409F4B5C57AA173FFB2C555
:10A2F00089899A89AB89BC89B7FF02C00C946E5CCE
:10A3000009E0B595A795979587950A95D1F79BAFE5
:10A310008AAF97FF02C00C947A5C8FA198A5A9A57B
:10A32000BAA5B7FF02C00C94745C19E0B595A79567
:10A33000979587951A95D1F7BC0197FF02C00C94A9
:10A34000695CAAADBBADA617B70714F47BAF6AAFC3
:10A350006AAD7BAD77FF02C00C94655C2B01559410
:10A36000479455944794559447940894411C511C24
:10A37000ECE1F2E0CE0EDF1E76010027F7FC00953F
:10A38000102FA4EEAA2EADEFBA2ECA0CDB1C6090E3
:10A39000AB097090AC098090AD099090AE09209106
:10A3A00086033091870340918803509189032D8F54
:10A3B0003E8F4F8F58A3C401B3010E94FB6BE21A7A
:10A3C000F30A040B150BC801B70128E631E040E0A1
:10A3D00050E00E94FB6BDC01CB018C01045B104060
:10A3E000A090A409B090A509C501B7FE02C00C94C5
:10A3F0005F5C8138910514F000E010E02090AA0322
:10A400003090AB0321143104A9F44AAD5BAD49315E
:10A41000510584F48091E7049091E804800F911F26
:10A420009093E8048093E70480917F05882311F0DE
:10A430000C94715DC801880F991F880F991F880FB0
:10A44000991FB2010E94C66B9B01442737FD4095BE
:10A45000542F260D371D481D591D2093AB093093ED
:10A46000AC094093AD095093AE09F0909B036F2D5A
:10A470007727AAADBBAD6A9FC0016B9F900D7A9FF5
:10A48000900D112497FF02C00C945C5C9595879504
:10A4900095958795959587959595879595958795A4
:10A4A000681B790B7BAF6AAF77FF02C00C94815CAD
:10A4B0002114310411F00C94965C0091B2041091B7
:10A4C000B3048091B0049091B104080F191F17FFD5
:10A4D00002C00C94BE5D15950795159507951595C9
:10A4E0000795005C1F4FCA01B9012D8D3E8D4F8D20
:10A4F00058A10E94FB6BDA01C9012091ED04309153
:10A50000EE04442737FD4095542F821B930BA40B78
:10A51000B50B845E9D4FAF4FBF4FBC01CD0128E608
:10A5200031E040E050E00E94FB6BDC01CB01845B3A
:10A5300090402AAD3BAD829FF001839FF00D929F2A
:10A54000F00D1124CF01B8010E94C66B83E0F89E84
:10A55000A00111245BAF4AAF4617570714F00C94C3
:10A56000895CBA01CB01AA2797FDA095BA2F20914B
:10A57000F9043091FA044091FB045091FC04820FDD
:10A58000931FA41FB51F8093F9049093FA04A0931E
:10A59000FB04B093FC0480917E0581508F3F09F449
:10A5A00062C480937E055D89552381F01092610518
:10A5B00010926205109263051092640510925D0579
:10A5C00010925E0510925F05109260056F896623F8
:10A5D00009F044C5809176099927AA27BB27BC01B9
:10A5E000CD0129893A894B895C890E94876BDC01FE
:10A5F000CB01BC01CD0128EF3AE240E050E00E94DF
:10A60000FB6B19017E89772309F025C580917609B6
:10A610009927AA27BB27BC01CD012FA138A549A5A1
:10A620005AA50E94876BDC01CB01BC01CD0128EF4C
:10A630003AE240E050E00E94FB6B3C832B83809029
:10A640004A0990904B0989EC881691040CF4F8C4DF
:10A65000B8EC8B2E912C90924B0980924A09009174
:10A66000550910915609093C11050CF4E1C408EC98
:10A6700010E0109356090093550980915709909165
:10A680005809AA2797FDA095BA2F2091A909C22E93
:10A69000DD24EE24FF24BC01CD01A70196010E9418
:10A6A000876B9B01AC01C401AA2797FDA095BA2F27
:10A6B000F7E0880F991FAA1FBB1FFA95D1F7280F43
:10A6C000391F4A1F5B1F57FDECC4E6E055954795BF
:10A6D00037952795EA95D1F74101820E931E240103
:10A6E0008091480990914909AA2797FDA095BA2F12
:10A6F000BC01CD01A70196010E94876B9B01AC01B3
:10A70000C801AA2797FDA095BA2F77E0880F991F57
:10A71000AA1FBB1F7A95D1F7280F391F4A1F5B1F4D
:10A7200057FDBAC466E055954795379527956A95C4
:10A73000D1F76B807C80620E731E6301AA0CBB1C78
:10A74000C501AA2797FDA095BA2F20914F0933275D
:10A7500044275527BC01CD010E94876B7B018C01EA
:10A7600097FD91C456E015950795F794E7945A958F
:10A77000D1F739A1832F9927AA27BB2720910D054F
:10A7800030910E0540910F0550911005BC01CD018F
:10A790000E94876BDC01CB01BC01CD0120EF35E5C8
:10A7A00040E050E00E94FB6B5701A20EB31EC501B2
:10A7B00041E0841640E4940624F0812C40E4942E79
:10A7C000240150E0851650EC95060CF02CC4812C29
:10A7D00030EC932E909258098092570961E06616EA
:10A7E00060E4760624F0612C20E4722E630170E0B0
:10A7F000671670EC77060CF011C4612C00EC702E1B
:10A800007092490960924809A1E0AA16A0E4BA062C
:10A8100024F0A12C10E4B12EC501B0E0AB16B0ECD1
:10A82000BB060CF0F6C3A12CB0ECBB2EB092A50970
:10A83000A092A40980910001482F552780912703F9
:10A84000909128034817590794F4209127033091D9
:10A850002803E981FA814E9FC0014F9F900D5E9FB2
:10A86000900D1124B9010E94B26B7A836983C9806B
:10A87000DA80CC0CDD1CCC0CDD1CDA82C982DAA0BB
:10A88000D0FE51C00E89002309F04DC01F8911234D
:10A8900009F049C080919E0590919F0590935008C2
:10A8A00080934F08809110049091110490934A086E
:10A8B00080934908209143053091440521153105C5
:10A8C00009F0F8C480911D0390911E0389599340AB
:10A8D00010F00C94DE5C80911D0390911E03843671
:10A8E000910510F00C94D95D87B58B3010F40C9461
:10A8F000745E809112048F5F809312049AE0890243
:10A900009001112480917308821B87BD8CE291E035
:10A910009093FC038093FB038EE591E090934405B4
:10A9200080934305E8C45090A30940905C09242D0E
:10A930003327C901880F991F880F991F8896E981CD
:10A94000FA81E817F90714F49A838983852D9927EA
:10A95000880F991F880F991F80559040C980DA8011
:10A960008C159D0514F49A8389838091460488236D
:10A97000A1F08091AE049091AF040297C09768F463
:10A98000E980FA801E141F0444F481E090E0909363
:10A99000AF048093AE043A83298309811A8110930E
:10A9A0003408009333088091650590916605A09165
:10A9B0006705B0916805880F991FAA1FBB1F880FF4
:10A9C000991FAA1FBB1FA81AB90AB9AEA8AE013AAF
:10A9D00011050CF40AC3C80117FDA1C3959587950D
:10A9E00028AD39AD8217930714F499AF88AF9095CD
:10A9F00081959F4F48AD59AD4817590714F499AF49
:10AA000088AF252D3327220F331F220F331FC90193
:10AA100049815A81841B950B68AD79AD86179707DC
:10AA200014F499AF88AF89819A81821B930BA8ADEA
:10AA3000B9ADA817B90714F499AF88AF8091DB04BA
:10AA40009091DC048401081B190B10936809009392
:10AA50006709A0907609AA2009F4C1C2281A390A08
:10AA6000C101AA2797FDA095BA2F20915D053091CD
:10AA70005E0540915F0550916005820F931FA41FF2
:10AA8000B51F80935D0590935E05A0935F05B0931D
:10AA9000600560915D0570915E0580915F05909104
:10AAA00060056130BAEF7B07B0E08B07B0E09B0731
:10AAB00074F080E09AEFA0E0B0E080935D059093A1
:10AAC0005E05A0935F05B0936005BC01CD016030C9
:10AAD000E6E07E07EFEF8E07EFEF9E0774F480E06D
:10AAE00096E0AFEFBFEF80935D0590935E05A09376
:10AAF0005F05B0936005BC01CD01E090A003F0902C
:10AB0000A1039701442737FD4095542F0E94FB6B0A
:10AB10006801C20ED31EB0908C036B2D7727882757
:10AB2000992728AD39AD37FDC9C237FDC4C2359567
:10AB3000279509811A81200F311F442737FD409541
:10AB4000542F0E94876B97FDB1C226E0959587959B
:10AB5000779567952A95D1F79B016C157D050CF4C7
:10AB60006B01309521953F4FC216D3060CF4690155
:10AB70008091D9049091DA048301081B190B10937A
:10AB8000470900934609AA2009F423C22B813C817E
:10AB9000281B390BC901AA2797FDA095BA2F209130
:10ABA0006105309162054091630550916405820F03
:10ABB000931FA41FB51F8093610590936205A09316
:10ABC0006305B093640560916105709162058091A1
:10ABD00063059091640561303AEF730730E08307B5
:10ABE00030E0930774F080E09AEFA0E0B0E080934B
:10ABF000610590936205A0936305B0936405BC0161
:10AC0000CD01603046E074074FEF84074FEF9407A3
:10AC100074F480E096E0AFEFBFEF8093610590930E
:10AC20006205A0936305B0936405BC01CD01970153
:10AC3000442737FD4095542F0E94FB6B7801E20EAC
:10AC4000F31E6B2D77278827992728AD39AD37FD5F
:10AC500043C237FD3EC235952795A981BA812A0F97
:10AC60003B1F442737FD4095542F0E94876B97FD6B
:10AC70002BC216E095958795779567951A95D1F72C
:10AC80009B016E157F050CF47B01309521953F4F9C
:10AC9000E216F3060CF479018601222717FD2095B0
:10ACA000322F0D871E872F87388B242D33273DABFE
:10ACB0002CAB452D55275FAB4EABB6E9CB2EB9E09B
:10ACC000DB2E03ED15E02701662457FC6094762CFB
:10ACD00068AD79AD4B01AA2497FCA094BA2CABE0E7
:10ACE0003A2EF7E7EF2EF9E0FF2E07C0FBAFEAAFF1
:10ACF000EAADD601EC930C94B561F80125851216E6
:10AD00000CF08FC049815A81CA01AA2797FDA095EE
:10AD1000BA2F332727FD3095432F532FBC01CD0188
:10AD20000E94876B97FD91C0E6E095958795779592
:10AD30006795EA95D1F77BAF6AAFF8018685282F32
:10AD4000332727FD3095432F532F6D857E858F85C3
:10AD500098890E94876B97FD73C056E095958795FB
:10AD6000779567955A95D1F72AAD3BAD260F371FDA
:10AD70003BAF2AAFF8018785282F332727FD309571
:10AD8000432F532FC301B2010E94876B97FD51C01F
:10AD900046E095958795779567954A95D1F72AADC1
:10ADA0003BAD260F371F3BAF2AAFF8018089282F14
:10ADB000332727FD3095432F532FC501B4010E943F
:10ADC000876BDC01CB01B7FD30C036E0B595A795A8
:10ADD000979587953A95D1F7F701608171812AADF2
:10ADE0003BAD820F931F0E945C31D7018D939C93E2
:10ADF00097FD24C095958795959587959BAF8AAFCC
:10AE0000ECA9FDA98E179F070CF470CF2EA93FA9BE
:10AE10004AAD5BAD241735070CF06ACF3BAF2AAFC4
:10AE200067CFD6011C920C94B561CF96A11DB11DC0
:10AE3000CCCF615C7F4F8F4F9F4FAACF0396DACF65
:10AE4000615C7F4F8F4F9F4F88CF615C7F4F8F4FEB
:10AE50009F4F6ACFA090A409B090A50980917E056C
:10AE6000815008F09ECB88E180937E058091F808A0
:10AE70009927880F991F880F991F7C010027F7FCDD
:10AE80000095102F69897A898B899C89A80197017F
:10AE90000E94FB6B30932608209325086FA178A5AC
:10AEA00089A59AA5A80197010E94FB6B30932808F9
:10AEB00020932708809193099091940997FDEAC403
:10AEC000959587959595879590932A08809329085D
:10AED0008091AF099091B00997FDDAC49595879557
:10AEE0009595879590932C0880932B08B0922E0807
:10AEF000A0922D088091D0049091D104A091D20409
:10AF0000B091D304BC01CD0125E030E040E050E039
:10AF10000E94FB6B3093300820932F0880916908C2
:10AF200090916A089093320880933108D092360845
:10AF3000C092350880912703909128039093380898
:10AF4000809337088091DE04992790933A08809384
:10AF500039088091AB099091AC09A091AD09B091ED
:10AF6000AE09209186033091870340918803509168
:10AF70008903BC01CD010E94FB6B30933C082093F8
:10AF80003B08809110049091110490934A0880939B
:10AF9000490880917E07992790934C0880934B082D
:10AFA0008091F7039091F80390934E0880934D0899
:10AFB0008091BF059091C0059093620880936108CD
:10AFC0008091BD059091BE059093640880936308BD
:10AFD000EACAC801AA2797FDA095BA2FE0CDC801FB
:10AFE000AA2797FDA095BA2F40CD68AD79AD613500
:10AFF000710524F080E590E099AF88AFA8ADB9ADB8
:10B00000A05BBF4F0CF0FDCC00EB1FEF19AF08AFFA
:10B01000F8CC9093A5098093A4090CCCD09249094F
:10B02000C0924809F1CB5092580940925709D6CBAB
:10B03000AFEF08331A070CF020CB08E31FEF19CB52
:10B0400098E389169FEF99060CF009CBA8E38A2EA6
:10B05000AFEF9A2E00CB1C821B82F1CA222433242C
:10B06000D1CAE092F904F092FA040093FB04109321
:10B07000FC041AC9D092CB04C092CA047093C904CC
:10B080006093C80449C82FE330E040E050E0E20E8E
:10B09000F31E041F151F66CB215C3F4F4F4F5F4FC0
:10B0A00041CB215C3F4F4F4F5F4F0FCB615C7F4FD8
:10B0B0008F4F9F4F4ACD2F5F3F4F39CD3095219510
:10B0C0003F4F33CD0396BBC8615C7F4F8F4F9F4F7F
:10B0D000D0CD2F5F3F4FBFCD309521953F4FB9CD9C
:10B0E00061507E4F8F4F9F4F96C8222733272A19D2
:10B0F0003B0983C88091AD0482608093AD040C94B9
:10B10000B1461092D6041092D5040C9447454D5F79
:10B110005F4F0C94A3444D5F5F4F0C9459440196CC
:10B120005DCC8091F808E82EFF240027112769895B
:10B130007A898B899C89A80197010E94FB6B390150
:10B140004A018091930990919409AA2797FDA095AF
:10B15000BA2F681A790A8A0A9B0A6FA178A589A56D
:10B160009AA5A80197010E94FB6B59016A01809181
:10B17000AF099091B009AA2797FDA095BA2FA81AF8
:10B18000B90ACA0ADB0AD401C30197FCF3C43C0123
:10B190004D0154E095948794779467945A95D1F72C
:10B1A000D601C501D7FCF2C45C016D0144E0D59421
:10B1B000C794B794A7944A95D1F78091B20490911F
:10B1C000B304813491050CF4C5C3C401B30123E079
:10B1D00030E040E050E00E94FB6B39014A01C601BB
:10B1E000B50123E030E040E050E00E94FB6B5901E4
:10B1F0006A018091E408E82FFF27EE0FFF1FE15559
:10B20000F74F808191810190F081E02DF7FDBAC464
:10B210007A97A4F0C401B30123E030E040E050E0AD
:10B220000E94FB6B39014A01C601B50123E030E001
:10B2300040E050E00E94FB6B59016A0171E2671621
:10B240007104810491042CF030E2632E712C812C66
:10B25000912C80EE68168FEF78068FEF88068FEFBF
:10B26000980644F420EE622E2FEF722E2FEF822EDE
:10B270002FEF922E91E2A916B104C104D1042CF053
:10B2800090E2A92EB12CC12CD12CA0EEAA16AFEFC2
:10B29000BA06AFEFCA06AFEFDA0614F00C949C4E74
:10B2A00080EEA82E8FEFB82E8FEFC82E8FEFD82EFE
:10B2B0000C949C4E8091D0049091D104A091D20422
:10B2C000B091D304F4E0880F991FAA1FBB1FFA9511
:10B2D000D1F78093130490931404A0931504B093B2
:10B2E0001604109211041092100421503040309333
:10B2F0004405209343054AA141FF3EC080919E032F
:10B30000823308F051C38091CB03815098F410929E
:10B31000EA048091D0049091D104A091D204B0911C
:10B32000D3048093CC049093CD04A093CE04B09327
:10B33000CF0481E08093CB0341C010927C05ED2DBA
:10B34000FF27EE0FFF1FE155F74F808191818C346D
:10B3500091050CF499C280917D058F5F893C08F4BA
:10B360001FC31092D40488EC80937D051092AF0423
:10B370001092AE040C94254420919E0380918A0380
:10B3800090918B03820F911D2091EE083327829FAD
:10B39000B001839F700D929F700D1124CB01AA27DD
:10B3A00097FDA095BA2F8093CC049093CD04A093E1
:10B3B000CE04B093CF0481E08093EA04E09086034A
:10B3C000F0908703009188031091890369897A8935
:10B3D0008B899C89A80197010E94FB6B59016A0126
:10B3E0006FA178A589A59AA5A80197010E94FB6B7A
:10B3F000B901C5010E94766A6C01CD971CF0ECE39F
:10B40000CE2ED12CC6010E941C696C018091EA04E9
:10B41000882309F469C18091AD0499279C012071AA
:10B42000307084FD61C1B0903909B0FC04C08091D6
:10B43000E90881FD5DC409811A8130939B05209341
:10B440009A056090D0047090D1048090D2049090BE
:10B45000D3048091CC049091CD04A091CE04B091FE
:10B46000CF0486159705A805B90514F0B0FC52C1A4
:10B47000E090D004F090D1048091CC049091CD0460
:10B48000E81AF90A80919D0399278E9D90018F9D5E
:10B49000300D9E9D300D1124C90137FDDAC59595FB
:10B4A0008795959587959595879595958795081B8B
:10B4B000190B209110043091110437FDC7C5359543
:10B4C00027953595279535952795293031050CF425
:10B4D000CCC328E030E0229FA001239F500D329F73
:10B4E000500D11249A0157FDAEC535952795359518
:10B4F00027958091100490911104280F391F809195
:10B500009F039927AA27BB27442737FD4095542F2F
:10B51000BC01CD010E94876B97FD90C5B7E0959562
:10B52000879577956795BA95D1F79B015FEF61385D
:10B5300075070CF092C321E83FEF021B130B6090DC
:10B54000F1047090F2048090F3049090F40497FC5E
:10B5500064C5A7E09594879477946794AA95D1F7EA
:10B5600080919C03282F332744275527C401B3011A
:10B570000E94876B97FD4CC5F5E09595879577956B
:10B580006795FA95D1F79B017FEF213837070CF0CB
:10B590004BC321E83FEF021B130B85E990E0E80E57
:10B5A000F91E9BE2E91691E0F906E8F480919A050C
:10B5B00090919B05892BB9F480919E0590919F05F0
:10B5C0001816190684F48091A0059091A10508171A
:10B5D00019070CF49FC28091C9039091CA03801788
:10B5E00091070CF497C28091430590914405892BF3
:10B5F00021F000919E0510919F0580919A03992753
:10B60000AA27BB272091180A332727FD3095432FFF
:10B61000532FBC01CD010E94876B97FD0AC5E7E05F
:10B620009595879577956795EA95D1F79B01AFEF4B
:10B6300061387A070CF0F0C221E83FEF021B130BD0
:10B64000C801AA2797FDA095BA2F5DE0880F991F22
:10B65000AA1FBB1F5A95D1F79601442737FD409585
:10B66000542FBC01CD010E94FB6B20936D053093DC
:10B670006E0540936F055093700500916D05109114
:10B680006E0580919C0590919D059C01220F331FB2
:10B69000280F391F200F311F37FDC8C4A901559548
:10B6A000479555954795BA018091EA08282F332789
:10B6B000220F331F220F331F421753070CF0BCC257
:10B6C000A901B9015090A309B0FE64C2E981FA81D1
:10B6D000E417F5070CF05EC2AF01F0939D05E0930F
:10B6E0009C055A83498318C06091F208662309F4C7
:10B6F0003AC17727663471050CF00EC226E430E0BB
:10B700003093C8032093C703E980FA80F0929D0527
:10B71000E0929C055090A3098091AD0481FFA7C0E1
:10B720008091AD0484FDA3C0E090A205F090A30534
:10B730000091A4051091A505E114F104010511057E
:10B74000B1F429813A8179010027F7FC0095102F87
:10B75000ECE0EE0CFF1C001F111FEA95D1F7E09200
:10B76000A205F092A3050093A4051093A50580916E
:10B77000100490911104809110049091110497FD90
:10B78000EEC3843691050CF072C069817A819B0109
:10B79000442737FD4095542FC601AA2797FDA09551
:10B7A000BA2FBC01CD010E94876B97FD6CC49B0131
:10B7B000AC017DE055954795379527957A95D1F75A
:10B7C00020936D0530936E0540936F05509370057F
:10B7D0008091AE049091AF0477E0803D970708F028
:10B7E00053C3D801C70169E0B695A795979587958A
:10B7F0006A95D1F7E81AF90A0A0B1B0BDA01C9019D
:10B8000023E0880F991FAA1FBB1F2A95D1F7E80EC6
:10B81000F91E0A1F1B1FE092A205F092A3050093D8
:10B82000A4051093A505D801C7011CE0B695A795FE
:10B83000979587951A95D1F790939F0580939E05CC
:10B840004091F008442309F414C355279C01BA0120
:10B850000E94C66BC901861B970B9093A10580932C
:10B86000A005260F371F3093CA032093C903A09069
:10B87000A409B090A509809057099090580960904C
:10B8800048097090490951C810927D050C942544CF
:10B89000039624CB039614CB909581959F4F0C94DF
:10B8A0006F4503960C94734503960C94874F9095BF
:10B8B00081959F4F0C94834F4F960C944652882746
:10B8C00099278A199B090C94F951695F7F4F0C9451
:10B8D000AE51709561957F4F0C94A15181509E4F50
:10B8E000AF4FBF4F0C94805181509E4FAF4FBF4F11
:10B8F0000C949551909581959F4F9BAF8AAF0C9476
:10B900008D5184EF91E09093AB038093AA030C9444
:10B91000CB528AAD9BAD909581959F4F6817790763
:10B9200014F00C94B252BC010C94B2520894210849
:10B9300031083092AB032092AA030C94CB52F095BD
:10B94000E195FF4F0C94584E61507E4F8F4F9F4FA3
:10B950000C94184E8091B0049091B10481349105FB
:10B960000CF447CC32CC40919E0550919F0557FD79
:10B97000B8C1559547955595479580912703909166
:10B980002803209100013327489F5001499FB00CA4
:10B99000589FB00C1124C501B9010E94C66BAACEF4
:10B9A00080937D050C94254481E08093EA0488EC23
:10B9B0008093CB0303CD80937C05C1CC87B5853FB5
:10B9C00008F0F3C08091120481500C947C54808163
:10B9D0009181855B9F4F0CF0F2C080917B058F5F5A
:10B9E00080937B05893C10F40C94A8472C3008F018
:10B9F0007EC32998A4E0B0E08FEF082E0E94236C4C
:10BA00001092D40410927B051092AF041092AE04F1
:10BA10000E94D53CA4E0B0E08091370590913805B4
:10BA200097FD41C4892F990F990B082E0E94236C12
:10BA3000A5E0B0E08091370590913805082E0E946E
:10BA4000236CA6E0B0E0809135059091360597FD16
:10BA500027C4892F990F990B082E0E94236CA7E009
:10BA6000B0E08091350590913605082E0E94236C38
:10BA700008E010E080912F0590913005A0913105EC
:10BA8000B0913205BC01CD010E94F06ADC01CB010E
:10BA90009C0197FDCDC3832F992787FD9A95D801E7
:10BAA000082E0E94236C09E010E080912F059091F0
:10BAB0003005A0913105B0913205BC01CD010E9445
:10BAC000F06ADC01CB01D801082E0E94236C0E9491
:10BAD000B50568E770E00E948E313091E3080C9460
:10BAE000A847C601AA2797FDA095BA2FBC01CD0192
:10BAF0002D8D3E8D4F8D58A10E94876B3B014C01CF
:10BB00000E94FB6B3093EE042093ED0410927F05AE
:10BB10000C941A528C0167CD6739710534F186E9AE
:10BB200090E09093C8038093C703EECD0196A11DCA
:10BB3000B11D0C94414E0196A11DB11D0C94354EC2
:10BB400081E080937F051092650510926605109242
:10BB50006705109268051092F9041092FA04109289
:10BB6000FB041092FC040C94B1467093C8036093DC
:10BB7000C703CACD0F96A11DB11D09CB095F1F4F89
:10BB80000C946B52F095E195FF4F42CB0F96A11D9F
:10BB9000B11D0ACB70939D0560939C055A83498320
:10BBA000BBCD80937B050C94A84781E08093A705CB
:10BBB000A2CB3F893093A6053093A7059CCB409339
:10BBC0007B050C94A847B0928D05A0928C0520911E
:10BBD000150A2C8F0C942F4B10928E050C94954BBC
:10BBE00020938405309385054093860550938705FF
:10BBF000109290050C94FC4C2092800530928105A7
:10BC0000409282055092830510928F050C94064C49
:10BC1000109291050C946E4D6F3F710509F00CF474
:10BC20000DCD2FEF30E00ACD2F3F310509F00CF498
:10BC3000B2CC2FEF30E0AFCC5090A309252D3327A5
:10BC4000220F331F220F331F205530402417350792
:10BC50000CF03ACDA901B90137CD6F3F710509F05C
:10BC60000CF46BCC2FEF30E068CC121613060CF4FA
:10BC700032CC229FC001239F900D329F900D112442
:10BC800097FD6DC39595879595958795209110049F
:10BC900030911104281B390B32CC0E94B50545E6C2
:10BCA00061EE78E00E945D058091E90880FF10C098
:10BCB00080911D0390911E03875B934038F480911F
:10BCC0001D0390911E038E5E924010F40E94711C21
:10BCD0001092F9030E94D53C81E08093F903579AB2
:10BCE000F6CE4D5F5F4F45CE81E08093A60503CB36
:10BCF0008091AD0481FFD1C12091C7033091C80369
:10BD0000C9010F964091D5045091D6048417950728
:10BD10000CF0EFC18091A605882309F0EAC180915B
:10BD2000A80581FFF8C28D7F6090D0047090D10487
:10BD30008090D2049090D3046092CC047092CD0491
:10BD40008092CE049092CF0481608093A805421B1C
:10BD5000530B9A012F50304037FDF4C280919A0561
:10BD600090919B05280F391F30939B0520939A05CE
:10BD700020919A0530919B05C90137FF04C088279F
:10BD80009927821B930B815092400CF481C18091C2
:10BD9000EE089927829FF001839FF00D929FF00D8E
:10BDA0001124CF0160E075E00E94C66BCB01AA2789
:10BDB00097FDA095BA2F2091CC043091CD044091ED
:10BDC000CE045091CF04820F931FA41FB51F809300
:10BDD000CC049093CD04A093CE04B093CF041092E2
:10BDE0009B0510929A05B1FE06C08BE490E09093FB
:10BDF000FC038093FB038091F208882309F048C17B
:10BE000000919E0510919F05A80117FD93C25595BD
:10BE10004795559547958091270390912803209148
:10BE200000013327489F7001499FF00C589FF00C88
:10BE30001124C701B9010E94C66B663471050CF06C
:10BE400073C226E430E03093C8032093C703809187
:10BE5000430590914405892B09F4FBCAD401C30121
:10BE60006092CC047092CD048092CE049092CF0464
:10BE7000F8CA1092A1051092A0058FEF93E090935D
:10BE8000CA038093C903F3CCAFE0803A9A0708F065
:10BE9000E2C0D801C701FAE0B695A79597958795B6
:10BEA000FA95D1F7E81AF90A0A0B1B0BDA01C90156
:10BEB000880F991FAA1FBB1F880F991FAA1FBB1F9E
:10BEC000A6CC1091E2080C940B4720938405309384
:10BED0008505409386055093870510928D05109235
:10BEE0008C05E8EE2E2EE3E03E2E3092AB0320923E
:10BEF000AA030C946E4D6092800570928105809229
:10BF000082059092830510928D0510928C0588EE23
:10BF1000282E83E0382E3092AB032092AA030C9493
:10BF2000064C7093C9046093C804D092CB04C092AD
:10BF3000CA04CB0177FD6BC1BC0175956795C6013D
:10BF4000D7FC63C16C01D594C7940C94494A299AD3
:10BF50000C94DF4681E0809391050C946E4D909592
:10BF600081959F4F0ECCB095A095909581959F4F50
:10BF7000AF4FBF4F0C94FD4A209384053093850545
:10BF8000409386055093870581E0809390050C943B
:10BF9000FC4CB095A095909581959F4FAF4FBF4FAA
:10BFA0000C945F4C2092800530928105409282056E
:10BFB0005092830581E080938F050C94064C81504C
:10BFC0009F4FAF4FBF4F0C94A04981509F4FAF4F31
:10BFD000BF4F0C94864981509F4FAF4FBF4F0C9479
:10BFE0001B4A81509F4FAF4FBF4F0C940E4A615078
:10BFF0007F4F8F4F9F4F0C94DE4961507F4F8F4F83
:10C000009F4F0C94C84981E080938E050C94954B0A
:10C01000615E7F4F8F4F9F4FAFCA6FE770E080E048
:10C0200090E0660E771E881E991E93CA2D5F3F4FC3
:10C0300035CB61587F4F8F4F9F4FF1CA61587F4F6B
:10C040008F4F9F4F6BCA2D5F3F4F4FCA295F3F4FA6
:10C0500036CA0F9624CA80549F4108F096C0D80172
:10C06000C7017BE0B695A795979587957A95D1F707
:10C07000E81AF90A0A0B1B0BDA01C901820F931F98
:10C08000A41FB51FC4CB6150704E8F4F9F4F8FCBF5
:10C0900000919E0510919F05DACE6090D0047090BB
:10C0A000D1048090D2049090D304D401C30180596C
:10C0B0009140A040B0408093CC049093CD04A093D5
:10C0C000CE04B093CF042091F208222309F446C095
:10C0D00033273093C8032093C70300919E05109126
:10C0E0009F05BFC9F095E195FF4F0C948A47299AA7
:10C0F00081CCC9010F97481759070CF058C080919F
:10C10000A705882309F053C08091A80580FF1EC1B0
:10C110008E7F6090D0047090D1048090D204909073
:10C12000D3046092CC047092CD048092CE0490929D
:10C13000CF0482608093A805421B530B9A01215FB4
:10C140003F4F37FD0EC180919A0590919B05821B50
:10C15000930B90939B0580939A050ACE28E730E0D5
:10C16000B8CF20938405309385054093860550937E
:10C1700087050C94E44C2093840530938505409307
:10C180008605509387050C94564DD801C7016CE085
:10C19000B695A795979587956A95D1F7E81AF90A04
:10C1A0000A0B1B0BE20EF31E041F151F34CB20914C
:10C1B000A805822F992783709070892B81F12C7F9D
:10C1C0002093A80510929B0510929A056090D004C8
:10C1D0007090D1048090D2049090D3046092CC04EB
:10C1E0007092CD048092CE049092CF04B1FEC0CD67
:10C1F00084EF91E09093FC038093FB03B9CD8150D1
:10C200009F4FAF4FBF4F0C94F04C01969BCE0196C1
:10C2100093CE295F3F4F4F4F5F4F0C94394D609045
:10C22000D0047090D1048090D2049090D304A0CD1B
:10C2300021503F4F30CC295F3F4F4F4F5F4F0C9401
:10C24000C74C81509E4FAF4FBF4F0C94B24C8150A2
:10C250009F4FAF4FBF4F0C94FA4BB095A095909560
:10C2600081959F4FAF4FBF4F0C94B34B295F3F4F0A
:10C270004F4F5F4F0C946B4B21503E4F4F4F5F4FD2
:10C280000C94524BB095A095909581959F4FAF4FD0
:10C29000BF4F0C944C4BF095E195FF4F0C94074722
:10C2A00081509F4FD6CB81509F4FBCCB81509F4F29
:10C2B000AF4FBF4F0C94624DF095E195FF4F0C943A
:10C2C000414A21503E4F4F4F5F4F0C94204DB09547
:10C2D000A095909581959F4FAF4FBF4F0C941A4DED
:10C2E00081509F4FAF4FBF4F0C948D4BB095A09591
:10C2F000909581959F4FAF4FBF4F0C94AE4C295FE7
:10C300003F4F4F4F5F4F0C94D24B21503E4F4F4FFA
:10C310005F4F0C94B94B6090D0047090D104809022
:10C32000D2049090D30410CD6739710534F026E91A
:10C3300030E089CD4D5F5F4F6ACD7093C803609345
:10C34000C70385CD309521953F4F08CD6090D0042F
:10C350007090D1048090D2049090D304EACE0396DA
:10C3600091CC309521953F4FEECE3A94E2E0F0E04B
:10C37000EE0EFF1E0C5F1F4F0894C11CD11C37FC32
:10C3800002C00C947D56ED960FB6F894DEBF0FBE3A
:10C39000CDBFDF91CF911F910F91FF90EF90DF9074
:10C3A000CF90BF90AF909F908F907F906F905F9055
:10C3B0004F903F902F9008958091B5059091B605CC
:10C3C000A091B705B091B8058093AD059093AE05E7
:10C3D000A093AF05B093B0058091B1059091B205DF
:10C3E000A091B305B091B4058093A9059093AA05D7
:10C3F000A093AB05B093AC0508951092C0051092C0
:10C40000BF051092BE051092BD05089584B1806AE3
:10C4100084B93D9A82E58CBD1DBC459A81E080932C
:10C42000B5098AEA8093B90983E88093BA099AE04A
:10C430009093BB091092BD091092BC091092BF09DC
:10C440001092BE091092170A1092DB091092DC09B3
:10C450008CE48093DD0986E08093DE099093DF0908
:10C460000895EF92FF920F931F938091F8089927F8
:10C47000880F991F880F991F7C010027F7FC0095F2
:10C48000102F8091290590912A05A0912B05B0913C
:10C490002C05BC01CD01A80197010E94FB6B3093D4
:10C4A000BD092093BC098091210590912205A0919E
:10C4B0002305B0912405BC01CD01A80197010E947C
:10C4C000FB6B3093BF092093BE092091AB093091DB
:10C4D000AC094091AD095091AE09DA01C901E3E020
:10C4E000880F991FAA1FBB1FEA95D1F7820F931FD0
:10C4F000A41FB51F820F931FA41FB51F2091860391
:10C50000309187034091880350918903BC01CD018C
:10C510000E94FB6B3093C5092093C409E091330559
:10C52000F091340580916D0990916E09BF010E94D0
:10C53000C66BCB019B01220F331F220F331F280F25
:10C54000391F280F391F37FD1CC1359527953595A3
:10C5500027953093C1092093C0098091A709909134
:10C56000A809BF010E94C66B9B01220F331F220F37
:10C57000331F260F371F260F371F37FDFFC0359596
:10C580002795359527953093C3092093C2091092BA
:10C5900034051092330510926E0910926D091092B5
:10C5A000A8091092A7098091BB0999278C309105A1
:10C5B00009F4A1C08D3091050CF069C08A30910555
:10C5C00009F4A4C10B9709F410C18091DB098823F9
:10C5D00009F4CBC02091E1093091E209C9018150F1
:10C5E0009E4F8F5F9340C8F44091E3095091E40956
:10C5F000CA0181509E4F8F5F934078F48091E90883
:10C6000085FF0BC03093C0052093BF055093BE0536
:10C610004093BD058AEF8093C2058091E709909110
:10C62000E80921E0893692070CF056C19C019093ED
:10C63000F0048093EF048091ED049091EE04281BA8
:10C64000390BC901845E9D4F68E671E00E94C66B9C
:10C65000845B90409093EC048093EB042091EB0971
:10C660003091EC098091FB039091FC0382179307B2
:10C6700040F480917E07882321F43093FC032093BB
:10C68000FB038091E009873609F0ADC12AC18E30E5
:10C69000910509F476C18E3091050CF475C00F97A1
:10C6A00009F093CF809110098093CC0980913809CB
:10C6B0008093CD09809192038093CE0980910909DE
:10C6C0008093CF0980910A098093D00980910B094A
:10C6D0008093D109809191038093D20980910D09B3
:10C6E0008093D30980910E098093D40980910F091A
:10C6F0008093D5096ACF80917E07863018F010921A
:10C700007E0785E08093CC09809135098093CD091F
:10C7100080912F08909130089093CF098093CE0993
:10C720008091CC049091CD04A091CE04B091CF041F
:10C73000BC01CD0125E030E040E050E00E94FB6B01
:10C740003093D1092093D00980912B098093D2098D
:10C7500080912C098093D30980912D098093D4096D
:10C760008091DB09882309F035CF1092C005109223
:10C77000BF051092BE051092BD0535C12D5F3F4F1C
:10C78000FECE2D5F3F4FE1CE809126098093CC09EC
:10C79000809127098093CD09809128098093CE0943
:10C7A000809129098093CF0980912A098093D0092B
:10C7B00080912E098093D10980912F098093D2090D
:10C7C000809130098093D309809133098093D409F3
:10C7D000809131098093D509809132098093D609DF
:10C7E000809134098093D709F0CEF8948091E308C2
:10C7F000E82FFF27EE0FFF1FE155F74F0190F08163
:10C80000E02DE038F1050CF0D1C02FEFE138F20750
:10C8100014F4E1E8FFEFE093CC098091E408E82FFD
:10C82000FF27EE0FFF1FE155F74F0190F081E02D3C
:10C83000E038F1050CF4CDC0EFE7F0E0E093CD096E
:10C840008091E208E82FFF27EE0FFF1FE155F74F19
:10C850000190F081E02DE038F1050CF4B2C0EFE773
:10C86000F0E0E093CE098091E108E82FFF27EE0F7A
:10C87000FF1FE155F74F0190F081E02DE038F10501
:10C880000CF497C0EFE7F0E07894E093CF09809143
:10C89000E5048093D0098091E3048093D1098091CD
:10C8A000E1048093D2098091DF048093D3098091C1
:10C8B000DE048093D4098091DD048093D5098091B2
:10C8C00033089091340897FD8CC095958795959580
:10C8D00087958093D60979CE2091EF043091F004AA
:10C8E000AACE8091ED098093140A8091EE0980937D
:10C8F000160A8091EF098093150A8091F0098093C0
:10C90000170A8091F1098093180A6DC08091C104C3
:10C910008093CC098091C0048093CD098091BF049D
:10C920008093CE098091BE048093CF098091BD048D
:10C930008093D0098091BC048093D1098091BB047D
:10C940008093D2098091BA048093D3098091AD0479
:10C950008093D4098091AD04837F8093AD0480914E
:10C960002703909128038093D5098091000180933B
:10C97000D609A2E0B0E00E94166C802D8093D70902
:10C9800024CE8091DC098093CC098091DD098093CD
:10C99000CD098091DE098093CE098091DF098093D3
:10C9A000CF09809102018093D0090FCEEFE7F0E02C
:10C9B00032CF8FEFE138F8070CF066CFE1E8FFEFF8
:10C9C00063CF6FEFE138F6070CF04BCFE1E8FFEFF4
:10C9D00048CF4FEFE138F4070CF030CFE1E8FFEF3C
:10C9E0002DCF039672CF1F910F91FF90EF90089576
:10C9F0008091B509882309F43BC0459889EB99E0FB
:10CA00009093B7098093B6098091C105E82FFF275D
:10CA1000E453FC4F982F9F5F80818093BB09973030
:10CA200008F027C09093C1051092B5090E943162A9
:10CA300081E08093B80900000000000000000000C1
:10CA400000000000000000000000000000000000E6
:10CA500000000000000000000000000000000000D6
:10CA60000000000000008091B9098093D8098EBDB4
:10CA700008951092C105D8CF2091B509222309F05D
:10CA800045C00DB407FE42C084E08093FA03459A86
:10CA90003EB58091C30599278130910509F437C0CF
:10CAA000823091050CF451C0029709F439C02091ED
:10CAB000B809203208F030C045980000000000009E
:10CAC0000000000000000000000000000000000066
:10CAD0000000000000000000000000000000000056
:10CAE00000000000000000000000E091B609F09195
:10CAF000B709E20FF11D80818EBD8091D809908128
:10CB0000890F8093D8092F5F2093B8090895353590
:10CB100051F12093C305CBCF81E08093B509F3CFCA
:10CB20008091DA09E82FFF27E650F64F30838F5FB8
:10CB30008093DA098A3100F18091C405381711F128
:10CB40002093DB091092C305B2CF892B09F0AFCF38
:10CB50002093DA093093C405313809F0A8CF81E079
:10CB60008093C305A4CF8091C405830F8093C4052F
:10CB700082E08093C3059BCF8091C405830F80938F
:10CB8000C40595CF8AE1EAEFF9E0A0EEB9E00190A3
:10CB90000D928A95E1F781E08093DB091092C3053D
:10CBA00086CF87B18C6087B9429843981092C605AA
:10CBB00080E88093D4031092C5058093D303089531
:10CBC0008091CB0581508F3F19F08093CB0508955C
:10CBD00084E08093CB058091AD0485FF16C0409121
:10CBE00024094093CC05609125096093CD055091AF
:10CBF0003709252F332724FF13C08091D4048823BD
:10CC000079F425FF17C0429A33C08091DE0488234F
:10CC100034F7409120094093CC0560912209E5CF7B
:10CC2000909121099B3FB8F080916F098D3D98F05C
:10CC300047FDE9CF4298252F332724FD1DC0909151
:10CC400023099B3F08F18091A209873EE8F067FD28
:10CC500019C0439808959B3F20F080916F098A3056
:10CC600008F18091C60581508F3F21F18093C60560
:10CC7000252F332724FFE3CF8091D4048823F9F6AE
:10CC800026FFE7CF439A08959B3F20F08091A209A9
:10CC90008A3060F08091C50581508F3FE1F080932C
:10CCA000C505089547FDC6CF429AE2CF67FDD1CFB3
:10CCB000439A089580916F0981508093C6058091B1
:10CCC000D4038130C9F086958093D403842309F47A
:10CCD000B1CF429ACDCF8091A20981508093C505F2
:10CCE0008091D303813051F086958093D3038623BE
:10CCF00009F4AFCF439A089580E8E6CF80E8F5CFF6
:10CD00008091C9008F778093C9008091C9008F7B83
:10CD10008093C9008091C9008F7D8093C9005A9A81
:10CD200052981092CD0084E190E08093CC008091E5
:10CD3000C80082608093C80080E18093C900809120
:10CD4000CA008F778093CA008091CA008F7B80933E
:10CD5000CA008091CA008F7D8093CA008091CA006A
:10CD60008F7E8093CA008091CA00877F8093CA001B
:10CD70008091C9008B7F8093C9008091CA00846034
:10CD80008093CA008091CA0082608093CA0080911B
:10CD9000C80087FF0CC08091CE008091C800882316
:10CDA00034F48091CE008091C8008823A4F3809150
:10CDB000C90080688093C90008951F93CF93DF93C3
:10CDC00080E197E20E94F517EC0110E08091C90024
:10CDD0008F778093C9008091C9008F7E8093C900AE
:10CDE0005A9888E298E09F938F931F930E9476143D
:10CDF0000F900F900F90CE010E94FE17882309F02C
:10CE000066C04A9BF8CF8AE590E00E94F517EC01D6
:10CE10008EE598E09F938F931F920E947614529A0A
:10CE20000F900F900F90CE010E94FE178823D9F328
:10CE300083E690E05A9A019797FFFCCF8FE891E044
:10CE40005A98019797FFFCCF89E090E05A9A019792
:10CE500097FFFCCF89E090E05A98019797FFFCCFAD
:10CE60008FE891E05A9A019797FFFCCF8FE891E005
:10CE70005A98019797FFFCCF89E090E05A9A019762
:10CE800097FFFCCF89E090E05A98019797FFFCCF7D
:10CE90008FE891E05A9A019797FFFCCF8FE891E0D5
:10CEA0005A98019797FFFCCF89E090E05A9A019732
:10CEB00097FFFCCF89E090E05A98019797FFFCCF4D
:10CEC0008FE891E05A9A019797FFFCCF0AC084E659
:10CED00098E09F938F931F930E9476140F900F906A
:10CEE0000F9052985A980E948066DF91CF911F91BF
:10CEF00008951F920F920FB60F921124EF92FF9296
:10CF00000F931F932F933F934F935F936F937F9351
:10CF10008F939F93AF93BF93CF93DF93EF93FF9341
:10CF20002091CE008091D503813009F44BC08091CF
:10CF3000CE058823C9F040E050E08091CF058823DA
:10CF4000C9F4452B09F44AC081E08093CF05809154
:10CF5000D0058F5F8093D00543E08091D00580316C
:10CF6000E8F44093CE0504C141E050E08091CF0544
:10CF7000882339F3813009F44AC08230B9F1833013
:10CF800009F44AC081E08093D5031092D005109235
:10CF9000D20544E48091D005803118F38091D20508
:10CFA000882331F48091D503882311F4809384037E
:10CFB0001092D0051092D2051092CF0584E4809390
:10CFC000CE05D6C01092D50384E48093CE0510928E
:10CFD000D0051092CF051092D105CAC044E48093C9
:10CFE000D0058093CF058093D105D4CF452B51F642
:10CFF00043E02093D1059091D005923009F492C07E
:10D0000083E08093CF059F5F9093D005C3CF452BDE
:10D0100009F0B8CF82E099CF452B09F0B3CF482F64
:10D0200082E08093CF058091D0058F5F8093D005FB
:10D030009091D105892F86958695E82FFF27EF706F
:10D04000F0703196892F9927982F88273327822BC4
:10D05000932B93708050924063E070E00E94C66B07
:10D06000EB30F10508F057C07F01EE0EFF1EF7010F
:10D07000E155F74F808191819B01281B390BC90134
:10D0800037FD6EC0069754F48091DE04883C08F0AA
:10D090005BC08091DE04865F8093DE04F701E1557A
:10D0A000F74F808191819C01220F331F280F391F78
:10D0B000260F371F37FD51C0E901D595C795D59586
:10D0C000C795CB0101968C179D07BCF521978091E0
:10D0D000DE04843B60F187010B53174FF701E155E4
:10D0E000F74F80819181FE01E81BF90BCF0163E0CE
:10D0F00070E00E94C66BCB01880F991F860F971FA7
:10D10000F801918380832FEA38E0E20EF31EF701E5
:10D11000D183C0833FCF729708F43CCF81E08093E6
:10D12000D50338CF27FD20C01092D20569CFF70173
:10D13000EB53F74F11821082E6CF61507040C61753
:10D14000D7072CF62196C3CF88EC8093DE0480911C
:10D150006F008F7D80936F00A1CF2D5F3F4FACCFCD
:10D16000909581959F4F8ECF81E08093D20548CFD7
:10D17000FF91EF91DF91CF91BF91AF919F918F91EF
:10D180007F916F915F914F913F912F911F910F91DF
:10D19000FF90EF900F900FBE0F901F901895CF93B8
:10D1A000FC0197FD21C0C1E028E631E0CF01B901C3
:10D1B0000E94C66BFC018B35910554F08B55904055
:10D1C0008A35910538F484EB90E08E1B9F0BFC01AF
:10D1D00041E013C0CF01855B90408A35910548F44A
:10D1E000E45BF0404FEF09C0CFEFF095E195FF4FC2
:10D1F000DBCF2E1B3F0BF9014FEFEE0FFF1FE75365
:10D20000F64F259134918C2F992787FD9095829F19
:10D21000B001839F700D929F700D1124842F992768
:10D2200087FD9095689FA001699F500D789F500DD4
:10D230001124CA01CF9108952AE530E0281B390B4B
:10D24000C9010E94CF6808951F93CF93DF93EB012C
:10D250006115710519F4009709F494C097FD3EC05B
:10D2600011E0209729F48AE51802B00111248AC040
:10D27000AA2797FDA095BA2F26E0880F991FAA1F0D
:10D28000BB1F2A95D1F79E01442737FD4095542FA7
:10D29000BC01CD010E94FB6BF90137FD2CC081E080
:10D2A000EA35F807ACF08CE1E73AF807CCF02AE56C
:10D2B00030E01C161D061CF5812F992787FD9095DF
:10D2C000829FB001839F700D929F700D11245AC0F0
:10D2D000E159F74F8491282F3327EBCF1FEFC1CFB0
:10D2E00089E0ED38F8078CF485E0EA3BF80784F034
:10D2F00028E530E0DECFF095E195FF4FD0CFD7FDA8
:10D300000EC0B901645B70403DC029E530E0D1CF6B
:10D3100084E0E731F80754F027E530E0CACF111672
:10D3200084F764EB70E0621B730B2CC083E0EE3279
:10D33000F8071CF026E530E0BCCF82E0E939F807B9
:10D340001CF025E530E0B5CF82E0E233F8071CF0B1
:10D3500024E530E0AECF81E0E73EF8071CF023E59E
:10D3600030E0A7CF81E0ED3AF8071CF022E530E08D
:10D37000A0CFEF57F1401CF021E530E09ACF20E537
:10D3800030E097CFCB01DF91CF911F910895EF92BD
:10D39000FF920F931F93CF93DF937B018C0120E0CB
:10D3A00030E040E050E0FA01E9016FE00BC0C21B41
:10D3B000D30BE40BF50B2F5F3F4F4F4F5F4F615087
:10D3C00067FD31C0220F331F441F551FCC0FDD1FD7
:10D3D000EE1FFF1FCC0FDD1FEE1FFF1FD801C7017F
:10D3E0007EE1B695A795979587957A95D1F7C80F61
:10D3F000D91FEA1FFB1FEE0CFF1C001F111FEE0CB4
:10D40000FF1C001F111F2F5F3F4F4F4F5F4FC21771
:10D41000D307E407F50758F621503040404050400C
:10D42000615067FFCFCF5695479537952795CA012D
:10D43000B901DF91CF911F910F91FF90EF90089567
:10D44000002422273327442751E0BB27EE27FF275C
:10D45000A0E1660F771F881F991F001C221F331F32
:10D46000441F660F771F881F991F001C221F331F40
:10D47000441F2AF4050E2B1F3E1F4F1F04C0051A20
:10D480002B0B3E0B4F0B550FBB1FEE1F587F5560EC
:10D4900047FD5250AA95E9F6E695B7955795E6955A
:10D4A000B7955795852F9B2F08952227332741E065
:10D4B000552768E0880F991F221F331F880F991F77
:10D4C000221F331F1AF4240F351F02C0241B350BF3
:10D4D000440F551F487F456037FD42506A9551F70C
:10D4E0005695479556954795842F0895AA2797FFF7
:10D4F00004C0809590958A1F9A1F77FF04C060959D
:10D5000070956A1F7A1F669F9001779FA001679FA1
:10D51000300D411D5A1F300D411D5A1F889FF001CB
:10D52000999F2E0F3F1F401D511D899F300D411D9A
:10D530005A1F300D411D5A1FCA01B901112480CF55
:10D54000FC014150504030F001900616D1F7319760
:10D55000CF0108958827992708955058192EA6D0ED
:10D5600001D08CC0BA176207730784079507B1F121
:10D5700088F40EF410940B2EBA2FA02D062E622FD5
:10D58000202D072E732F302D082E842F402D092E8D
:10D59000952F502DFF275523B9F0591B49F0573EC1
:10D5A00098F0469537952795A795F0405395C9F77C
:10D5B00076F0BA0F621F731F841F30F4879577953A
:10D5C0006795B795F040939517FA0F2E0895BF1BF6
:10D5D000BB27BA0B620B730B840BF6CFDEF692C03F
:10D5E00097FB70D09F3738F0FEE9F91B982F872FF3
:10D5F000762F6B2F05C083C0969587957795679595
:10D60000F150D0F73EF490958095709561957F4FDD
:10D610008F4F9F4F0895E89403C097FB0EF4F3DFFC
:10D62000B62F672F782F892F9EE9002427C00ED0B0
:10D630005EF004C00BD026F001C008D019F020F431
:10D640008FEF089580E0089581E0089597FB092EFB
:10D65000052600F868942DD0E89407FC07C06217EF
:10D6600073078407950721F008F4009407949894B1
:10D6700008959A95BB0F661F771F881F1124992361
:10D68000A1F08823B2F79F3F59F0BB0F48F421F473
:10D69000002011F460FF04C06F5F7F4F8F4F9F4FDA
:10D6A000881F9795879597F9089529C0052E092613
:10D6B00007FA440F551F5F3F79F0AA27A51708F016
:10D6C00051E04795880F991F9F3F31F0BB27B9174D
:10D6D00008F091E0879508959F919F91112414C0BF
:10D6E00097FB880F991F9F3F31F0BB27B91708F0B0
:10D6F00091E0879508959F919F91112405C0662719
:10D7000077278827992708959FEF80EC0895629FD7
:10D71000D001739FF001829FE00DF11D649FE00D29
:10D72000F11D929FF00D839FF00D749FF00D659F8A
:10D73000F00D9927729FB00DE11DF91F639FB00D89
:10D74000E11DF91FBD01CF0111240895991B79E056
:10D7500004C0991F961708F0961B881F7A95C9F781
:10D7600080950895AA1BBB1B51E107C0AA1FBB1FD0
:10D77000A617B70710F0A61BB70B881F991F5A955D
:10D78000A9F780959095BC01CD01089597FB092ECE
:10D7900007260AD077FD04D0E5DF06D000201AF472
:10D7A000709561957F4F0895F6F7909581959F4FFD
:10D7B0000895A1E21A2EAA1BBB1BFD010DC0AA1FD2
:10D7C000BB1FEE1FFF1FA217B307E407F50720F0EA
:10D7D000A21BB30BE40BF50B661F771F881F991F65
:10D7E0001A9469F760957095809590959B01AC01AE
:10D7F000BD01CF01089597FB092E05260ED057FDD8
:10D8000004D0D7DF0AD0001C38F4509540953095ED
:10D8100021953F4F4F4F5F4F0895F6F790958095B4
:10D82000709561957F4F8F4F9F4F0895F999FECF67
:10D83000B2BDA1BDF89A119600B40895F7DF019228
:10D840001A94E1F70895F999FECFB2BDA1BD00BCCD
:10D8500011960FB6F894FA9AF99A0FBE08950190AE
:08D86000F2DF1A94E1F70895CC
:10D868005E010A0151756164726F0000416E676C58
:10D87800654E69636B20202020202020416E676C54
:10D8880065526F6C6C202020202020204163634E5D
:10D8980069636B20202020202020202041636352D0
:10D8A8006F6C6C2020202020202020204779726F68
:10D8B8004769657220202020202020204869676859
:10D8C800742056616C756520202020204163635ABE
:10D8D8002020202020202020202020204761732085
:10D8E800202020202020202020202020436F6D7021
:10D8F8006173732056616C7565202020566F6C74B7
:10D90800616765202020202020202020456D70663A
:10D91800616E672020202020202020204779726F08
:10D92800204B6F6D70617373202020204D6F746FD2
:10D93800722046726F6E7420202020204D6F746F05
:10D948007220526561722020202020204D6F746F54
:10D9580072204C6566742020202020204D6F746F43
:10D9680072205269676874202020202020202020FF
:10D97800202020202020202020202020202020209F
:10D98800202020202020202020202020566172697D
:10D998006F4D657465722020202020204D4B334D3B
:10D9A80061672043616C53746174652053657276B6
:10D9B8006F2020202020202020202020486F6F76F4
:10D9C80065726761732020202020202020202020DD
:10D9D800202020202020202020202020202020203F
:10D9E800202020202020202020202020202020202F
:10D9F800202020202020202020202020202020201F
:10DA0800202020202020202020202020202020200E
:10DA180020202020202020202020202020202020FE
:10DA28002020202020202020202020204932432D83
:10DA38004572726F72202020202020202020202074
:10DA48002020202020202020202020204750535F05
:10DA58004E69636B20202020202020204750535FF0
:10DA6800526F6C6C2020202020202020C8000164E8
:10DA7800FF01FFFF01FC01FC0101737373FF030049
:10DA88007D0000C409C40964000E48616C6C6F20F5
:10DA980057656C74000000000000000000000000E2
:10DAA800000000000000000000000000000000006E
:10DAB800000000000000000000000000000000005E
:10DAC800000000000000000000000000000000004E
:10DAD8000000000000000000000001020304050629
:10DAE8000708090A01040B050000ECFF6440415ACD
:10DAF8004664640A02969696960840403A10FB30AF
:10DB0800380190D0030090D00300F40164005370F2
:10DB18006F727400004E6F726D616C000042656731
:10DB2800696E6E657200007800FF03640A0B0D0BC6
:06DB38000C0E0F010101BB
:00000001FF
